:100000000C942B150C945C150C945C150C945C15DD
:100010000C945C150C945C150C945C150C945C159C
:100020000C945C150C945C150C945C150C945C158C
:100030000C945C150C945C150C945C150C945C157C
:100040000C945C150C945C150C945C150C945C156C
:100050000C945C150C945C150C9484490C94EDC2C2
:100060000C945C150C942DBD0C945C150C945C15D3
:100070000C945C150C944B480C945C150C945C151A
:100080000C94624A0C945C150C945C150C945C15F1
:100090000C945C150C945C150C945C150C9498579E
:1000A0000C945C150C945C150C945C150C945C150C
:1000B0000C945C150C945C150C945C150C941F4A04
:1000C0000C945C150C945C150C945C150C945C15EC
:1000D0000C945C150C945C150C945C150C945C15DC
:1000E0000C945C15FF4F0450095013501D509B5049
:1000F00027502F50375041504B50555064506E5040
:100100009B507D5087509150C050C350B250B65054
:10011000BC50FA50C750CB50D150D550D950DF50B9
:10012000E350E750FA50ED50F150F55092AD92ADDA
:1001300092AD50AD52AD6DAD70AD92AD92AD92AD90
:1001400092AD92AD084AD73B3BCE016E84BCBFFD59
:10015000C12F3D6C74319ABD56833DDA3D00C77F97
:1001600011BED9E4BB4C3E916BAAAABE0000008030
:100170003F05A84CCDB2D44EB93836A9020C50B9BF
:10018000918688083CA6AAAA2ABE000000803F00EB
:100190004E414E494E495459494E46CDCCCC3D0A6C
:1001A000D7233C17B7D13877CC2B329595E6241F4F
:1001B000B14F0A000020410000C84200401C462008
:1001C000BCBE4CCA1B0E5AAEC59D74257325730068
:1001D0002573002569206D696E2C202569207365C3
:1001E0006300205425693A20205820256620205994
:1001F0002025660A00204C002046002043002044B1
:100200000020490020500020204D3330312045008F
:10021000205A00205900205800486F6D65206F66F5
:100220006673657420286D6D293A00204500205AB8
:100230000020580020420020540020204D3230354C
:10024000205300416476616E636564207661726953
:1002500061626C65733A20533D4D696E2066656539
:10026000647261746520286D6D2F73292C20543DB4
:100270004D696E2074726176656C20666565647286
:1002800061746520286D6D2F73292C20423D6D69A6
:100290006E696D756D207365676D656E7420746928
:1002A0006D6520286D73292C20583D6D6178696D2E
:1002B000756D205859206A65726B20286D6D2F73FB
:1002C000292C20205A3D6D6178696D756D205A206A
:1002D0006A65726B20286D6D2F73292C2020453D97
:1002E0006D6178696D756D2045206A65726B202897
:1002F0006D6D2F73290020540020204D32303420A2
:100300005300416363656C65726174696F6E3A2076
:10031000533D616363656C65726174696F6E2C2017
:10032000543D7265747261637420616363656C65CA
:10033000726174696F6E00205A3A0020593A004386
:100340006F756E7420583A0020453A00205A3A00E2
:1003500020593A00583A004649524D574152455F9C
:100360004E414D453A204D61726C696E484F4820B0
:1003700056302E362D484F482028686F65686E65C8
:100380006D616E6E2E6E65742920534F5552434534
:100390005F434F44455F55524C3A68747470733AEA
:1003A0002F2F6464642E4B383430302E686F6568AC
:1003B0006E656D616E6E2E6E65742050524F544F97
:1003C000434F4C5F56455253494F4E3A312E3020E1
:1003D0004D414348494E455F545950453A4B383496
:1003E0003030202045585452554445525F434F55B4
:1003F0004E543A3220555549443A6365646532613A
:1004000032662D343161322D343734382D39623132
:10041000322D6335356336326633363766660A0009
:100420004D33323A202573202569004D3332206345
:10043000616C6C3A2025732F6E004572726F723AB0
:10044000000A004572726F723A006563686F3A0085
:100450006563686F3A000A006563686F3A00204B75
:10046000703A2025660A204B693A2025660A204BFF
:10047000643A2025660A0020436C61737369632027
:10048000504944200A004B753A20256620205475B7
:100490003A2025660A00204B703A2025660A204B38
:1004A000693A2025660A204B643A2025660A002016
:1004B000436C617373696320504944200A004B7593
:1004C0003A202566202054753A2025660A00626984
:1004D00061733A20256920643A202569206D696E90
:1004E0003A20252E3166206D61783A20252E31661E
:1004F0000A005049442072656C61792074756E69F8
:100500006E670A00204B703A2025660A204B693A34
:100510002025660A204B643A2025660A0020436C99
:10052000617373696320504944200A00536C6F70F3
:10053000653A202566202044656C61793A2025665D
:100540000A004B66203D2025660A002066283130CF
:10055000302525293A202566200A00206865617427
:100560003A2025690A0020662837352525293A20B2
:100570002566200A0020686561743A2025690A0012
:100580004B66203D2025660A002066282569252522
:10059000293A202566200A0020686561743A2025E2
:1005A000690A0020662835302525293A202566204D
:1005B0000A0020686561743A2025690A0072656640
:1005C00020686561743A2025690A0044656320311A
:1005D0003520323031370028486F6C67657220480B
:1005E0006F65686E656D616E6E29004465632031CC
:1005F0003520323031372032313A34373A32330015
:1006000056657273696F6E20312E302E300A00737A
:10061000746172740A00256920686F7572732025F1
:1006200069206D696E75746573004D31313000203D
:100630005A200A002059200A002058200A004D3272
:1006400039005A004578747275646572004572729B
:100650006F723A00256900203FECED3F5C7C3F2241
:1006600063617F3F3F52B0DF3F323327E4F1A52C77
:1006700031DF7E3F3F3F3F3F3F3F3FE13F3F3F3F17
:100680003F3F3F3F3F3F3F3F3F3F3F3F3FEF783F91
:100690003F3F3FF53F3FE23F3F3F3FE13F3F3F3F6F
:1006A0003F3F3F3F3F3F3F3FEE3F3F3F3FEFFD3F3D
:1006B0003F3F3FF53F3F3F00002100240027002A35
:1006C000002D003000330001010000040107010A81
:1006D0000100002200250028002B002E00310034EC
:1006E0000002010000050108010B010000200023A9
:1006F00000260029002C002F00320000010000031A
:100700000106010901050505050705080808080295
:100710000202020A0A08080404040401010101019A
:100720000101010303030303030303040707070C89
:100730000C0C0C0C0C0C0C0202020206060606063F
:100740000606060B0B0B0B0B0B0B0B0102102020EC
:100750000808102040102040800201020108040215
:10076000010102040810204080804020100804028B
:1007700001800402018040201008040201080402E4
:1007800001010204081020408001020408102040EA
:100790008000000A0B02090C0D0E0807030401007B
:1007A0000000000000000000000000000000000049
:1007B0000000000000000000000000000012111006
:1007C0000000000000000000000000000000000029
:1007D0000000000000000024F4D43050C38E20C27A
:1007E000A24017828B7011127A910D816CD90AA8E0
:1007F00061E108C7586607615143061E4B5D05C19C
:1008000045A7041A411104093D9803713931034089
:1008100036DB0265339102D4305402802E1D026310
:100820002CEE01752AC501B028A001102781018F87
:100830002564012B244B01E0223401AC211F018DE2
:10084000200D01801FFC00841EED00971DDF00B805
:100850001CD200E61BC600201BBC00641AB200B20A
:1008600019A8000A19A0006A189900D11791004030
:10087000178B00B516840031167E00B31579003A47
:10088000157300C7146F0058146A00EE13660088D1
:1008900013630025135E00C7125B006C125700152E
:1008A000125400C111510070114F0021114B00D69C
:1008B0001049008D1047004610440002104200C04D
:1008C0000F4000800F3E00420F3C00060F3B00CB64
:1008D0000E3800930E37005C0E3500270E3400F3FF
:1008E0000D3200C10D3100900D3000600D2E003230
:1008F0000D2D00050D2C00D90C2B00AE0C29008508
:100900000C29005C0C2700350C27000E0C2600E893
:100910000B2400C40B2400A00B23007D0B23005AE2
:100920000B2100390B2100180B2000F80A1F00D9F9
:100930000A1E00BB0A1E009D0A1D00800A1D0063DE
:100940000A1C00470A1B002C0A1B00110A1A00F798
:10095000091A00DD091900C4091900AB0919009230
:100960000917007B091800630917004C09160036A7
:10097000091600200916000A091500F5081500E0FF
:10098000081400CC081400B8081400A4081400903F
:100990000813007D0812006B081300580812004667
:1009A0000812003408110023081100120811000178
:1009B000081100F0071000E0071000D0071000C079
:1009C000071000B0070F00A107100091070E008369
:1009D000070F0074070F0065070E0057070E004948
:1009E000070E003B070D002E070E0020070D001319
:1009F000070D0006070D00F9060C00ED060D00E0DE
:100A0000060C00D4060C00C8060C00BC060C00B096
:100A1000060C00A4060B0099060C008D060B008244
:100A2000060B0077060B006C060B0061060A0057E8
:100A3000060B004C060A0042060A0038060A002E81
:100A4000060A0024060A001A060A00100609000712
:100A5000060A00FD050900F4050900EB050900E29E
:100A6000050900D9050900D0050900C7050900BE20
:100A7000050900B5050800AD050800A50509009C9D
:100A8000050800940508008C050800840508007C12
:100A9000050800740508006C050700650508005D81
:100AA000050700560508004E0507004705070040EA
:100AB00005080038050700310507002A050700234F
:100AC0000507001C050600160507000F05070008AE
:100AD00005060002050700FB040600F5040700EE0A
:100AE000040600E8040600E2040700DB040600D563
:100AF000040600CF040600C9040600C3040600BDB6
:100B0000040600B7040600B1040500AC040600A604
:100B1000040600A00405009B04060095040500904F
:100B20000406008A04050085040500800406007A96
:100B300004050075040500700405006B04050066DB
:100B4000040500610405005C04050057040500521B
:100B50000405004D04050048040500430405003E5B
:100B60000404003A04050035040500300404002C98
:100B700004050027040400230405001E0404001AD1
:100B800004040016040500110404000D0404000907
:100B90000405000404040000040400FC030400F83D
:100BA000030400F4030400F0030400EC030400E871
:100BB000030400E4030400E0030400DC030400D8A1
:100BC000030400D4030400D0030400CC030400C8D1
:100BD000030300C503030024F404D9201BC40C5CE8
:100BE0000E9804C4095F0265077101F405F900FB62
:100BF00004B30048048700C103690058035500038B
:100C0000034500BE023A008402310053022A002943
:100C100002250004022000E4011C00C8011900AFF5
:100C20000117009801140084011300710110006184
:100C300001100051010E0043010D0036010B002B85
:100C4000010B0020010B00150109000C0109000334
:100C5000010800FB000800F3000800EB000700E4B7
:100C6000000600DE000600D8000600D2000600CC18
:100C7000000500C7000500C2000500BD000400B962
:100C8000000400B5000400B1000400AD000400A998
:100C9000000400A5000300A20003009F0004009BC5
:100CA00000030098000300950002009300030090E9
:100CB0000003008D0002008B000300880002008604
:100CC00000020084000300810002007F0002007D1A
:100CD0000002007B0002007900020077000100762C
:100CE0000002007400020072000100710002006F37
:100CF0000002006D0001006C0002006A0001006942
:100D00000002006700010066000100650001006448
:100D10000002006200010061000100600001005F4C
:100D20000002005D0001005C0001005B0001005A50
:100D30000001005900010058000100570001005651
:100D40000001005500010054000100530000005351
:100D50000001005200010051000100500001004F4D
:100D60000001004E0000004E0001004D0001004C4B
:100D70000001004B0000004B0001004A0001004947
:100D80000001004800000048000100470001004643
:100D9000000000460001004500000045000100443D
:100DA0000001004300000043000100420000004237
:100DB0000001004100000041000100400001003F2F
:100DC0000000003F0001003E0000003E0001003D29
:100DD0000000003D0001003C0000003C0000003C21
:100DE0000001003B0000003B0001003A0000003A17
:100DF000000100390000003900010038000000380F
:100E00000000003800010037000000370001003604
:100E100000000036000000360001003500000035FB
:100E200000000035000100340000003400000034F0
:100E300000010033000000330000003300010032E5
:100E400000000032000000320001003100000031DB
:100E500000000031000100300000003000000030D0
:100E60000001002F0000002F0000002F0000002FC5
:100E70000001002E0000002E0000002E0001002DB9
:100E80000000002D0000002D0000002D0001002CAE
:100E90000000002C0000002C0000002C0001002BA2
:100EA0000000002B0000002B0000002B0001002A96
:100EB0000000002A0000002A0000002A000100298A
:100EC000000000290000002900000029000000297E
:100ED0000001002800000028000000280000002871
:100EE0000000002800010027000000270000002764
:100EF0000000002700000027000100260000002657
:100F00000000002600000026000000260001002549
:100F1000000000250000002500000025000000253D
:100F2000000000250001002400000024000000242F
:100F30000000002400000024000100230000002322
:100F40000000002300000023000000230000002315
:100F50000000002300010022000000220000002207
:100F600000000022000000220000002200010021F9
:100F700000000021000000210000002100000021ED
:100F800000000021000000210001002000000020DE
:100F900000000020000000200000002000000020D1
:100FA00000000020000000200001001F0000001FC2
:100FB0000000001F0000001F0000001F0000001FB5
:100FC0000000001F0001001E0000001E0000001EA7
:100FD0000000001E000000436172642073697A659E
:100FE0003A2025694D420A00556E6B6E6F776E0A86
:100FF00000534458430A00534448430A20005344D2
:10100000320A005344310A004361726420747970DB
:10101000653A20005350492073746F707065643ACC
:10102000206572726F720053504920647269766550
:10103000722073657474696E67732075706461746F
:101040006564005350492073746F707065640020AC
:1010500053442045726B656E6E756E6720616267E2
:10106000657363686C6F7373656E0020534420482A
:10107000432065726B616E6E740020636865636BFC
:1010800020736468630020696E697469616C697AB1
:1010900065205344002053442030322065726B6138
:1010A0006E6E7400636865636B20534420766572CE
:1010B00073696F6E00535049207374617274656474
:1010C0000020686F65686E656D616E6E2E6E65746A
:1010D000002020206464642E6B383430302E0020D1
:1010E0002056302E362D484F482048454144533A2B
:1010F0003200564552544558203344205052494EF0
:1011000054455200256900253369002532690025C0
:10111000316900062533692525202053442D2D2DC6
:10112000252520072D2D3A2D2D000625336925254F
:1011300020205344253369252520072532693A2587
:101140003269005820253369205920253369205AF7
:101150002025332E326600202025336920202025CB
:10116000336920202025332E3266202020000225DE
:10117000332E30662F25332E306601200225332E84
:1011800030662F25332E306601004D3630300A1A76
:101190000054310A1A0054300A1A004D38330A47F5
:1011A000312045352046323030300A1A004D38346F
:1011B00020582059205A20450A1A004D32340A1A64
:1011C000004D32310A1A004D3131372050726570AE
:1011D0006172696E672E2E2E0A4732380A473930FF
:1011E0000A4D38320A4730204631323030302058EC
:1011F0003130302059313030205A3130300A5431BA
:101200000A54300A54310A4D3130392054310A47DA
:1012100039322045300A4D38330A473120453135BF
:10122000204635300A4D31313720556E6C6F616480
:10123000696E672066696C616D656E740A4731205E
:10124000452D3337302046323030300A4731204583
:101250002D3337302046323030300A47323820586C
:1012600020590A4739300A4D38320A4D313034207E
:1012700054312053300A54300A4D38340A4D31313C
:1012800037205665727465782069732072656164D1
:101290007920202020200A1A004D31313720507249
:1012A00065706172696E672E2E2E0A4732380A47C2
:1012B00039300A4D38320A4730204631323030302A
:1012C00020583130302059313030205A3130300AF6
:1012D00054300A54310A54300A4D313039205430D8
:1012E0000A4739322045300A4D38330A4731204504
:1012F0003135204635300A4D31313720556E6C6F0F
:101300006164696E672066696C616D656E740A4719
:101310003120452D3337302046323030300A4731C6
:1013200020452D3337302046323030300A473238AE
:10133000205820590A4739300A4D38320A4D313089
:10134000342054302053300A54300A4D38340A4D7A
:101350003131372056657274657820697320726563
:1013600061647920202020200A1A004D3131372075
:10137000507265706172696E672E2E2E0A47323880
:101380000A4739300A4D38320A4730204631323068
:10139000303020583130302059313030205A3130FF
:1013A000300A54310A54300A54310A4D3130392050
:1013B00054310A4739322045300A4D38330A473113
:1013C00020453135204635300A4D31313720556EB4
:1013D0006C6F6164696E672066696C616D656E74BF
:1013E0000A473120452D3337302046323030300A1D
:1013F000473120452D3337302046323030300A47D0
:101400003238205820590A4739300A4D38320A4DAF
:101410003130342054312053300A54300A4D38349E
:101420000A4D313137205665727465782069732012
:10143000726561647920202020200A1A004D313124
:101440003720507265706172696E672E2E2E0A47C2
:1014500032380A4739300A4D38320A47302046318F
:101460003230303020583130302059313030205A2D
:101470003130300A54300A54310A54300A4D313078
:10148000392054300A4739322045300A4D38330A62
:10149000473120453135204635300A4D313137202E
:1014A000556E6C6F6164696E672066696C616D650D
:1014B0006E740A473120452D3337302046323030A4
:1014C000300A473120452D33373020463230303016
:1014D0000A473238205820590A4739300A4D3832E5
:1014E0000A4D3130342054302053300A54300A4DE4
:1014F00038340A4D31313720566572746578206969
:101500007320726561647920202020200A1A004D22
:1015100031313720507265706172696E672E2E2EE0
:101520000A4732380A4739300A4D38320A473020E4
:10153000463132303030205831303020593130305F
:10154000205A3130300A54310A54300A54310A4D8D
:101550003130392054310A4739322045300A4D386C
:10156000330A473120453337302046323030300A95
:10157000473120453239302046313030300A4D3144
:1015800031372046656564696E672066696C616DF8
:10159000656E740A473120453930204635300A4798
:1015A0003238205820590A4739300A4D38320A4D0E
:1015B0003130342054312053300A54300A4D3834FD
:1015C0000A4D3231342054310A4D313137205665BD
:1015D00072746578206973207265616479202020B7
:1015E00020200A1A004D3131372050726570617227
:1015F000696E672E2E2E0A4732380A4739300A4D57
:1016000038320A47302046313230303020583130BD
:10161000302059313030205A3130300A54300A5499
:10162000310A54300A4D3130392054300A473932AA
:101630002045300A4D38330A4731204533373020B2
:1016400046323030300A4731204532393020463179
:101650003030300A4D3131372046656564696E6738
:101660002066696C616D656E740A473120453930BA
:10167000204635300A473238205820590A47393039
:101680000A4D38320A4D3130342054302053300A5C
:1016900054300A4D38340A4D3231342054300A4D1A
:1016A0003131372056657274657820697320726510
:1016B00061647920202020200A1A004D3131372022
:1016C000507265706172696E672E2E2E0A4732382D
:1016D0000A4739300A4D38320A4730204631323015
:1016E000303020583130302059313030205A3130AC
:1016F000300A54310A54300A54310A4D31303920FD
:1017000054310A4739322045300A4D38330A4731BF
:1017100020453337302046323030300A47312045BB
:101720003239302046313030300A4D3131372046A1
:10173000656564696E672066696C616D656E740AC3
:10174000473120453930204635300A473238205855
:1017500020590A4739300A4D38320A4D3130342089
:1017600054312053300A54300A4D38340A4D323146
:10177000342054310A4D3131372056657274657802
:1017800020697320726561647920202020200A1A64
:10179000004D31313720507265706172696E672E6D
:1017A0002E2E0A4732380A4739300A4D38320A4756
:1017B00030204631323030302058313030205931ED
:1017C0003030205A3130300A54300A54310A543003
:1017D0000A4D3130392054300A4739322045300A19
:1017E0004D38330A473120453337302046323030C8
:1017F000300A473120453239302046313030300A06
:101800004D3131372046656564696E672066696CC5
:10181000616D656E740A4731204539302046353098
:101820000A473238205820590A4739300A4D383291
:101830000A4D3130342054302053300A54300A4D90
:1018400038340A4D3231342054300A4D313137208A
:1018500056657274657820697320726561647920B9
:10186000202020200A1A004D38340A1A0047323846
:101870000A1A00454F465F434841521A000D0A00BC
:101880002F2000200073657276696365206E7220D8
:1018900025690A000000204100002041000040406E
:1018A0000101FF00003E430000344300003E4300BE
:1018B0000048430000484300003E43000020410030
:1018C00000A0410000000000004843000048430021
:1018D00000000058005900756E646566696E6564A5
:1018E000206572726F7220636F6465000A00204089
:1018F00025693A2569002042403A256920403A2569
:101900006900205425693A252E3166202F252E3076
:10191000660020423A252E3166202F252E316600A2
:10192000543A252E3166202F252E30660020204384
:101930003A20256620463A2025660A0A00202050D3
:101940003A20256620493A20256620443A2025661B
:101950000A0020486561746572202025693A0A00F2
:101960004368616E67652066696C616D656E740AB7
:1019700000756E6B6E6F776E20636F6D6D616E6458
:101980003A205C25735C200A0020204D3230312043
:101990005820256C2C205920256C2C205A20256C91
:1019A0002C204520256C0A0A004D6178696D756D03
:1019B00020416363656C65726174696F6E20286D88
:1019C0006D2F73322920284D323031293A0A0020F8
:1019D000204D32303320582025662C205920256692
:1019E0002C205A2025662C20452025660A0A004D09
:1019F0006178696D756D2066656564726174657383
:101A000020286D6D2F732920284D323033290A3A52
:101A10000020582025312E32662C20592025312EC9
:101A200032662C205A2025312E32662C2045202566
:101A3000312E32660A0A0053746570732070657225
:101A400020756E697420284D3932293A0A002065C4
:101A50006570726F6D206279746573206C6F61645C
:101A600065643A2025690A0048617264636F6465A1
:101A7000642044656661756C7420506172616D65A7
:101A8000746572204C6F616465640020746F6F2010
:101A90006C6F6E6720657874727573696F6E2070F5
:101AA000726576656E7465640A0020636F6C6420ED
:101AB000657874727573696F6E2070726576656E85
:101AC0007465640A002054656D7065726174757286
:101AD00065206E6F7420726561636865642C206197
:101AE000626F727420617420252E31660A002052C4
:101AF00065647563696D672066616E2073706565E6
:101B000064210A00205265706561742054656D700F
:101B1000657261747572652073746162696C697352
:101B20006174696F6E200A0046616E204175746FA2
:101B300074756E65207374617274696E670A002033
:101B400048656174657220737769746368656420A1
:101B50006F66662E204D494E54454D502074726973
:101B6000676765726564206F6E204578747275646E
:101B70006572202569210A0020486561746572201C
:101B80007377697463686564206F66662E204D41C3
:101B90005854454D502074726967676572656420BA
:101BA0006F6E204578747275646572202569210A0C
:101BB0000020457874727573696F6E20636F656677
:101BC00066696369656E74204B632025690A00208D
:101BD0004865617420402025696D6D203A20256993
:101BE0000A005374657020323A2074756E65206562
:101BF0007874727573696F6E20706172616D65744F
:101C00006572005374657020313A2074756E6520DA
:101C100066616E20706172616D657465720A005351
:101C2000746172742074756E696E67202D202D208A
:101C30002D0A0041626F72742074756E696E672C94
:101C4000206E6F7420617420686F6D6520706F73F3
:101C50006974696F6E0A00504944204175746F744D
:101C6000756E652066696E697368656421205049E8
:101C70004420706172616D65746572732075706463
:101C8000617465640A00504944204175746F74752D
:101C90006E652066696E697368656421205075748D
:101CA00020746865206C617374204B702C204B6924
:101CB00020616E64204B6420636F6E7374616E7478
:101CC000732066726F6D2061626F766520696E7435
:101CD0006F20436F6E66696775726174696F6E2EEF
:101CE000680A00504944204175746F74756E652010
:101CF0006661696C6564212074696D656F75740A2D
:101D000000504944204175746F74756E652066619A
:101D1000696C6564212054656D70657261747572BB
:101D20006520746F6F20686967680054656D706521
:101D30007261747572652073746162696C69736530
:101D4000642061742025660A0053746162696C69BD
:101D5000736520686F74656E640A005049442041C1
:101D600075746F74756E6520737461727400504978
:101D700044204175746F74756E65206661696C6589
:101D8000642E2042616420657874727564657220E7
:101D90006E756D6265722E005049442072657365E0
:101DA0007400416374697665204578747275646562
:101DB000723A204525690A006572726F723A2054A2
:101DC000256920496E76616C696420657874727546
:101DD000646572206E756D6265720A006563686F76
:101DE0003A204D256920496E76616C6964206578DA
:101DF000747275646572205425690A0043686563CE
:101E00006B73756D203A202025690A00436865636D
:101E10006B73756D206572726F72206F6E207072B9
:101E2000696E74657220706172616D65746572733C
:101E30002E204661696C736176652076616C7565EC
:101E400073206C6F616465640A005072696E74651A
:101E5000722068616C7465642E206B696C6C282933
:101E60002063616C6C6564210A005072696E746550
:101E7000722073746F707065642064756520746F70
:101E8000206572726F72732E2046697820746865BF
:101E9000206572726F7220616E6420757365204DCB
:101EA00039393920746F20726573746172742E2011
:101EB0002854656D70657261747572652069732050
:101EC00072657365742E2053657420697420616691
:101ED0007465722072657374617274696E67290A21
:101EE0002000486F74656E64206F66667365747356
:101EF0003A00537465707261746520746F6F206866
:101F00006967683A202569200A00656E6473746FFA
:101F10007073206869743A20006F70656E0A00540F
:101F200052494747455245440A20007A5F6D61781F
:101F30003A2000795F6D61783A2000785F6D6178B2
:101F40003A20005265706F7274696E6720656E6426
:101F500073746F70207374617475730A0053554203
:101F6000524F5554494E452043414C4C20746172A8
:101F70006765743A2225732220706172656E743A27
:101F80002225732220706F732025690A00747279EC
:101F9000696E6720746F2063616C6C207375622DAD
:101FA00067636F64652066696C6573207769746820
:101FB00020746F6F206D616E79206C6576656C732F
:101FC0002E204D4158206C6576656C2069733A204F
:101FD00025690A0057726974696E6720746F2066FC
:101FE000696C653A2025730A004E6F7720646F692B
:101FF0006E672066696C653A2025730A004E6F771C
:102000002066726573682066696C653A2025730ADC
:102010000044656C6574696F6E206661696C656407
:102020002C2046696C653A2025730A0046696C6568
:102030002064656C657465643A2025730A004E6FF0
:1020400074205344207072696E74696E670A00537D
:1020500044207072696E74696E67206279746520BD
:102060002569202F2025690A006F70656E20666142
:10207000696C65642C2046696C653A2025730A00FA
:1020800046696C65206F70656E65643A2025732023
:1020900053697A653A2025690A00456E64206669AD
:1020A0006C65206C6973740A00426567696E20660E
:1020B000696C65206C6973740A00446F6E652070EA
:1020C00072696E74696E672066696C650A0046699C
:1020D0006C652073656C65637465640A0053442005
:1020E00063617264206F6B0A00566F6C756D6520BA
:1020F0006973204641542569200A0043616E2774A4
:102100002066696E6420612076616C6964204641B6
:102110005431362F464154333220706172746974E1
:10212000696F6E2E0A00534420696E6974206661DF
:10213000696C006F6B0A00526573656E643A202506
:102140006C0A004E6F204C696E65204E756D62659D
:1021500072207769746820636865636B73756D2C92
:10216000204C617374204C696E653A2025690A0021
:102170004E6F20436865636B73756D207769746873
:10218000206C696E65206E756D6265722C204C61E5
:102190007374204C696E653A2025690A006368658E
:1021A000636B73756D206D69736D617463682C204A
:1021B0004C617374204C696E653A2025690A004CA5
:1021C000696E65204E756D626572206973206E6F51
:1021D00074204C617374204C696E65204E756D627D
:1021E00065722B312C204C617374204C696E653AFA
:1021F0002025690A00446F6E6520736176696E67F9
:102200002066696C652E0A0020436F6D70696C65ED
:10221000643A20002020506C616E6E6572427566D3
:1022200066657242797465733A2025690A00204612
:10223000726565204D656D6F72793A2025690020C1
:102240004C61737420557064617465643A20002099
:102250007C20417574686F723A20004F6666736522
:102260007420592020202025312E3266004F6666CA
:1022700073657420582020202025312E32660041BD
:102280006D617820452020202025356C00416D614E
:1022900078205A2020202025356C00416D6178205F
:1022A000592020202025356C00416D617820582070
:1022B00020202025356C00466C6F772074696D6591
:1022C0002020202020202533690045737465707319
:1022D0002F6D6D2020202025352E3166005A737415
:1022E0006570732F6D6D20202025352E31660059C5
:1022F00073746570732F6D6D20202025352E326626
:10230000005873746570732F6D6D20202025352E55
:10231000326600412D74726176656C00412D7265E4
:102320007472616374202020202025352E306600D1
:102330005654726176206D696E2020202020202561
:10234000332E306600566D696E202020202020201C
:102350002020202025332E306600566D61782045E0
:10236000202020202020202025342E306600566D8D
:102370006178205A20202020202020202025332E64
:10238000306600566D6178205920202020202020C2
:10239000202025332E306600566D6178205820208D
:1023A0002020202020202025332E30660056652D49
:1023B0006A65726B202020202020202025332E30BB
:1023C0006600567A2D6A65726B202020202020201E
:1023D00025352E3266005678792D6A65726B20207D
:1023E000202020202025332E306600416363656C59
:1023F00020202020202020202025352E306600504F
:1024000049442D4620426564202020202020253389
:102410002E3066005049442D432042656420202020
:102420002025352E3266005049442D4420426564F3
:102430002020202025352E3266005049442D492089
:102440004265642020202025352E32660050494404
:102450002D50204265642020202025352E32660034
:102460005049442D46203220202020202025342E83
:102470003266005049442D43203220202020202065
:1024800025352E3266005049442D4420322020202C
:1024900020202025352E3266005049442D49203217
:1024A00020202020202025352E3266005049442D42
:1024B00050203220202020202025352E326600504A
:1024C00049442D46203120202020202025342E3242
:1024D00066005049442D4320312020202020202513
:1024E000352E3266005049442D44203120202020D2
:1024F000202025352E3266005049442D49203120B8
:10250000202020202025352E3266005049442D50B1
:10251000203120202020202025352E326600466CD8
:102520006F77203220202020202020202025336992
:1025300000466C6F77203120202020202020202092
:1025400025336900466C6F77202020202020202032
:102550002020202533690064656C617920322020B9
:102560002020202020202533690064656C617920BB
:102570003120202020202020202533690070726522
:1025800073735F6164765F322020202025332E3004
:10259000660070726573735F6164765F312020201E
:1025A0002025332E30660046616E207370656564A9
:1025B000202020202020253369004265642020202F
:1025C000202020202020202020253369004E6F7AF3
:1025D0007A6C6520322020202020202025336900BD
:1025E0004E6F7A7A6C652031202020202020202513
:1025F0003369004E6F7A7A6C6520202020202020DD
:102600002020253369004572723A204D494E5445C9
:102610004D50004572723A204D415854454D50007E
:1026200053544F505045440042656420646F6E65BA
:102630002E0053746F700053746172740045787487
:102640007275646572004D6F7665205A004D6F7625
:10265000652059004D6F76652058004D6F766520D6
:1026600031306D6D004D6F766520316D6D004D6FB1
:10267000766520302E316D6D0053706565642020C5
:10268000202020202020202025336900052E2E0028
:102690000552656672657368004368616E67652000
:1026A0005344206361726400496E69742E20534460
:1026B0002063617264005072696E742066726F6D7F
:1026C0002053440053746F70207072696E7400520E
:1026D0006573756D65207072696E740050617573F5
:1026E00065207072696E74004E6F205344206361E0
:1026F0007264005468656E20707265737320627531
:1027000074746F6E002076697369626C6520696EFF
:1027100020747562650020756E74696C20312E35E9
:10272000636D20697300496E736572742066696C0D
:10273000616D656E74005072656865617420414218
:102740005320416C6C005072656865617420414291
:1027500053203200507265686561742041425320F5
:1027600031005072656865617420504C4120416CA5
:102770006C005072656865617420504C41203200D5
:102780005072656865617420504C41203100556E6F
:102790006C6F616420504C41206C656674004C6F16
:1027A000616420504C41206C65667400556E6C6FFE
:1027B000616420504C41207269676874004C6F61FD
:1027C0006420504C4120726967687400556E6C6FCC
:1027D000616420414253206C656674004C6F6164F3
:1027E00020414253206C65667400556E6C6F6164C5
:1027F00020414253207269676874004C6F61642005
:1028000041425320726967687400526573746F7235
:1028100065206661696C73616665004C6F61642058
:102820006D656D6F72790053746F7265206D656DA3
:102830006F72790053746F707761746368004164DC
:1028400076616E636564004D6F74696F6E005465E8
:102850006D70657261747572650045787472756427
:102860006572206F66667365747300436F6F6C6486
:102870006F776E0044697361626C65207374657074
:1028800070657273004D6F766520617869730050D2
:1028900072656865617420414253005072656865D5
:1028A000617420504C4100556E6C6F616420666904
:1028B0006C616D656E74004C6F61642066696C615B
:1028C0006D656E74004175746F20686F6D650046AC
:1028D00069726D776172652076657273696F6E00DB
:1028E000436F6E74726F6C00507265706172650038
:1028F00054756E6500496E666F2053637265656E30
:10290000004D61696E005072696E74696E67206473
:102910006F6E652E005072696E74696E672E2E2E72
:102920000048656174696E6720646F6E652E0048AB
:10293000656174696E672E2E2E004B38343030205E
:1029400072656164792E0077616974004D61726C03
:10295000696E5F484F48200070012C0190012701EB
:10296000B0012201C0011D01F00118011002130184
:1029700030020E016002090190020401C002FF0052
:102980000003FA004003F5008003F000D003EB00E1
:102990002004E6007004E100E004DC004005D700FC
:1029A000C005D2004006CD00D006C8008007C30095
:1029B0003008BE00F008B900C009B400B00AAF008A
:1029C000B00BAA00D00CA500000EA000500F9B0079
:1029D000C01096005012910000148C00C0158700A2
:1029E000B0178200B0197D00D01B7800001E730064
:1029F00040206E0090226900F024640040275F00B0
:102A000090295A00E02B5500102E500020304B002A
:102A100010324600E033410090353C00103737005B
:102A200070383200A0392D00B03A2800A03B2300B6
:102A3000603C1E00103D1900903D1400103E0F0038
:102A4000703E0A00C03E0500003F0000257325735C
:102A5000000091CC82CC11241FBECFEFD1E2DEBFAB
:102A6000CDBF00E00CBF15E0A0E0B2E0ECE4F8EB75
:102A700001E00BBF02C007900D92A03EB107D9F74D
:102A800027E1A0EEB5E001C01D92A434B207E1F742
:102A900015E1CAE2D5E100E006C021970109802FC7
:102AA000FE010E94B4DAC932D10780E00807A9F715
:102AB0000E9447C30C9415DC0C9400002F923F92A7
:102AC0004F925F926F927F928F929F92AF92BF923E
:102AD000CF92DF92EF92FF920F931F93CF93DF93EA
:102AE000CDB7DEB7C454D1090FB6F894DEBF0FBE20
:102AF000CDBF87E40E94872B882309F428C10E9458
:102B0000B72B0E9441D86430710509F44AC044F4DF
:102B10006230710589F1CCF577FF23C00C94B5289C
:102B20006A35710509F4E0C034F46C31710509F4BB
:102B3000A0C00C94B5286B35710509F4D9C06C356B
:102B4000710511F00C94B5280E94D58D16E0C12EA8
:102B500015E0D12E00E8E02E02E1F02E00E010E0BA
:102B6000E1C08091160C81110C94B5280E94D9C146
:102B70000E946B8C0C94B5288091160C81110C94DA
:102B8000B5280E943BC281E008C08091160C8111DB
:102B90000C94B5280E943BC280E00E949ABE0C941F
:102BA000432A1092E8051092E9051092EA05109266
:102BB000EB0580E50E94872B882361F00E94B72BEC
:102BC0000E9447D86093E8057093E9058093EA0571
:102BD0009093EB0583E50E94872B882391F00E9458
:102BE000B72B20E030E04AE754E40E9485CE0E94F3
:102BF00047D86093E8057093E9058093EA059093C0
:102C0000EB050E94D58D0E94E1C20091E80510916C
:102C1000E9052091EA053091EB05DC01CB01800F3D
:102C2000911FA21FB31F8093E8059093E905A0931D
:102C3000EA05B093EB050E94E1C26093DE0B70934E
:102C4000DF0B8093E00B9093E10B0E94E1C20091B7
:102C5000E8051091E9052091EA053091EB05601730
:102C600071078207930710F00C94B5280E94B3B344
:102C7000ECCF1092E7051092E6051092E50588E585
:102C80000E94872B882319F081E08093E50589E570
:102C90000E94872B882319F081E08093E6058AE55E
:102CA0000E94872B882319F081E08093E7058091AB
:102CB000E50581110FC08091E60581110BC080915F
:102CC000E705811107C081E08093E7058093E60561
:102CD0008093E5054091E7056091E6058091E50563
:102CE0000E94218F0C94B52810921F170C94B528C0
:102CF00081E080931F170C94B52803301105D1F49F
:102D00000E94B72BAB01BC0183E090E00E94A3536B
:102D1000F4E0EF0EF11C0F5F1F4F0430110511F4AA
:102D20000C94B528F60181916F010E94872B8823AE
:102D300079F3E3CF0E94B72BF701208131814281E3
:102D400053810E94E7D6AB01BC01C801DFCF8DE4FF
:102D50000E94872B882311F40C9471270E94B72BB3
:102D60000E9441D8AB01BC01CA014237510511F4A0
:102D70000C941B1F0CF0CAC04F31510509F4C2C599
:102D80000CF045C04631510509F46AC324F54131C0
:102D9000510509F423C39CF457FF02C00C944D273E
:102DA000423051050CF49AC24031510511F00C9497
:102DB0004D2782E090E00E943A910C94B52844316E
:102DC000510509F419C30CF047C34231510509F408
:102DD00043C70C944D274A31510509F4A0C33CF474
:102DE0004831510509F45FC30CF440C382C34C3130
:102DF000510509F4E3C30CF4A2C34D31510509F4A4
:102E000016C44E31510509F416C40C944D274435AF
:102E1000510509F421C77CF54C34510509F4BCC5B2
:102E200074F44A32510509F493C54B34510509F441
:102E3000ADC54032510511F00C944D27BBC441354E
:102E4000510509F4EFC64CF44D34510511F00C94C2
:102E50004D270E944EAA0C94B5284235510509F41D
:102E6000F7C64335510511F00C944D2781E080934E
:102E700023170C94B5284936510509F4CCC5B4F58F
:102E80004C35510509F433C74836510509F488C556
:102E90004535510511F00C944D2783E50E94872B91
:102EA0000E94B72B20E030E04AE754E40E9485CE30
:102EB0000E9447D86B017C016093E20B7093E30B97
:102EC0008093E40B9093E50B0E94E1C2DC01CB01FF
:102ED0008C0D9D1DAE1DBF1D8093F60B9093F70BBF
:102EE000A093F80BB093F90B0C94B5284B36510511
:102EF00009F492C60CF47CC64D36510509F496C50A
:102F00004E36510509F4A8C50C944D274D3D510589
:102F100011F40C9461230CF06EC0483C510511F47F
:102F20000C947E2074F54837510511F40C94F51F6C
:102F3000B4F44537510509F450C74737510511F42A
:102F40000C94F91F4337510511F00C944D2767E598
:102F500073E08AED9BE00E9461460C94B5284C38E2
:102F6000510509F441C54E3B510509F488C549375F
:102F7000510511F00C944D2781E08093700C0C9456
:102F8000B5284D3C510511F40C948D21ACF44B3C0B
:102F9000510511F40C94412114F00C945E21493C2C
:102FA000510511F00C944D2796E0E92E95E0F92E8D
:102FB00000E010E00C942521463D510511F40C94DD
:102FC0000A226CF44E3C510511F00C944D27B6E0EA
:102FD000EB2EB5E0FB2E00E010E00C94F9214A3D09
:102FE000510511F40C94D2224C3D510511F40C946E
:102FF00052230C944D27443F21E0520711F40C94C6
:103000008925ACF58E3241E0940711F40C947925B2
:1030100094F4803F910511F40C94B5288D32E1E0D1
:103020009E0711F40C949623823E910511F00C94A6
:103030004D270C9487238036F1E09F077CF48E3572
:1030400021E0920714F00C94B5288F32914011F0D2
:103050000C944D270E94C02B0C94B52880399140C8
:1030600011F00C944D270E94D58D0C94B52848354D
:10307000E2E05E0711F40C9421270CF005C1463FF5
:1030800021E0520711F40C948F2514F40C948C2534
:10309000873F914011F00C944D270AED1BE0E09121
:1030A000DC0BF091DD0BE058FE4F60817181C801AF
:1030B0000E94614680914B128F9380914A128F93A8
:1030C000809149128F93809148128F93809147127B
:1030D0008F93809146128F93809145128F938091A8
:1030E00044128F93809143128F93809142128F9359
:1030F000809141128F93809140128F9380913F1263
:103100008F9380913E128F9380913D128F93809187
:103110003C128F93E091DC0BF091DD0BEE57FE4FEC
:1031200081818F9380818F931F930F930E949E467E
:10313000C8010E94EB2AE091DC0BF091DD0BEC570B
:10314000FE4F60817181C8010E94614680915B12CF
:103150008F9380915A128F93809159128F938091FF
:1031600058128F93809157128F93809156128F939C
:10317000809155128F93809154128F9380915312A6
:103180008F93809152128F93809151128F938091DF
:1031900050128F9380914F128F9380914E128F9384
:1031A00080914D128F9380914C128F93E091DC0BA4
:1031B000F091DD0BEA57FE4F81818F9380818F93D1
:1031C0001F930F930E949E460FB6F894DEBF0FBE6A
:1031D000CDBFC8010E94EB2AE091DC0BF091DD0B22
:1031E000E857FE4F60817181C8010E94614680915D
:1031F000F7128F938091F6128F938091F5128F932F
:103200008091F4128F938091F3128F938091F21238
:103210008F938091F1128F938091F0128F93809110
:10322000EF128F938091EE128F938091ED128F9316
:103230008091EC128F938091EB128F938091EA1220
:103240008F938091E9128F938091E8128F93E09190
:10325000DC0BF091DD0BE657FE4F81818F9380816F
:103260008F931F930F930E949E46C8010E94EB2AE2
:10327000E2E0F3E084910FB6F894DEBF0FBECDBF5D
:1032800002E013E00C949225403AE3E05E0709F473
:10329000FDC24CF44B5853404230510510F40C948D
:1032A000B5280C944D27473E534011F00C944D2700
:1032B0001092160C8091241790912517A091261733
:1032C000B09127178093F6059093F705A093F80522
:1032D000B093F9050E948CC20C94B52884E090E06C
:1032E0009093190C8093180C1092E8051092E90540
:1032F0001092EA051092EB0580E50E94872B882347
:1033000061F00E94B72B0E9447D86093E805709344
:10331000E9058093EA059093EB0583E50E94872BEE
:10332000882391F00E94B72B20E030E04AE754E474
:103330000E9485CE0E9447D86093E8057093E90506
:103340008093EA059093EB050E94D58D0E94E1C21F
:103350006093DE0B7093DF0B8093E00B9093E10B97
:10336000C090E805D090E905E090EA05F090EB0503
:10337000C114D104E104F10441F10E94E1C2C60E7E
:10338000D71EE81EF91EC092E805D092E905E0922A
:10339000EA05F092EB050E94E1C20091E805109168
:1033A000E9052091EA053091EB0560177107820766
:1033B000930710F00C94B52880914B0982FF02C04E
:1033C0000C94B5280E94B3B3E6CF80914B0982FFDD
:1033D00002C00C94B5280E94B3B3F7CF5F988A98C7
:1033E0009FB7F894809108018D7F809308019FBF5B
:1033F000129847980C94B528E091DC0BF091DD0B06
:10340000EC5EFE4F608171818AED9BE00E94614617
:1034100088E696E10E94959661E474E188E696E17B
:103420000E94879540E050E0BA0188E696E10E944C
:103430007A9461E088E696E10E949993E091DC0B32
:10344000F091DD0BEA5EFE4F608171818AED9BE0B9
:103450000E9461460C94B5280E9443520C94B528F2
:1034600010929613109295130C94B5280091E005D4
:103470001091E1050C5F1F4F6AE270E0C8010E94E5
:10348000C4DB009711F0FC0110828091951390919C
:103490009613892B11F40C94B52861E0C8010E94A1
:1034A000B3910C94B5280E94A19110920B0C10922C
:1034B0000A0C10920E0C10920F0C1092100C10921D
:1034C000110C1092120C1092130C1092140C1092FA
:1034D000150C10920D0C10920C0C8AE09CE00E94CE
:1034E000F74983E090E09093190C8093180C0C94AA
:1034F000B5288091951390919613029741F483E03B
:1035000090E090939613809395130E94E3B184E02A
:1035100090E09093190C8093180C0C94B52880912E
:10352000951390919613019711F00C94B52883E5AB
:103530000E94872B81110C94B8280C94B528809197
:10354000951390919613E091DC0BF091DD0B892B94
:1035500051F4E25EFE4F608171818AED9BE00E9432
:1035600061460C94B5288091D3168F938091D21622
:103570008F938091D1168F938091D0168F938091E5
:10358000DB168F938091DA168F938091D9168F93E3
:103590008091D8168F938AED9BE0E45EFE4F2181E7
:1035A0002F9320812F939F938F930E949E460FB657
:1035B000F894DEBF0FBECDBF0C94B5288091E00516
:1035C0009091E1056AE270E004960E94C4DB8C01F0
:1035D000892BD9F020910C0930910D09C901B6E071
:1035E000880F991FBA95E1F76EE470E0845F994FF8
:1035F0000E94C4DB60E270E00E94C4DB01969093FD
:10360000E1058093E005F80110828091E00590913A
:10361000E1052091951330919613232B11F40C940E
:10362000B52860E004960E94B3910C94B5281092DE
:1036300093130C94B528809195139091961301974C
:1036400011F00C94B5280E940A938091E0059091A6
:10365000E1056AE270E004960E94C4DB8C01892BCC
:10366000D9F020910C0930910D09C901A6E0880F0D
:10367000991FAA95E1F76EE470E0845F994F0E946C
:10368000C4DB60E270E00E94C4DB01969093E10528
:103690008093E005F8011082E091E005F091E105EA
:1036A0008091951390919613892B11F40C94B52861
:1036B000CF01049621E030E03093961320939513C8
:1036C00024812F3279F49F938F9380ED91E09F9323
:1036D0008F930E94115AD82EC92E0F900F900F90E1
:1036E0000F9014C09F938F938BE993E19F938F93D7
:1036F0008BEC91E09F938F930E94115AD82EC92E84
:103700000F900F900F900F900F900F9019821A82C8
:1037100021E04D2D5C2D68E676E18E010F5F1F4F95
:10372000C8010E94A396882311F40C94B52819A20D
:103730001AA222E04D2D5C2D68E676E1CE0181963D
:103740000E94A3968823E1F019821A8289A183FF3F
:1037500017C08BA181FF14C021964CAD5DAD6EAD3D
:103760007FAD2197411551056105710511F40C9448
:10377000CA288FA198A50E94AB8481110C94CA28F5
:10378000CF92DF928AED9BE0E091DC0BF091DD0BB4
:10379000EE5DFE4F21812F9320812F939F938F9376
:1037A0000E949E460F900F900F900F900F900F90D9
:1037B0000C94B5288091951390919613019711F46C
:1037C0000E94D58D8091E1058F938091E0058F93C4
:1037D0008BE294E09F938F938AED9BE09F938F936E
:1037E0000E949E460091E0051091E1050C5F1F4F7D
:1037F0006AE270E0C8010E94C4DB7C0161E270E013
:10380000C8010E94C4DB0F900F900F900F900F9093
:103810000F90009719F08C010F5F1F4FE114F10416
:1038200011F0F701108280919513909196130297F1
:1038300011F00C94B5281F921F921F930F9380E2F2
:1038400094E09F938F938AED9BE09F938F930E94C8
:103850009E460FB6F894DEBF0FBECDBF8091951384
:1038600090919613892B21F061E0C8010E94B391D9
:103870000E94A1918AE09CE00E94F74983E090E0D9
:103880009093190C8093180C0C94B5288091E00546
:103890009091E1056AE270E005960E94C4DB8C011C
:1038A000892BD9F080910C0990910D0966E0880F61
:1038B000991F6A95E1F76EE470E0845F994F0E946A
:1038C000C4DB60E270E00E94C4DB01969093E105E6
:1038D0008093E005F801319710828091E005909186
:1038E000E10521E0209394132091951330919613D4
:1038F000232B11F40C94B52860E005960E94B39137
:103900000C94B5288AE09CE00E94D049BC0180E07C
:1039100090E02CE330E040E050E00E94ABD67F9393
:103920006F933F932F9383ED91E09F938F93CE01FD
:1039300001969F938F930E943DD38AED9BE00E9456
:10394000EB2A0FB6F894DEBF0FBECDBF0C94B5289E
:1039500083E50E94872B882311F40C94B5280E94DC
:10396000B72B6B017C0180E50E94872B882311F423
:103970000C94B528C701B6010E9441D86F3F71056C
:1039800009F010F40C9478290C94B5288AE09CE096
:103990000E94F7490C94B5280E94E3B10C94B52815
:1039A00088E690E00E9477BD81110C94B52883E5EC
:1039B0000E94872B882311F40C94B5280E94B72B02
:1039C0000091281710E0000F111F0C55154F0E9491
:1039D00041D8F8017183608381E090E09093190CE5
:1039E0008093180C0C94B52883E50E94872B8823BC
:1039F00011F40C94B5280E94B72B0E9441D8709303
:103A0000AD0A6093AC0A81E090E09093190C80932A
:103A1000180C0C94B52889E690E00E9477BD8111BE
:103A20000C94B5280E947CAA0C94B5288DE690E0F1
:103A30000E9477BD81110C94B52883E50E94872BE5
:103A4000F82E81110C947A2982E50E94872B81112E
:103A50000C947A290C94F9298EE40E94872B8823F0
:103A600011F40C94B5280E94AC2B6093FA05709366
:103A7000FB058093FC059093FD050C94B52883E528
:103A80000E94872B882389F00E94B72B0E9441D87F
:103A90007093AD0A6093AC0A81E090E09093190CAA
:103AA0008093180C8093000215C082E50E94872B3A
:103AB000882381F00E94B72B0E9441D87093AD0AF1
:103AC0006093AC0A81E090E09093190C8093180CFD
:103AD000109200020E94E1C26093E8057093E9052C
:103AE0008093EA059093EB056091AC0A7091AD0A62
:103AF000072E000C880B990B0E9472D311E02091C5
:103B0000A80A3091A90A4091AA0A5091AB0A0E94D2
:103B10002DD918160CF010E01093E4058091E405FF
:103B20006091AC0A7091AD0A8823B1F1072E000CA8
:103B3000880B990B0E9472D32091A80A3091A90A90
:103B40004091AA0A5091AB0A0E942DD91816D4F5BB
:103B50000E94E1C20091E8051091E9052091EA0573
:103B60003091EB05DC01CB01801B910BA20BB30B59
:103B7000893E9340A105B10560F00E947CAA0E9495
:103B8000E1C26093E8057093E9058093EA0590939C
:103B9000EB050E94B3B3C2CF072E000C880B990B24
:103BA0000E9472D32091A80A3091A90A4091AA0AD2
:103BB0005091AB0A0E946CD387FF04C08091000231
:103BC000882331F2E091DC0BF091DD0BEC57FF4FD5
:103BD000808191810E94695C0E94E1C26093DE0B4A
:103BE0007093DF0B8093E00B9093E10B0C94B5285E
:103BF00083E50E94872B882349F00E94B72B0E94FF
:103C000041D8CB010E9411AD0C94B5288FEF90E004
:103C10000E9411AD0C94B52880E090E00E9411AD97
:103C20000C94B5280E942FB60E94D58D129A479AFF
:103C30000E94679180E090E00E9411AD68EE73E011
:103C400080E090E00E9454570E94765C0C94B52866
:103C5000109223170C94B52883E50E94872B8823A4
:103C600061F10E94B72B20E030E04AE754E40E9463
:103C700085CE0E9447D86093E60B7093E70B809344
:103C8000E80B9093E90B0E94E1C20091E60B1091C2
:103C9000E70B2091E80B3091E90BDC01CB01800FA1
:103CA000911FA21FB31F8093FA0B9093FB0BA0935D
:103CB000FC0BB093FD0B0C94B52888E50E94872B74
:103CC00081110C941A2A89E50E94872B81110C948A
:103CD0001A2A8AE50E94872B81110C941A2A85E4FE
:103CE0000E94872B81110C941A2A0C94402A26E0FA
:103CF000C22E25E0D22E08E312E1F12CF6018191CB
:103D00006F010E94872B882309F45FC0F3E0FF1244
:103D100055C00E94B72B2B013C0120E030E040EA67
:103D200051E40E946CD387FF43C0A3019201F801C4
:103D300064817581868197810E94D0D74B015C0197
:103D40009B01AC01609178127091791280917A1286
:103D500090917B120E9485CE6093781270937912B5
:103D600080937A1290937B12A5019401F8016489E3
:103D70007589868997890E9485CEF801648B758B39
:103D8000868B978B1801F4EC2F0E311CF1016081AA
:103D90007181828193810E9470D3A50194010E9458
:103DA00085CE0E9447D8F10160837183828393831B
:103DB000F801448255826682778207C00E94B72B41
:103DC000F8016483758386839783F3940C5F1F4F98
:103DD000F4E0FF1293CF0C94B5280091E005109108
:103DE000E1050B5F1F4F6AE270E0C8010E94C4DB6F
:103DF000009719F0FC01319710824CE350E0B801B4
:103E000082E29AE00E94D6DB0E948BB582E080932A
:103E10002B020E94E1C2DC01CB01805F984DAF4FC5
:103E2000BF4F8093060C9093070CA093080CB0939F
:103E3000090C0C94B528E4E5F3E084918F01882304
:103E400039F00E9470BD0F5F1F4FF8018491F7CFCA
:103E50006091610A7091620A8091630A9091640A8C
:103E600042E00E94CAA9E0E5F3E084918F01882333
:103E700039F00E9470BD0F5F1F4FF8018491F7CF9A
:103E80006091650A7091660A8091670A9091680A4C
:103E900042E00E94CAA9ECE4F3E084918F018823F8
:103EA00039F00E9470BD0F5F1F4FF8018491F7CF6A
:103EB0006091690A70916A0A80916B0A90916C0A0C
:103EC00042E00E94CAA9E8E4F3E084918F018823CC
:103ED00039F00E9470BD0F5F1F4FF8018491F7CF3A
:103EE00060916D0A70916E0A80916F0A9091700ACC
:103EF00042E00E94CAA9EFE3F3E084918F01882396
:103F000039F00E9470BD0F5F1F4FF8018491F7CF09
:103F10002FB7F8946091100A7091110A8091120ADB
:103F20009091130A2FBF0E9472D320913C123091BE
:103F30003D1240913E1250913F120E94D0D742E074
:103F40000E94CAA9EBE3F3E084918F01882339F042
:103F50000E9470BD0F5F1F4FF8018491F7CF2FB7FC
:103F6000F8946091140A7091150A8091160A909144
:103F7000170A2FBF0E9472D3209140123091411234
:103F800040914212509143120E94D0D742E00E94C9
:103F9000CAA9E7E3F3E084918F01882339F00E94F6
:103FA00070BD0F5F1F4FF8018491F7CF2FB7F894C2
:103FB0006091180A7091190A80911A0A90911B0A4F
:103FC0002FBF0E9472D3209144123091451240912C
:103FD0004612509147120E94D0D742E00E94CAA9CF
:103FE0008AE00E9470BD0C94B5281092700C0C945D
:103FF000B528E091DC0BF091DD0BE25DFE4F6081B6
:1040000071818AED9BE00E946146E091DC0BF091AA
:10401000DD0BE05DFE4F608171818AED9BE00E94C7
:104020006146E091DC0BF091DD0B659B03C088E3FA
:1040300091E002C086E391E0E80FF91F81818F9340
:1040400080818F938AED9BE09F938F930E949E4681
:10405000E091DC0BF091DD0BEE5CFE4F6081718135
:104060008AED9BE00E946146E091DC0BF091DD0B54
:10407000809103010F900F900F900F9081FF03C06C
:1040800088E391E002C086E391E0E80FF91F8181A7
:104090008F9380818F938AED9BE09F938F930E94F3
:1040A0009E46E091DC0BF091DD0BEC5CFE4F6081F5
:1040B00071818AED9BE00E946146E091DC0BF091FA
:1040C000DD0B0F900F900F900F904B9B03C088E378
:1040D00091E002C086E391E0E80FF91F81818F93A0
:1040E00080818F938AED9BE09F938F930E949E46E1
:1040F0000F900F900F900F900C94B52884E40E94BD
:10410000872B882311F40C94B5280E94B72B20E04C
:1041100030E040E05FE30E9485CE6B017C0120E04F
:1041200030E0A9010E946CD3882379F0A7019601A1
:10413000C701B6010E9485CE2BED3FE049E450E473
:104140000E9485CE9B01AC0104C020E030E040E835
:104150005FE38091210A8093281784E522962FAF90
:10416000229723963FAF239724964FAF2497259607
:104170005FAF25970E94872B22962FAD229723961B
:104180003FAD239724964FAD249725965FAD259795
:10419000882309F446C00E94B72B0E9447D8609339
:1041A000281722962FAD229723963FAD239724966A
:1041B0004FAD249725965FAD2597623090F11F9201
:1041C0006F931F9288EC8F938AED9BE0E091DC0B5C
:1041D000F091DD0BE85BFE4F61816F9360816F931F
:1041E0009F938F9322962FAF229723963FAF2397CB
:1041F00024964FAF249725965FAF25970E949E4641
:104200000FB6F894DEBF0FBECDBF25965FAD2597E4
:1042100024964FAD249723963FAD239722962FAD3A
:1042200022970091281794E0099F80011124075FCD
:104230001D4F60E070E080E89FE30E94D0D7F80156
:10424000608371838283938390C7F70181917F019B
:104250000E94872B882369F00E94B72B9801285170
:104260003D4E69010E9447D8F601608371838283C5
:1042700093830C5F1F4F0031110539F70E94BF7FF8
:1042800074C718E3E12E12E1F12E06E015E084E098
:10429000D82ED00EF80181918F010E94872B8823A0
:1042A00039F00E94B72BF701648B758B868B978B47
:1042B000F4E0EF0EF11CD012EDCF57C783E50E945A
:1042C000872B882351F00E94B72B60936012709364
:1042D0006112809362129093631284E50E94872B8F
:1042E000882351F00E94B72B60936412709365127B
:1042F00080936612909367128DE40E94872B882327
:1043000009F433C70E94B72B609368127093691247
:1043100080936A1290936B1228C783E50E94872BC3
:10432000882351F00E94B72B60935C1270935D124A
:1043300080935E1290935F1284E50E94872B8823FE
:1043400051F00E94B72B60937C1270937D12809382
:104350007E1290937F1282E40E94872B882361F063
:104360000E94B72B0E9447D86093F8127093F912FD
:104370008093FA129093FB1288E50E94872B882382
:1043800091F00E94B72B609370127093711280931A
:1043900072129093731260936C1270936D128093EB
:1043A0006E1290936F128AE50E94872B882351F03A
:1043B0000E94B72B609374127093751280937612DB
:1043C0009093771285E40E94872B882309F4CDC649
:1043D0000E94B72B609378127093791280937A12AF
:1043E00090937B12C2C60C5F1F4F0C30110509F46D
:1043F000BCC6F70181917F010E94872B882399F326
:104400000E94B72BF801E058FD4E608371838283D0
:104410009383E9CF0091210A84E50E94872B8111C3
:1044200002C010E005C00E94B72B0E9441D88B014A
:1044300002301105CCF01F930F938AED9BE0E091C1
:10444000DC0BF091DD0BE65BFE4F21812F93208189
:104450002F939F938F930E949E460F900F900F90E3
:104460000F900F900F9081C68BE40E94872B9801CC
:104470002A5D3F4F4901882371F00E94B72BF40158
:10448000EE0FFF1FEE0FFF1FE85CFD4E6083718390
:104490008283938312C0F901EE0FFF1FEE0FFF1FFF
:1044A000E85CFD4E1082118212821382F801EE0F39
:1044B000FF1FE852FD4E1182108284E40E94872B78
:1044C000882371F00E94B72B9801220F331FA90196
:1044D00048525D4E7A010E9441D8F7017183608392
:1044E000E12CF12C2801012E000C66087708C4018C
:1044F000880F991F880F991F9C01285C3D4E490128
:10450000C801880F991FAC0148525D4E6A018AEDBF
:104510009BE00E94EB2AE016F106E1F5EAE0AE2E00
:10452000E5E0BE2EF50181915F01882319F00E941C
:1045300070BDF8CFC301B2010E94DBB47EE0A72EAC
:1045400075E0B72EF50181915F01882319F00E9473
:1045500070BDF8CFF401608171818281938142E066
:104560000E94CAA962E1A62E65E0B62EF5018191EE
:104570005F01882319F00E9470BDF8CFF6016081B9
:104580007181072E000C880B990B0E94DBB48AE026
:104590000E9470BDEA94EF2809F4E7C5EE24E39485
:1045A000F12CB5CF8AED90E00E9477BD8111DDC579
:1045B00088E50E94872B882381F00091281710E05E
:1045C0000E94B72B000F111F000F111FF801EC54B0
:1045D000FD4E608371838283938389E50E94872BDC
:1045E000882381F00091281710E00E94B72B000F5C
:1045F000111F000F111FF801E454FD4E60837183F9
:1046000082839383E091DC0BF091DD0BE25CFE4F43
:10461000608171818AED9BE0A1D71092281702EE8C
:1046200011E03AEDE32E3BE0F32E80912817823023
:1046300008F09BC5E82FF0E0DF01AA0FBB1FAA0F0F
:10464000BB1FA454BD4E13969C9113979F93129633
:104650009C9112979F9311969C9111979F939C9177
:104660009F93EE0FFF1FEE0FFF1FEC54FD4E938143
:104670009F9392819F9391819F9390819F931F928B
:104680008F931F930F93FF92EF920E949E4680910B
:1046900028178F5F809328170FB6F894DEBF0FBEE0
:1046A000CDBFC3CF83E50E94872B882309F45DC566
:1046B0000E94B72B0E9441D870932A02609329026E
:1046C00054C583E50E94872B882309F44EC50E94B8
:1046D000B72B0E9441D86B017C0184E50E94872B97
:1046E000882381F08DED90E00E9477BD81113DC55A
:1046F000E0912817F0E0EE0FFF1FED5FFD4FD18234
:10470000C08233C5D0920802C09207022EC580E550
:10471000FED7882309F429C50E94B72B83E5F7D774
:10472000882309F422C50E94B72B1FC585E4EFD763
:10473000882331F00E94B72B0E9441D88B0102C020
:1047400000E010E082E4E3D7811105C002301105DA
:104750000CF0B3C102C00FEF1FEF80E5D8D788235C
:10476000C1F00E94B72B17FF09C06093C412709369
:10477000C5128093C6129093C7120BC0F801EE0FBA
:10478000FF1FEE0FFF1FE457FD4E6083718382838E
:10479000938389E4BCD7882341F1E9D717FF0FC081
:1047A0002DEB37E346E05EE30E9485CE6093C812AE
:1047B0007093C9128093CA129093CB1214C09801BF
:1047C000220F331F220F331FA9014C565D4E7A0171
:1047D0002DEB37E346E05EE30E9485CEF701608370
:1047E0007183828393830E94F6B484E490D78823F4
:1047F00041F1BDD717FF0FC02DEB37E346E05EE375
:104800000E94D0D76093CC127093CD128093CE12B9
:104810009093CF1214C09801220F331F220F331F21
:10482000A90144565D4E7A012DEB37E346E05EE385
:104830000E94D0D7F70160837183828393830E94A3
:10484000F6B483E464D78823B9F091D717FD14C078
:104850009801220F331F220F331FA9014C555D4EC3
:104860007A012DEB37E346E05EE30E9485CEF70147
:10487000608371838283938386E449D78823B9F068
:1048800076D717FD14C09801220F331F220F331F54
:10489000A90144555D4E7A012DEB37E346E05EE316
:1048A0000E9485CEF70160837183828393838CE4B9
:1048B0002ED7882339F05BD70E9441D87093E30547
:1048C0006093E2058091E2059091E305C39734F08F
:1048D00082E390E09093E3058093E2050E94F6B4B2
:1048E0008AED9BE078D61F930F938AED9BE0E091D1
:1048F000DC0BF091DD0BE057FE4F21812F932081DF
:104900002F939F938F930E949E460F900F900F902E
:104910000F900F900F9017FF2AC02DEB37E346E062
:104920005EE36091CC127091CD128091CE12909185
:10493000CF120E9485CEF62EE72ED82EC92E2DEB53
:1049400037E346E05EE36091C8127091C91280912E
:10495000CA129091CB120E94D0D79B014091C412F1
:104960005091C5126091C6127091C71232C0F80101
:10497000EE0FFF1FEE0FFF1FE456FD4E2DEB37E34A
:1049800046E05EE360817181828193810E9485CEE1
:10499000F62EE72ED82EC92EF801EE0FFF1FEE0FD0
:1049A000FF1FEC56FD4E2DEB37E346E05EE36081E2
:1049B0007181828193810E94D0D79B01F801EE0F13
:1049C000FF1FEE0FFF1FE457FD4E408151816281B2
:1049D0007381CF92DF92EF92FF929F938F933F93D9
:1049E0002F937F936F935F934F938AED9BE0E091BA
:1049F000DC0BF091DD0BEE56FE4F21812F932081D1
:104A00002F939F938F930E949E460FB6F894DEBF1C
:104A10000FBECDBF17FD17C0F801EE0FFF1FEE0F41
:104A2000FF1FE455FD4E4081518162817381000F6B
:104A3000111F000F111FF801EC55FD4E808191816F
:104A40002281338108C040E050E060E070E080E007
:104A500090E020E030E07F936F935F934F933F931C
:104A60002F939F938F938AED9BE0E091DC0BF09165
:104A7000DD0BEC56FE4F21812F9320812F939F93C6
:104A80008F930E949E460AE115E00FB6F894DEBFB0
:104A90000FBECDBFF80181918F01882319F00E94CC
:104AA00070BDF8CF6091E2057091E305072E000C10
:104AB000880B990B0E94DBB458C31F930F9381E0BE
:104AC0008F938DE28F938AED9BE0E091DC0BF09168
:104AD000DD0BE85BFE4F21812F9320812F939F9365
:104AE0008F930E949E460FB6F894DEBF0FBECDBFD7
:104AF0003CC383E50CD6882311F039D603C060E0AF
:104B000070E0CB010E9441D87093B20A6093B10A61
:104B10002CC30E94478029C30E94618B26C30E9438
:104B2000758023C3882339F00E94D04F0F5F1F4F39
:104B3000F8018491F7CF8AE00E94D04F8AED9BE084
:104B40004AD5409160125091611260916212709149
:104B5000631289EF92E00E94773D40916412509178
:104B60006512609166127091671286EF92E00E9462
:104B7000773D8AE00E94D04F8AED9BE02CD5E3E49C
:104B8000F2E084918F01882339F00E94D04F0F5FAB
:104B90001F4FF8018491F7CF8AE00E94D04F8AED31
:104BA0009BE019D540915C1250915D1260915E12AC
:104BB00070915F128AE392E00E94773D40917C12EF
:104BC00050917D1260917E1270917F1287E392E086
:104BD0000E94773DC090F812D090F912E090FA123E
:104BE000F090FB12E4E3F2E084918F01882339F026
:104BF0000E9470BD0F5F1F4FF8018491F7CF4AE00C
:104C0000C701B6010E9454B440916C1250916D12CC
:104C100060916E1270916F1281E392E00E94773D75
:104C200040917412509175126091761270917712C2
:104C30008EE292E00E94773D409178125091791275
:104C400060917A1270917B128BE292E00E94773D24
:104C50008AE00E94D04F8AED9BE0BDD4E9E1F2E00A
:104C600084918F01882339F00E94D04F0F5F1F4F2E
:104C7000F8018491F7CF8AE00E94D04F8AED9BE043
:104C8000AAD4409180125091811260918212709149
:104C9000831286E192E00E94773D40918412509108
:104CA0008512609186127091871283E192E00E94D2
:104CB000773D409188125091891260918A127091CB
:104CC0008B1280E192E00E94773D8AE00E94D04FF3
:104CD0008AED9BE080D460E070E087E092E00E9483
:104CE000933D40918C1250918D1260918E12709173
:104CF0008F1284E092E00E94773D2DEB37E346E08F
:104D00005EE3609194127091951280919612909149
:104D100097120E94D0D7AB01BC0181E092E00E94C3
:104D2000773D2DEB37E346E05EE360919C12709196
:104D30009D1280919E1290919F120E9485CEAB0190
:104D4000BC018EEF91E00E94773D4091A4125091FA
:104D5000A5126091A6127091A7128BEF91E00E94AC
:104D6000773D4091AC125091AD126091AE127091AE
:104D7000AF1288EF91E00E94773D6091E20570915B
:104D8000E30585EF91E00E94933D8AE00E94D04FB9
:104D90008AED9BE020D461E070E087E092E00E9421
:104DA000933D4091901250919112609192127091A6
:104DB000931284E092E00E94773D2DEB37E346E0CA
:104DC0005EE3609198127091991280919A1290917D
:104DD0009B120E94D0D7AB01BC0181E092E00E94FF
:104DE000773D2DEB37E346E05EE36091A0127091D2
:104DF000A1128091A2129091A3120E9485CEAB01C4
:104E0000BC018EEF91E00E94773D4091A812509135
:104E1000A9126091AA127091AB128BEF91E00E94DF
:104E2000773D4091B0125091B1126091B2127091E1
:104E3000B31288EF91E00E94773D8AE00E94D04F44
:104E400094C185E464D4811192D48AE560D481113F
:104E50008ED488E55CD481118AD489E558D4811137
:104E600086D48CE454D4811182D40E94D58D129AB8
:104E7000479A64E670E080E090E00E945457809189
:104E80004B0982FD03C00E94B3B3F9CF8CE43FD439
:104E9000882309F46AC16BD468C180910C09909190
:104EA0000D0916E0880F991F1A95E1F7845F994F55
:104EB0009F938F938AED9BE0E091DC0BF091DD0BEB
:104EC000E457FE4F21812F9320812F939F938F933F
:104ED0000E949E460F900F900F900F900F900F9092
:104EE00044C184E514D4882309F41CC140D40E9431
:104EF00041D84B015C0186E40AD4811138D4182DC5
:104F00001230D0F099249F928F928AED9BE0E0912D
:104F1000DC0BF091DD0BE65BFE4F21812F932081AE
:104F20002F939F938F930E949E460F900F900F9008
:104F30000F900F900F9019C10E94D58D0091210AFA
:104F4000801609F4D4C080E1E1E6FAE0A4E7BAE013
:104F500001900D928A95E1F77401FF2410E0F701AA
:104F6000EE0FFF1FEE0FFF1FEC54FD4ED801AA0FEE
:104F7000BB1FAA0FBB1FAC54BD4E2D913D914D914F
:104F80005C9160817181828193810E94E6D69B0150
:104F9000AC016091610A7091620A8091630A9091FC
:104FA000640A0E94E7D66093610A7093620A809354
:104FB000630A9093640AF701EE0FFF1FEE0FFF1FC5
:104FC000E454FD4E000F111F000F111FD801A4540F
:104FD000BD4E2D913D914D915C9160817181828199
:104FE00093810E94E6D69B01AC016091650A7091A5
:104FF000660A8091670A9091680A0E94E7D66093DA
:10500000650A7093660A8093670A9093680A809293
:10501000210A2DE63AE049E65AE065E67AE081E6C3
:105020009AE00E942B8D8091160C811102C00E9483
:105030006B8CE091210A24E0E29FF0011124E15AF7
:10504000F54F80916D0A90916E0AA0916F0AB09110
:10505000700A83AB94ABA5ABB6ABF701EE0FFF1FA5
:10506000EE0FFF1FE15AF54F63A974A985A996A910
:1050700060936D0A70936E0A80936F0A9093700A22
:10508000209148123091491240914A1250914B128E
:105090000E9485CE0E94DAD96093AE0C7093AF0C5B
:1050A0008093B00C9093B10C8FB7F8944091AE0CF4
:1050B0005091AF0C6091B00C7091B10C40931C0AF0
:1050C00050931D0A60931E0A70931F0A8FBF809130
:1050D0006D0A90916E0AA0916F0AB091700A809348
:1050E0000A0A90930B0AA0930C0AB0930D0A8091C0
:1050F000210A1F928F938AED9BE0E091DC0BF091E7
:10510000DD0BE45BFE4F21812F9320812F939F9332
:105110008F930E949E460F900F900F900F900F90CC
:105120000F9023C080910C0990910D0946E0880FE3
:10513000991F4A95E1F7845F994F9F938F938AED6A
:105140009BE0E091DC0BF091DD0BE457FE4F2181F9
:105150002F9320812F939F938F930E949E460F90B1
:105160000F900F900F900F900F900E946DC28BC107
:10517000F3D2AB01BC014093D8165093D91660937B
:10518000DA167093DB1680919316909194160E9414
:105190007A94EBCF61E0CE0181960E9441967C012A
:1051A000009711F40C94C01B0E946794B82E85EEF2
:1051B000F701808319A28FA198A580960E945A8337
:1051C000882311F40C94C01B9CA1992309F46BC093
:1051D00089A59AA5ABA5BCA50097A105B10549F481
:1051E0006FA178A5C8010E948795811113C00C9406
:1051F000C01B20E2F80111922A95E9F720E12983EA
:1052000021E02B832FA138A538872F838D8F9E8F88
:10521000AF8FB8A399249394F5EEAF2E8CA1891586
:1052200010F40C94C01BE92CF12C4DA15EA14E1979
:105230005F0960E070E0E5E0440F551F661F771FCF
:10524000EA95D1F7C8010E947A94882311F40C944E
:10525000C01B60E0C8010E943E95FC01892B11F43F
:105260000C94C01B83858F3011F00C94C01B2081DF
:10527000822F8F7190E0E816F90611F00C94C01B94
:105280008585B8120C94C01BA082EFA1F8A580A15F
:10529000816080A326FF05C0CF0180960E945A83BB
:1052A00002C09394BBCF882311F40C94C01BCF92FF
:1052B000DF928AED9BE0E091DC0BF091DD0BE05E8C
:1052C000FE4F21812F9320812F939F938F930E94D4
:1052D0009E461092D8161092D9161092DA16109295
:1052E000DB160F900F900F900F900F900F903DCF07
:1052F0003ED23BCF3CD24B015C010091281710E01D
:10530000000F111F0C55154F0E9441D8F8017183F1
:10531000608381E090E09093190C8093180C20E05A
:1053200030E040EA52E4C501B4010E946CD3181683
:105330003CF00E944EAA1092190C1092180C04C056
:105340008AE09CE00E94F749E091281724E0E29F60
:10535000F0011124E656F54F2281338144815581B5
:10536000C501B4010E942DD9181634F481E090E0F3
:105370009093190C8093180C0091281710E0F801F5
:10538000EE0FFF1FEC55F54F60817181072E000C69
:10539000880B990B0E9472D34B015C01F801EE0F50
:1053A000FF1FEE0FFF1FE656F54F22813381448128
:1053B00055810E946CD3881F8827881FF1100CC06C
:1053C00069F020E030E040EA52E4C501B4010E94F7
:1053D0006CD387FDCACE02C08111C7CE61E0C8017F
:1053E0000E946EB082E090E09093190C8093180CAC
:1053F000BCCE8AE09CE00E94F749E09128170E2F6E
:1054000010E0F801EE0FFF1FEC55F54F6081718140
:10541000072E000C880B990B0E9472D3F801EE0F37
:10542000FF1FEE0FFF1FE656F54F228133814481A7
:10543000558198CF0E94D58D88E569D1882319F0D0
:105440005F9A1092710A89E562D1882319F08A9ACD
:105450001092720A8AE55BD1882351F09FB7F894C5
:10546000809108018260809308019FBF1092730AA7
:1054700085E44DD1882309F478CE129A479A75CEE7
:105480000E94679172CECC5BDF4F0FB6F894DEBFFF
:105490000FBECDBFDF91CF911F910F91FF90EF9085
:1054A000DF90CF90BF90AF909F908F907F906F9044
:1054B0005F904F903F902F90089541155105B1F0A6
:1054C000FB0180818EBD4230510568F081813296AA
:1054D000460F571F0DB407FEFDCF8EBDE417F5072D
:1054E00011F08191F7CF0DB407FEFDCF08956EBD89
:1054F0000DB407FEFDCF089541155105D9F0415077
:1055000051098FEF8EBDFB012FEFCF01861B970B4B
:105510008417950738F40DB407FEFDCF8EB52EBD68
:105520008193F3CF0DB407FEFDCF8EB5FB01E40FE1
:10553000F51F808380E008958FEF8EBD0DB407FEC8
:10554000FDCF8EB508950895FC01228183812CBD85
:105550008DBD0895FC017383628308950F931F939B
:10556000CF93DF93EC018B01E881F9810480F58111
:10557000E02D68E574E01995E881F9810480F581F2
:10558000E02DB801CE011995E881F9810480F581FB
:10559000E02D66E574E0CE01DF91CF911F910F9170
:1055A00019940F931F93CF93DF93EC018B01E88144
:1055B000F9810480F581E02D60E574E01995E881BA
:1055C000F9810480F581E02DB801CE01DF91CF9102
:1055D0001F910F911994DC01ED91FC910480F581EC
:1055E000E02D6AE474E019940F931F93CF93DF9337
:1055F000EC018B01E881F9810480F581E02D63E401
:1056000074E01995E881F9810480F581E02DB801F5
:10561000CE011995E881F9810480F581E02D61E4DE
:1056200074E0CE01DF91CF911F910F911994DC01AD
:10563000ED91FC910480F581E02D6AE374E019940A
:10564000089561E0FC0184810C94E95660E0FC015E
:1056500084810C94E956CF93DF93EC01862F6C8301
:1056600061E00E94185761E08C810E94E956CFB733
:10567000F8948091F405811127C0EAE3F7E0849162
:10568000E0E8F7E09491E82FF0E0EE0FFF1FE95417
:10569000F94FA591B491EC91E92321F461E085E300
:1056A0000E94E95661E085E30E9418578CB580613D
:1056B0008CBD8CB580648CBD61E084E30E9418577A
:1056C00061E083E30E9418578091F4058F5F809317
:1056D000F405CFBFDF91CF910895682F880F770B26
:1056E00080910A0690910B0626E0880F991F2A9553
:1056F000E1F7845F994F0E94C4DB9C019093E10520
:105700008093E00581E0232B09F480E00895682F61
:10571000880F770B80910C0990910D0926E0880F76
:10572000991F2A95E1F7845F994F0E94C4DB9C0181
:105730009093E1058093E00581E0232B09F480E05C
:1057400008958091E0059091E1054AE050E060E025
:1057500070E001960C94CCD18091E0059091E10528
:105760004AE050E060E070E001960C94CCD180916A
:10577000E0059091E10560E070E001960C9466D040
:105780002F923F924F925F926F927F928F929F9251
:10579000AF92BF92CF92DF92EF92FF920F931F933F
:1057A000CF93DF93CDB7DEB7C755D1090FB6F894C5
:1057B000DEBF0FBECDBF85E4AADF882339F0D7DF77
:1057C0000E9441D81B0177FD0AC002C0212C312C58
:1057D0001C861D8A26E12E8B33E43E8706C01C867C
:1057E0001D8A4CE84E8B52E45E8783E590DF882368
:1057F00029F0BDDF6C877D8B8E8B9E8783E487DFEE
:10580000882331F0B4DF0E9441D87FAB6EAB04C077
:1058100087E090E09FAB8EAB85E579DF88AF84E5CC
:1058200076DF2E968FAF2E970E94E1C28091DC0B1F
:105830009091DD0BFC01A3E02A1631041CF0E05B23
:10584000FE4FA8C3EE5AFE4F608171818AED9BE046
:1058500085DE0E942FB683EB9AE00E94F749C101D2
:10586000880F991F880F991FFC01E456F54F7F019F
:1058700001E010E037FC0FC020E030E048EC52E4DB
:10588000D7016D917D918D919C910E942DD9181613
:1058900014F40C94403A1092B40A1092B30A109285
:1058A000B70A1092B80A1092B90A1092BA0A109266
:1058B000BB0A1092BC0A1092BD0A1092BE0A109246
:1058C000B60A1092B50A80E090E00E9411AD37FE52
:1058D00002C00C94AC3B0AED1BE0E091DC0BF091B4
:1058E000DD0BEC5AFE4F60817181C8010E94614658
:1058F00065E070E0C1010E94D5B560E0C1010E9481
:105900006EB069AF7AAF8BAF9CAF9F938F93BAADF8
:10591000BF93E9ADEF93E091DC0BF091DD0BEA5A18
:10592000FE4F81818F9380818F931F930F930E94ED
:105930009E460E94E1C262966CAF7DAF8EAF9FAF74
:1059400062976FEF70E0C1010E94D5B50FB6F89471
:10595000DEBF0FBECDBF39AD3E834AAD4F875BADD5
:10596000598B8CAD8F8B62968CAC9DACAEACBFACC2
:1059700062971E8E1AA21EA21AA61A8E1B8E188657
:105980001C8E1AAA1BAA1CAA1DAA2A961FAE2A9709
:105990002B961FAE2B972C961FAE2C972D961FAED5
:1059A0002D9719821B821C821D8222961FAE229780
:1059B00023961FAE239724961FAE249725961FAEDD
:1059C00025971DAE1EAE1FAE21961FAE21971EA6B7
:1059D0001FA690E898ABAFEBA9ABC101880F991F48
:1059E000880F991FFC01E456F54FF98FE88F0E944C
:1059F000E1C22091480B222311F40C94743ADC018B
:105A0000CB0188199909AA09BB0989309740A105DA
:105A1000B10510F40C94743A0E94F0AC1092480B4B
:105A2000A88DB98DBC91B983E88DF98DF181FB8387
:105A3000A88DB98D1296BC91BC83E88DF98DF38148
:105A4000FD830E94E1C22B013C017E816F85998913
:105A50008F89272F362F492F582F69817B818C8181
:105A60009D810E94E6D66B017C01C301B2016819D9
:105A700079098A099B090E9470D320E030E04AE747
:105A800054E40E94D0D79B01AC01C701B6010E942B
:105A9000D0D726966FAF269727967FAF2797289661
:105AA0008FAF289729969FAF29972AA93BA94CA980
:105AB0005DA92A966FAD2A972B967FAD2B972C96D2
:105AC0008FAD2C972D969FAD2D970E94E7D62A8DEE
:105AD0003B8D48855C8D0E94E7D62E8D3AA14EA164
:105AE0005AA50E94E7D626962FAD269727963FAD5A
:105AF000279728964FAD289729965FAD29970E9442
:105B0000E7D620E030E040EA50E40E94D0D7679624
:105B10006FAF679768967FAF6897182F092F9B0123
:105B2000482F592F6AA97BA98CA99DA90E94E6D666
:105B30002A8D3B8D48855C8D0E94E7D667962FADF8
:105B4000679768963FAD6897412F502F0E94E6D621
:105B50002E8D3AA14EA15AA50E94E7D667962FAD89
:105B6000679768963FAD6897412F502F0E94E6D601
:105B700026962FAD269727963FAD279728964FADAF
:105B8000289729965FAD29970E94E7D667962FAD93
:105B9000679768963FAD6897412F502F0E94E6D6D1
:105BA0002A962FAD2A972B963FAD2B972C964FAD6B
:105BB0002C972D965FAD2D970E94E7D667962FAD57
:105BC000679768963FAD6897412F502F0E94E6D6A1
:105BD00027E137EB41ED58E30E94E7D66B017C01EA
:105BE00020E030E0A9010E942DD9181614F40C947D
:105BF000B23BA701960150586EA57FA588A999A927
:105C00000E94E6D69B01AC0167966FAD67976896D8
:105C10007FAD6897812F902F0E946CD387FD02C0C3
:105C20000C94B63B2DEC3CEC4CEC5DE367966FAD11
:105C3000679768967FAD6897812F902F0E942DD926
:105C4000181614F00C94BF3B60E070E0C1010E9494
:105C5000D5B5C501B40162962CAD3DAD4EAD5FAD7D
:105C60006297621B730B840B950B0E9470D320E02C
:105C700030E04AE754E40E94D0D76B017C0179AD53
:105C80006AAD9BAD8CAD272F362F492F582FBE8183
:105C9000AF85F989EF896B2F7A2F8F2F9E2F0E9466
:105CA000E6D62EA53FA548A959A90E94D0D79B01A9
:105CB000AC01C701B6010E94E6D622966FAF2297CB
:105CC00023967FAF239724968FAF249725969FAF77
:105CD00025973EA567963FAF67974FA568964FAF4C
:105CE000689718A909A93DAF4EAF1FAF21960FAF16
:105CF000219780E066968FAF66970E947CAA3AA9AA
:105D00002A963FAF2A974BA92B964FAF2B975CA9AA
:105D10002C965FAF2C979DA92D969FAF2D97AA8D9E
:105D2000AAABBB8DBBABE885ECABFC8DFDAB2E8D80
:105D30002A8F3AA13B8F4EA148875AA55C8F2696A1
:105D40009FAD26979E8F2796AFAD2797AAA328963B
:105D5000BFAD2897BEA32996EFAD2997EAA767960E
:105D6000FFAD6797FEA768962FAD68972FA718AB72
:105D700009AB5301420166968FAD669766968FAF69
:105D800066970E94765C66968FAD669781112FCEDE
:105D900025963FAD25973F9324964FAD24974F937B
:105DA00023965FAD23975F9322968FAD22978F93B3
:105DB00021969FAD21979F93AFADAF93BEADBF939B
:105DC000EDADEF938CE295E09F938F93BAED4B2E60
:105DD000BBE05B2E5F924F920E949E462296EFACF4
:105DE00022972396FFAC239724960FAD24972596F0
:105DF0001FAD25979701A801BDADAEADFFAD2196B2
:105E0000EFAD21976B2F7A2F8F2F9E2F0E9485CE7B
:105E10009B01AC0160E070E089E993E40E94D0D777
:105E2000D62EC72EB82EA92E20E030E040E05FE34A
:105E3000D601F5016B2F7A2F8F2F9E2F0E9485CED2
:105E40002E2D3F2D402F512F0E94D0D7962E872EDA
:105E5000782E692E2AE939E949E95EE3D601F50190
:105E60006B2F7A2F8F2F9E2F0E9485CE2E2D3F2DA8
:105E7000402F512F0E9485CE162F072FF82EE92E86
:105E80006DE175E0C2010E946146EF92FF920F93AF
:105E90001F936F927F928F929F92AF92BF92CF92F9
:105EA000DF9284E095E09F938F935F924F920E94E0
:105EB0009E460FB6F894DEBF0FBECDBF0E94E1C272
:105EC0006B017C0137FC02C00C94773A8FEF90E0B5
:105ED0000E94ADB562EF74E08AED9BE00E946146DE
:105EE000C98ADA8AEB8AFC8ACAA6DBA6ECA6FDA6DA
:105EF000512C412C3AE739AB44E44AAB1F8A188E47
:105F00001A8E1B8E8FEF90E09F838E8366246A9497
:105F1000712C1EA21FA218A619A61AA21BA21CA2AF
:105F20001DA21E8E1F8E18A219A291E09887188AB2
:105F30001F86AC85AEA7BD89BFA7EE89E8ABC101BE
:105F4000880F991F880F991F9C012456354F3D8F4C
:105F50002C8F8091480B81110C947E3A20E030E028
:105F600040EA51E46C857D898E899E850E94E7D642
:105F70009B01AC0169817B818C819D810E942DD91F
:105F8000181614F00C94173BE091DC0BF091DD0B2C
:105F9000E85AFE4F608171818AED9BE025DBDCC011
:105FA0008F859889AEA9BFA9A817B90714F00C94DA
:105FB000A83BBD01BB0F880B990B0E9472D320E058
:105FC00030E040E050E40E94E6D64B015C019B01CA
:105FD000AC016E8D7F8D88A199A10E94D0D78B01D5
:105FE000782E692EA50194016AA17BA18CA19DA1A7
:105FF0000E94D0D75B016C01DF928F93BF926F93A9
:106000006F927F921F930F9386E894E09F938F93F4
:106010006AEDE62E6BE0F62EFF92EF920E949E460E
:1060200020E030E040E05FE3F301602F712F8F2F1D
:106030009E2F0E9485CE8B01582E492E2A2D3B2D56
:106040004C2D5D2DF201602F712F8F2F9E2F0E94FE
:10605000D0D73B014C012AE939E949E95EE3F20175
:10606000602F712F8F2F9E2F0E9485CE2A2D3B2DC2
:106070004C2D5D2D0E9485CE5B016C0167E774E0BD
:10608000C7010E946146DF92CF92BF92AF929F926A
:106090008F927F926F924F925F921F930F938EE534
:1060A00094E09F938F93FF92EF920E949E460FB6CB
:1060B000F894DEBF0FBECDBFF8ADFF2311F40C94F2
:1060C0009A3B37FC02C00C94573B9201802F912FD2
:1060D000A32FB22F8093C4129093C512A093C6121F
:1060E000B093C7122DEB37E346E05EE3662D772DC4
:1060F000882D992D0E9485CE6093C8127093C91285
:106100008093CA129093CB120E94F6B437FC02C05F
:106110000C94813B2DEB37E346E05EE36A2D7B2D4B
:106120008C2D9D2D0E94D0D76093CC127093CD12F0
:106130008093CE129093CF120E94F6B4E091DC0BC4
:10614000F091DD0BE25AFE4F608171818AED9BE098
:106150000E9461460E94F6B48091710A882341F042
:106160008091720A882321F08091730A81110DC0F9
:106170002E96FFAD2E97FF2311F40C945D3D41E068
:1061800061E081E00E94218F07C02E962FAD2E97EF
:10619000222311F40C945D3DE091DC0BF091DD0BBA
:1061A000EE59FE4F608171818AED9BE00E9461464D
:1061B0003091210A3F872092210A37FE0BC06C855F
:1061C0007D898E899E850E9441D87093AD0A609327
:1061D000AC0A0FC0C101880F991F8C010C55154FD7
:1061E0006C857D898E899E850E9441D8D8016D93EA
:1061F0007C9381E090E09093190C8093180CE091CF
:10620000DC0BF091DD0BEC59FE4F608171818AED62
:106210009BE00E94614680E090E0A8ECB2E48093AD
:10622000740A9093750AA093760AB093770A8093C4
:10623000780A9093790AA0937A0AB0937B0A80E057
:1062400090E0A0E8BFE380937C0A90937D0AA0933E
:106250007E0AB0937F0A80916D0A90916E0AA09198
:106260006F0AB091700A8093800A9093810AA0937C
:10627000820AB093830A0E946B8C80E090E00E94B7
:1062800011AD1092B40A1092B30A1092B70A10928C
:10629000B80A1092B90A1092BA0A1092BB0A109268
:1062A000BC0A1092BD0A1092BE0A1092B60A109251
:1062B000B50AE091DC0BF091DD0BE059FE4F6081F7
:1062C00071818AED9BE00E94614683EB9AE00E9417
:1062D000F74983EB9AE00E94D0494E9728F40E9438
:1062E00028AD0E94765CF5CF1092B40A1092B30AE2
:1062F0001092B70A1092B80A1092B90A1092BA0A0C
:106300001092BB0A1092BC0A1092BD0A1092BE0AEB
:106310001092B60A1092B50A61E0C1010E946EB0F7
:10632000F62EE72E982E892E14E0C12ED12CF101E5
:106330003596FF83EE83CF01880F991F9C01265667
:10634000354F5901D5016D917C91072E000C880BBA
:10635000990B0E9472D3D701F4012B2F3E2D4F2FA2
:10636000582D0E94E6D62B013C0120E030E0A90127
:106370000E942DD90091DC0B1091DD0B18160CF04A
:1063800041C020E030E040E050E4C301B2010E948F
:106390002DD918160CF440C08F929F92EF92FF9265
:1063A000BAEDEB2EBBE0FB2EF801EA5AFE4F8181DD
:1063B0008F9380818F93FF92EF920E949E4648E8D0
:1063C00053E160E070E0C1010E94C58B2B013C01EC
:1063D0007F926F925F926F938DEB95E09F938F9377
:1063E000FF92EF920E949E4680E890E00E9411ADDD
:1063F00083EB9AE00E94F7490FB6F894DEBF0FBE18
:10640000CDBF21C020E030E040E050ECC301B2013C
:106410000E946CD387FFC0CFF1E0CF1AD10809F4F6
:10642000BBCFF801EE58FE4F608171818AED9BE091
:106430000E94614661E0C1010E946EB0F62EE72E17
:10644000982E892E7FCF83EB9AE00E94D049449703
:1064500028F40E9428AD0E94765CF5CF1092B40A11
:106460001092B30A1092B70A1092B80A1092B90AA1
:106470001092BA0A1092BB0A1092BC0A1092BD0A7E
:106480001092BE0A1092B60A1092B50A61E0C101DC
:106490000E946EB0D62EC72EF82EE92E00E010E036
:1064A0008E819F81880F991F9C012656354F3A8314
:1064B0002983A981BA816D917C91072E000C880BEC
:1064C000990B0E9472D3D601F7012B2F3C2D4F2F31
:1064D0005E2D0E94E6D64B015C0120E030E0A90170
:1064E0000E942DD918165CF420E030E040E050E422
:1064F000C501B4010E942DD918165CF025C020E01A
:1065000030E040E050ECC501B4010E946CD387FF3D
:106510001BC00330110509F4C4C0E091DC0BF091FD
:10652000DD0BEE58FE4F608171818AED9BE00E9489
:10653000614661E0C1010E946EB0D62EC72EF82ED2
:10654000E92E0F5F1F4FB5CF0330110509F4A9C025
:10655000EF92FF92CF92DF920AED1BE0E091DC0B0D
:10656000F091DD0BEA5AFE4F81818F9380818F93EA
:106570001F930F930E949E4648E853E160E070E04D
:10658000C1010E94C58B9F938F937F936F9322EBE2
:1065900035E03F932F931F930F9363966FAF6397ED
:1065A00064967FAF649766968FAF669765969FAF48
:1065B00065970E949E4663966FAD639764967FAD24
:1065C000649766968FAD669765969FAD65976419DB
:1065D0007509860997090E9470D32DEB37E346E0D1
:1065E0005EE30E9485CE20E030E040EA50E40E9465
:1065F000D0D76B017C018E819F81880F991F8656B1
:10660000954FFC01608171810FB6F894DEBF0FBE1B
:10661000CDBF77FF02C06D5F7F4F7595679575950C
:106620006795072E000C880B990B0E9472D39B0173
:10663000AC01C701B6010E94E6D66B017C016091F6
:10664000AE0A7091AF0A072E000C880B990B0E94BE
:1066500072D39B01AC01C701B6010E94D0D76C83F5
:106660007D838E839E879F938F933D813F934C8143
:106670004F9383EA95E09F938F938AED9BE09F93DE
:106680008F930E949E4680EC90E00E9411AD83EBB8
:106690009AE00E94F7490FB6F894DEBF0FBECDBF57
:1066A00049C18091AE0A9091AF0A40970E9411AD06
:1066B00061E0C1010E946EB0162F072FF82EE92E5F
:1066C0008E819F81880F991FDC01A656B54F6D0101
:1066D000F60160817181072E000C880B990B0E94D6
:1066E00072D39B01AC01D801F7016B2F702F8F2F54
:1066F0009E2D0E94E6D64B015C0120E030E0A9010E
:106700000E942DD91816D4F420E030E040E450E483
:10671000C501B4010E942DD91816D4F48091AE0A97
:106720009091AF0A40970E9411AD61E0C1010E94B3
:106730006EB0162F072FF82EE92ECACF20E030E0DA
:1067400040E450ECC501B4010E946CD387FDE6CF54
:10675000EF92FF920F931F935AEDC52E5BE0D52E5B
:10676000E091DC0BF091DD0BEA5AFE4F81818F93B3
:1067700080818F93DF92CF920E949E4648E853E13A
:1067800060E070E0C1010E94C58B9F938F937F935F
:106790006F9328E935E03F932F93DF92CF92639672
:1067A0006FAF639764967FAF649766968FAF669777
:1067B00065969FAF65970E949E46C090AE0AD090A6
:1067C000AF0A63966FAD639764967FAD64976696E4
:1067D0008FAD669765969FAD6597641975098609B3
:1067E00097090E9470D32DEB37E346E05EE30E94E9
:1067F00085CE20E030E040EA50E40E94D0D74B0143
:106800005C018E819F81880F991F8656954FDC0110
:106810006D917C910FB6F894DEBF0FBECDBF77FFB0
:1068200002C06D5F7F4F7595679575956795072ECB
:10683000000C880B990B0E9472D39B01AC01C5011F
:10684000B4010E94E6D64B015C01B6010D2C000C90
:10685000880B990B0E9472D39B01AC01C501B40156
:106860000E94D0D74B015C01BF928F939F926F9390
:1068700024E62C9DC0012D9D900D11246FEF70E03A
:106880000E9485DA7F936F9389E895E09F938F93B9
:106890004AEDC42E4BE0D42EDF92CF920E949E464A
:1068A000BF92AF929F928F9280E895E09F938F93D3
:1068B000DF92CF920E949E460FB6F894DEBF0FBEC5
:1068C000CDBF38AD3323D9F037FC19C0C101880FD3
:1068D000991F880F991FAC0144555D4E6A012DEB3D
:1068E00037E346E05EE3682D792D8A2D9B2D0E94CB
:1068F00085CED6016D937D938D939C931397EF92E4
:10690000FF920F931F938AED9BE0E091DC0BF091D7
:10691000DD0BEA58FE4F21812F9320812F939F9307
:106920008F930E949E4680E090E00E9411AD0E94ED
:10693000F6B464C183EB9AE00E94D049449728F4EE
:106940000E9428AD0E94765CF5CF1092B40A109296
:10695000B30A1092B70A1092B80A1092B90A1092AC
:10696000BA0A1092BB0A1092BC0A1092BD0A109289
:10697000BE0A1092B60A1092B50A8AED9BE0E09129
:10698000DC0BF091DD0BE25BFE4F21812F93208128
:106990002F939F938F930E949E4661E0C1010E94B6
:1069A0006EB0D62EC72E89839B830F900F900F90C9
:1069B0000F90E12CF12C81010B5F1F4FC801880F54
:1069C000991F9C012656354F3D872C87AC85BD8588
:1069D0006D917C91072E000C880B990B0E9472D34D
:1069E000D601F981EB812B2F3C2D4F2F5E2F0E947A
:1069F000E6D64B015C0120E030E0A9010E942DD9D0
:106A0000E091DC0BF091DD0BF987E88718165CF458
:106A100020E030E040E050E4C501B4010E942DD9EF
:106A200018165CF025C020E030E040E050ECC501D5
:106A3000B4010E946CD387FF1BC0F3E0EF16F10492
:106A400009F4C4C0E885F985EE58FE4F6081718174
:106A50008AED9BE00E94614661E0C1010E946EB038
:106A6000D62EC72E89839B833FEFE31AF30AAECF5E
:106A700023E0E216F10409F4A9C03B813F93498168
:106A80004F93CF92DF92FAEDEF2EFBE0FF2EE885D9
:106A9000F985EA5AFE4F81818F9380818F93FF920F
:106AA000EF920E949E4648E853E160E070E0C10129
:106AB0000E94C58B9F938F937F936F9325E735E05B
:106AC0003F932F93FF92EF9263966FAF6397649615
:106AD0007FAF649766968FAF669765969FAF659711
:106AE0000E949E4663966FAD639764967FAD6497F0
:106AF00066968FAD669765969FAD65976419750923
:106B0000860997090E9470D32DEB37E346E05EE3D8
:106B10000E9485CE20E030E040EA50E40E94D0D7C9
:106B20006B017C01000F111FF801E656F54F6081E3
:106B300071810FB6F894DEBF0FBECDBF77FF02C0E4
:106B40006D5F7F4F7595679575956795072E000C5E
:106B5000880B990B0E9472D39B01AC01C701B6014F
:106B60000E94E6D66B017C016091AE0A7091AF0A7B
:106B7000072E000C880B990B0E9472D39B01AC016D
:106B8000C701B6010E94D0D76B837C878D8B9E8B0B
:106B90009F938F939C859F93AB81AF9386E695E0FF
:106BA0009F938F938AED9BE09F938F930E949E46C5
:106BB0008FEF90E00E9411AD83EB9AE00E94F749BD
:106BC0000FB6F894DEBF0FBECDBF1EC0FB81FF9392
:106BD00029812F93CF92DF928AED9BE0E885F9859A
:106BE000EA58FE4F21812F9320812F939F938F93FB
:106BF0000E949E4680E090E00E9411AD0FB6F8948E
:106C0000DEBF0FBECDBF9EC183EB9AE00E94D0498C
:106C10004E9728F40E9428AD0E94765CF5CF109222
:106C2000B40A1092B30A1092B70A1092B80A1092DE
:106C3000B90A1092BA0A1092BB0A1092BC0A1092BA
:106C4000BD0A1092BE0A1092B60A1092B50A61E00F
:106C5000C1010E946EB0162F072FB82EA92E812CCD
:106C6000912CC10105969A838983880F991FDC01B5
:106C7000A656B54FBA8BA98BE989FA8960817181D3
:106C8000072E000C880B990B0E9472D3D801F501D6
:106C90002B2F302F4F2F5A2D0E94E6D66B017C01EF
:106CA00020E030E0A9010E942DD92091DC0B309129
:106CB000DD0B3987288718165CF420E030E040E0CF
:106CC00050E4C701B6010E942DD918165CF025C00A
:106CD00020E030E040E050ECC701B6010E946CD3E8
:106CE00087FF1BC033E08316910409F40CC1E885CB
:106CF000F985EE58FE4F608171818AED9BE00E941C
:106D0000614661E0C1010E946EB0162F072FB82EB8
:106D1000A92EBFEF8B1A9B0AAFCF43E084169104D4
:106D200009F4F1C0AF92BF920F931F930AED1BE0DD
:106D3000E885F985EA5AFE4F81818F9380818F9390
:106D40001F930F930E949E4648E853E160E070E075
:106D5000C1010E94C58B9F938F937F936F932BE507
:106D600035E03F932F931F930F9363966FAF639715
:106D700064967FAF649766968FAF669765969FAF70
:106D800065970E949E4663966FAD639764967FAD4C
:106D9000649766968FAD669765969FAD6597641903
:106DA0007509860997090E9470D32DEB37E346E0F9
:106DB0005EE30E9485CE20E030E040EA50E40E948D
:106DC000D0D76B017C01E981FA81EE0FFF1FE656F7
:106DD000F54F608171810FB6F894DEBF0FBECDBF55
:106DE00077FF02C06D5F7F4F7595679575956795C5
:106DF000072E000C880B990B0E9472D39B01AC01EB
:106E0000C701B6010E94E6D66B017C018091AE0AF3
:106E10009091AF0ABC01990F880B990B0E9472D315
:106E20009B01AC01C701B6010E94D0D79F938F93FD
:106E30007F936F932BE435E03F932F930AED1BE094
:106E40001F930F9363966FAF639764967FAF6497BA
:106E500066968FAF669765969FAF65970E949E4630
:106E6000BC81AD81FE81EE852B2F3A2F4F2F5E2FF7
:106E700063966FAD639764967FAD649766968FADAA
:106E8000669765969FAD65970E94E7D6EB81BC85B6
:106E9000AD89FE892E2F3B2F4A2F5F2F0E94E7D608
:106EA00020E030E040E450E40E94D0D79F938F93DD
:106EB0007F936F9322E435E03F932F931F930F93BB
:106EC00063966FAF639764967FAF649766968FAF54
:106ED000669765969FAF65970E949E460FB6F89499
:106EE000DEBF0FBECDBF63966FAD639764967FAD77
:106EF000649766968FAD669765969FAD6597B8ADBA
:106F0000BB23E1F005C0AF92BF920F931F9364CEF5
:106F100037FC14C09101220F331F220F331F890148
:106F200004551D4E2DEB37E346E05EE30E9485CE0F
:106F3000D8016D937D938D939C93139780E090E09F
:106F40000E9411AD80E090E0A8ECB2E48093740A56
:106F50009093750AA093760AB093770A8093780A83
:106F60009093790AA0937A0AB0937B0A80937C0A63
:106F700090937D0AA0937E0AB0937F0A80916D0A58
:106F800090916E0AA0916F0AB091700A8093800A66
:106F90009093810AA093820AB093830A0E946B8C1B
:106FA00037FC0BC0F101EE0FFF1FEE0FFF1FEC557A
:106FB000FD4E10821182128213828091610A90919B
:106FC000620AA091630AB091640A8093740A909354
:106FD000750AA093760AB093770A8091650A90911A
:106FE000660AA091670AB091680A8093780A909324
:106FF000790AA0937A0AB0937B0A8091690A9091EA
:107000006A0AA0916B0AB0916C0A80937C0A9093F3
:107010007D0AA0937E0AB0937F0A20E030E040EA28
:1070200051E460916D0A70916E0A80916F0A90919F
:10703000700A0E94E7D66093800A7093810A809359
:10704000820A9093830A0E946B8C0AED1BE0E09108
:10705000DC0BF091DD0BEA59FE4F60817181C801B4
:107060000E946146C8010E94EB2A61E0C1010E94B2
:107070006EB061E0C1010E946EB09F938F937F93C9
:107080006F93E091DC0BF091DD0BEA5AFE4F8181AA
:107090008F9380818F931F930F930E949E4648EA9F
:1070A00051E660E070E0C1010E94C58B6B017C017C
:1070B00061E0C1010E946EB09F938F937F936F93A5
:1070C000E091DC0BF091DD0BEA5AFE4F81818F934A
:1070D00080818F931F930F930E949E468091610A37
:1070E0009091620AA091630AB091640A8093740A35
:1070F0009093750AA093760AB093770A8091650AF7
:107100009091660AA091670AB091680A8093780A04
:107110009093790AA0937A0AB0937B0A8091690AC6
:1071200090916A0AA0916B0AB0916C0A80937C0AD4
:1071300090937D0AA0937E0AB0937F0A20E030E00E
:1071400040E251E460916D0A70916E0A80916F0A7D
:107150009091700A0E94E7D66093800A7093810A2A
:107160008093820A9093830A0E946B8C48EA51E6CE
:1071700060E070E0C1010E94C58B6C197D098E0929
:107180009F092AE030E040E050E00E94ABD6490180
:107190005A019F922F931F928AE08F93E091DC0B0C
:1071A000F091DD0BE859FE4F81818F9380818F93A1
:1071B0001F930F930E949E4661E0C1010E946EB032
:1071C0009F938F937F936F93E091DC0BF091DD0B96
:1071D000EA5AFE4F81818F9380818F931F930F9383
:1071E0000E949E468091610A9091620AA091630A72
:1071F000B091640A8093740A9093750AA093760AFA
:10720000B093770A8091650A9091660AA091670A07
:10721000B091680A8093780A9093790AA0937A0AC9
:10722000B0937B0A8091690A90916A0AA0916B0AD7
:10723000B0916C0A80937C0A90937D0AA0937E0A99
:10724000B0937F0A20E030E040EA50E460916D0A9C
:1072500070916E0A80916F0A9091700A0E94E7D631
:107260006093800A7093810A8093820A9093830AC4
:107270000FB6F894DEBF0FBECDBF0E946B8C48EAFC
:1072800051E660E070E0C1010E94C58B6C197D0978
:107290008E099F0925E030E040E050E00E94ABD627
:1072A00029013A015F922F931F9285E08F93E0911D
:1072B000DC0BF091DD0BE859FE4F81818F938081CB
:1072C0008F931F930F930E949E4661E0C1010E941D
:1072D0006EB09F938F937F936F93E091DC0BF0914F
:1072E000DD0BEA5AFE4F81818F9380818F931F932C
:1072F0000F930E949E468091610A9091620AA0912C
:10730000630AB091640A8093740A9093750AA093FB
:10731000760AB093770A8091650A9091660AA091E7
:10732000670AB091680A8093780A9093790AA093CB
:107330007A0AB0937B0A8091690A90916A0AA091B7
:107340006B0AB0916C0A80937C0A90937D0AA0939B
:107350007E0AB0937F0A20E030E040E751E460917C
:107360006D0A70916E0A80916F0A9091700A0E9466
:10737000E7D66093800A7093810A8093820A909383
:10738000830A0E946B8C48EA51E660E070E0C1011C
:107390000E94C58B6C197D098E099F092FE030E092
:1073A00040E050E00E94ABD63F932F931F928FE0B6
:1073B0008F93E091DC0BF091DD0BE859FE4F81815A
:1073C0008F9380818F931F930F9365962FAF65974F
:1073D00066963FAF669763964FAF639764965FAFCD
:1073E00064970E949E46840C951C65962FAD659708
:1073F00066963FAD6697C401820F931F63E070E00D
:107400000E9471DA80E090E00E9470D30FB6F89489
:10741000DEBF0FBECDBF37FC12C02DEB37E346E019
:107420005EE30E9485CEF101EE0FFF1FEE0FFF1FFE
:10743000EC55FD4E608371838283938303C060E0CB
:1074400070E0CB010E9441D87F936F938AED9BE05F
:10745000E091DC0BF091DD0BE659FE4F21812F937B
:1074600020812F939F938F930E949E463F85309358
:10747000210A0F900F900F900F900F900F901DC347
:107480008FEF90E00E9411AD0E9428AD83EB9AE04F
:107490000E94D049029720F10E947CAA1092B70A5C
:1074A0001092B80A1092B90A1092BA0A1092BB0A46
:1074B0001092BC0A1092BD0A1092BE0A1092B60A2F
:1074C0001092B50A1093B40A0093B30A0E94E1C265
:1074D0006093B70A7093B80A8093B90A9093BA0A76
:1074E0000E94765C0C943A2C81E00C94BE2E6FEFD7
:1074F00070E0C1010E94D5B50C946A2F0E94F0ACD7
:107500001092480B37FE0DC03091A80A3983409184
:10751000A90A4B835091AA0A5C838091AB0A8D83A0
:1075200011C0AC8DBD8DBC91B983EC8DFD8DF18109
:10753000FB83AC8DBD8D1296BC91BC83EC8DFD8D13
:10754000F381FD8329813B814C815D81BF89A88DB9
:10755000FA8DEB8D6B2F7A2F8F2F9E2F0E942DD9B6
:10756000181644F029812F8B3B81388F4C814A8F2C
:107570005D815B8F29813B814C815D81D201F9A9BD
:10758000EAA96B2F742D8F2F9E2F0E946CD387FD3D
:1075900006C059804B808C8189AB9D819AABA885B0
:1075A000AA2309F4F7C02C853D894E895E8569813F
:1075B0007B818C819D810E942DD9181614F00C942A
:1075C000AE2F0E94E1C2DC01CB018C199D09AE09EE
:1075D000BF0989389341A105B10510F40C94AE2F71
:1075E000C3012E813F81821B930B37FE03C00E9493
:1075F000ADB504C0BC01C1010E94D5B50E94E1C275
:10760000698B7A8B8B8B9C8BDC01CB018C199D0950
:10761000AE09BF098EA39FA3A8A7B9A79EA59F8B5C
:10762000AFA5A88FB8A9BA8FEE85EB8FB3C00E9423
:10763000E1C2DC01CB012AA53BA54CA55DA5821BBF
:10764000930BA40BB50B813D9740A105B10540F00C
:107650000E947CAA0E94E1C26AA77BA78CA79DA773
:107660000E94E1C24B015C010E94E1C209891A89B2
:107670002B893C890C0D1D1D2E1D3F1D801A910A62
:10768000A20AB30A860E971EA81EB91E41E08416F0
:107690004FE9940644E2A406B10410F40C94D02FF0
:1076A000E091DC0BF091DD0BE65AFE4F49C0F10191
:1076B000EE0FFF1FEE0FFF1FE457FD4E9201802FCC
:1076C000912FA32FB22F80839183A283B383C10113
:1076D000880F991F880F991F8C010C561D4E2DEB9A
:1076E00037E346E05EE3662D772D882D992D0E94C5
:1076F00085CED8016D937D938D939C9313970C94B5
:107700008430C101880F991F880F991F8C0104567E
:107710001D4E2DEB37E346E05EE36A2D7B2D8C2D6D
:107720009D2D0E94D0D7F80160837183828393835B
:107730000C949C30E091DC0BF091DD0BE45AFE4F91
:10774000608171818AED9BE00E9461460C94AC30AF
:107750000E94765C0C94A92F19821B821C821D82C8
:107760000C945E2FA70196010C94FC2D59815E8329
:107770008B818F879C81998BAD81AF8B08C0B9813C
:10778000BE83EB81EF87FC81F98B2D812F8B81E00C
:107790000C947A2E2C853D894E895E8569817B818A
:1077A0008C819D810E946CD387FF84C10E94E1C2BD
:1077B000DC01CB0129893A894B895C89821B930BB7
:1077C000A40BB50B89389341A105B10508F472C12A
:1077D0000E94E1C26B017C014F8558891416150681
:1077E0000CF04BC1DC01CB0129893A894B895C89BA
:1077F000821B930BA40BB50B2EA13FA148A559A545
:10780000280F391F4A1F5B1F288739874A875B87E4
:107810002EA13FA148A559A5281B390B4A0B5B0B8C
:10782000AE81BF810E94BCDA288539854A855B8597
:107830000E9498DA260D371D243131059CF039015C
:1078400036EA631671041CF0E5EA6E2E712C40E8EE
:10785000641671047CF08EEF90E0861997099F837F
:107860008E830AC074E1672E712CA4E1B0E0BF835F
:10787000AE8302C07F826E82BB8DBF93EA8DEF9391
:10788000F88DFF932F892F933AA93F9349A94F93DE
:107890004F925F925F815F938E818F937F926F9201
:1078A000AEECB4E0BF93AF93AAEDBBE0BF93AF9350
:1078B0000E949E460FB6F894DEBF0FBECDBF4F8527
:1078C0005889433051050CF4D8C0AE81BF81BD0149
:1078D000BB0F880B990B0E9472D320E030E040E888
:1078E00050E40E9485CE4B015C01B20199A98AA99E
:1078F000272F342D492F582FBF89A88DFA8DEB8D56
:107900006B2F7A2F8F2F9E2F0E94E6D620ED3FE01F
:1079100049E450E40E9485CE9B01AC01C501B4014D
:107920000E94D0D74B015C01762F272F392D4A2D8D
:107930005B2D6E8D7F8D88A199A10E94E7D66E8FF9
:107940007F8F88A399A3688579858A859B850E9406
:1079500072D320E030E04AE754E40E94D0D78B0194
:107960008AAB9BAB762F982F8BA9272F312F492FCE
:10797000582F6AA17BA18CA19DA10E94E7D66AA382
:107980007BA38CA39DA3BBA9BF93EAA9EF931F93ED
:107990000F93BF92AF929F928F92AEEBB4E0BF93E2
:1079A000AF93AAEDBBE0BF93AF930E949E4620E049
:1079B00030E040E05FE3682D792D8A2D9B2D0E94F9
:1079C00085CEB62EA72E982E892E9AA98BA9202F68
:1079D000312F492F582FD501F4016B2F7A2F8F2F7C
:1079E0009E2F0E94D0D7688779AB582E492E2DEC58
:1079F0003CEC4CEC5EE3D501F4016B2F7A2F8F2F1A
:107A00009E2F0E9485CEFAA9EBA9202F312F4F2F50
:107A10005E2F0E9485CE9B01182F092F6FEA74E01C
:107A20008AED9BE065962FAF659766963FAF6697A8
:107A30000E9461460F931F9366963FAD66973F93F2
:107A400065962FAD65972F934F925F92F9A9FF939B
:107A500028852F938F929F92AF92BF92A6E9B4E0B0
:107A6000BF93AF93AAEDBBE0BF93AF930E949E4636
:107A70000FB6F894DEBF0FBECDBF8E819F81860DFD
:107A8000971D37FE03C00E94ADB504C0BC01C10103
:107A90000E94D5B54F8558894F5F5F4F588B4F87F0
:107AA0005EA44FA458A959AB8E858AAB91E0988704
:107AB0000C94AE2F18860C94AE2FC95ADF4F0FB618
:107AC000F894DEBF0FBECDBFDF91CF911F910F9114
:107AD000FF90EF90DF90CF90BF90AF909F908F90EE
:107AE0007F906F905F904F903F902F900895CF922E
:107AF000DF92EF92FF92CF93DF93EC016A017B015B
:107B0000FE018491882321F00E9470BD2196F8CF58
:107B100042E0C701B601DF91CF91FF90EF90DF9077
:107B2000CF900C94CAA90F931F93CF93DF93EC01CE
:107B30008B01FE018491882321F00E9470BD219663
:107B4000F8CFB801110F880B990BDF91CF911F91DE
:107B50000F910C94DBB4AF92BF92CF92DF92EF9271
:107B6000FF920F931F93CF93DF9310924909809157
:107B7000400990914109A0914209B0914309813097
:107B80009048A105B10540F01092400910924109BA
:107B9000109242091092430980914009809348094C
:107BA00090914709891710F480934709D0914709AC
:107BB00010914B0912FB112710F9C0E084E0C82E88
:107BC000D12CE12CF12C94E0B92E22E0A22E909140
:107BD0004809D1112CC081E0911180E080934609C1
:107BE00090912B02992359F0E091DC0BF091DD0B81
:107BF0004489558903E023E06C2F0E94DA69112340
:107C000009F4B0C080914609882309F4ABC00E94F2
:107C1000545D8CE497EADF91CF911F910F91FF9013
:107C2000EF90DF90CF90BF90AF900C943F5DD1303C
:107C300011F581E0913009F080E080934609909140
:107C40002B02992359F0E091DC0BF091DD0B42AD52
:107C500053AD0EE72EE36C2F0E94DA69112309F46D
:107C600081C080914609882309F47CC00E94545D3C
:107C700086E494E46BC0D23021F581E0923009F0C3
:107C800080E08093460990912B02992369F0E0915E
:107C9000DC0BF091DD0BEE5BFF4F408151810EE775
:107CA0002EE36C2F0E94DA69112309F45BC08091E6
:107CB0004609882309F456C00E94545D85E593E483
:107CC00045C0D33001F581E0933009F080E0809326
:107CD000460990912B02992359F0E091DC0BF09129
:107CE000DD0B46AD57AD0EE72EE36C2F0E94DA692F
:107CF0001123C1F1809146098823A1F10E94545DAE
:107D000084E692E423C0D43069F581E0943009F030
:107D100080E08093460990912B02992369F0E091CD
:107D2000DC0BF091DD0BEA5BFF4F408151810EE7E8
:107D30002EE36C2F0E94DA691123A1F0809146098D
:107D4000882381F00E94545D83E791E4DF91CF9115
:107D50001F910F91FF90EF90DF90CF90BF90AF9069
:107D60000C942D5D80914809853050F0C0924009F7
:107D7000D0924109E0924209F0924309B092480939
:107D8000209148098091470990E00396422F50E0E6
:107D9000841795074CF48DEF820F80934709A092CA
:107DA0002B02DCEFD20FCFEFCF5FDF5FC43008F4E0
:107DB0000ECFDF91CF911F910F91FF90EF90DF9049
:107DC000CF90BF90AF900895BF92CF92DF92EF9285
:107DD000FF920F931F93CF93DF93109249098091E5
:107DE000400990914109A0914209B0914309813025
:107DF0009048A105B10540F0109240091092410948
:107E000010924209109243098091400980934809D9
:107E100090914709891710F480934709D091470939
:107E200010914B0912FB112710F9C0E083E0C82E16
:107E3000D12CE12CF12C92E0B92E90914809D1116E
:107E40002BC081E0911180E08093460990912B0234
:107E5000992359F0E091DC0BF091DD0B44895589B1
:107E600003E023E06C2F0E94DA69112309F48CC02F
:107E700080914609882309F487C00E94545D8CE4F0
:107E800097EADF91CF911F910F91FF90EF90DF90D4
:107E9000CF90BF900C943F5DD13021F581E09130BF
:107EA00009F080E08093460990912B02992369F0B4
:107EB000E091DC0BF091DD0BEA58FF4F40815181DE
:107EC0000EE72EE36C2F0E94DA69112309F45CC0DF
:107ED00080914609882309F457C00E94545D82E3CB
:107EE00091E447C0D23011F581E0923009F080E092
:107EF0008093460990912B02992369F0E091DC0B65
:107F0000F091DD0BEC58FF4F408151810EE72EE3DD
:107F10006C2F0E94DA691123B9F1809146098823F8
:107F200099F10E94545D8FE391E423C0D33061F551
:107F300081E0933009F080E08093460990912B0214
:107F4000992369F0E091DC0BF091DD0BEE58FF4FC7
:107F5000408151810EE72EE36C2F0E94DA691123D4
:107F600099F080914609882379F00E94545D8CE451
:107F700091E4DF91CF911F910F91FF90EF90DF90EF
:107F8000CF90BF900C942D5D80914809843058F0BB
:107F9000C0924009D0924109E0924209F09243090F
:107FA00083E080934809209148098091470990E037
:107FB0000396422F50E0841795074CF48DEF820F03
:107FC00080934709B0922B02DCEFD20FCFEFCF5F47
:107FD000DF5FC43008F431CFDF91CF911F910F9153
:107FE000FF90EF90DF90CF90BF900895FF920F9396
:107FF0001F93CF93DF93109249098091400990918C
:108000004109A0914209B091430981309048A105EE
:10801000B10540F0109240091092410910924209B6
:108020001092430980914009809348099091470933
:10803000891710F480934709D091470910914B0993
:1080400012FB112710F9C0E082E0F82E9091480948
:10805000D11127C081E0911180E080934609909171
:108060002B02992359F0E091DC0BF091DD0B44A138
:1080700055A103E023E06C2F0E94DA69112309F473
:1080800058C080914609882309F453C00E94545D6A
:1080900084EE9EE3DF91CF911F910F91FF900C949E
:1080A0003F5DD13011F581E0913009F080E080939F
:1080B000460990912B02992369F0E091DC0BF09135
:1080C000DD0BE858FF4F408151810EE72EE36C2F06
:1080D0000E94DA69112369F180914609882349F1E8
:1080E0000E94545D81EB92EA7FC0D23011F581E0AD
:1080F000923009F080E08093460990912B029923F9
:1081000069F0E091DC0BF091DD0BE658FF4F408108
:1081100051810EE72EE36C2F0E94DA69112349F09A
:1081200080914609882329F00E94545D86EF91EAE8
:108130005BC020E030E040E251E4609117097091AB
:1081400018098091190990911A090E946CD387FF30
:1081500052C090914809D33021F581E0933009F065
:1081600080E08093460990912B02992369F0E09179
:10817000DC0BF091DD0BE458FF4F408151810EE79D
:108180002EE36C2F0E94DA69111102C085E034C021
:10819000809146098823D1F30E94545D89E995E4D2
:1081A00023C0D43099F781E0943009F080E08093C7
:1081B000460990912B02992369F0E091DC0BF09134
:1081C000DD0BE258FF4F408151810EE72EE36C2F0B
:1081D0000E94DA691123D1F2809146098823B1F215
:1081E0000E94545D8DE195E4DF91CF911F910F9135
:1081F000FF900C942D5D83E090914809981798F0BA
:10820000482F50E041505109052E000C660B770BAA
:108210004093400950934109609342097093430988
:10822000815080934809209148098091470990E046
:108230000396422F50E0841795074CF48DEF820F80
:1082400080934709F0922B02DCEFD20FCFEFCF5F84
:10825000DF5FC43008F4FACEDF91CF911F910F9108
:10826000FF90089580E090E0A0E2B1E480931709C8
:1082700090931809A0931909B0931A09B7CE80E01A
:1082800090E0A0E8BFE38093170990931809A093AA
:108290001909B0931A09AACE8DEC9CECACECBDE3A5
:1082A0008093170990931809A0931909B0931A099C
:1082B0009DCE8091DC129091DD129093A70A80935D
:1082C000A60A81E090E09093190C8093180C80919D
:1082D000E0129091E1120E9411AD84E090E00E94C2
:1082E0003A910C94CB69AF92BF92CF92DF92EF920A
:1082F000FF920F931F93CF93DF93109249098091C0
:10830000400990914109A0914209B09143098130FF
:108310009048A105B10540F0109240091092410922
:1083200010924209109243098091400980934809B4
:1083300090914709891710F480934709D091470914
:1083400010914B0912FB112710F9C0E083E0C82EF1
:10835000D12CE12CF12C93E0B92E22E0A22E9091A9
:108360004809D1112BC081E0911180E0809346092A
:1083700090912B02992369F0E091DC0BF091DD0BD9
:10838000EA5AFF4F4081518100E22EE36C2F0E9498
:10839000DA69112309F44CC080914609882309F455
:1083A00047C00E94545DDF91CF911F910F91FF90C4
:1083B000EF90DF90CF90BF90AF907BCFD13089F41A
:1083C00081E0913009F080E08093460990912B0282
:1083D0009923F9F2E091DC0BF091DD0BE85AFF4FA5
:1083E000D1CFD23089F481E0923009F080E08093DF
:1083F000460990912B02992361F2E091DC0BF091F8
:10840000DD0BE65AFF4FBECFD33091F481E09330BD
:1084100009F080E08093460990912B02992309F49A
:10842000B8CFE091DC0BF091DD0BE45AFF4FAACFFF
:1084300080914809843050F0C0924009D09241099F
:10844000E0924209F0924309B0924809209148090C
:108450008091470990E00396422F50E084179507DA
:108460004CF48DEF820F80934709A0922B02DCEF32
:10847000D20FCFEFCF5FDF5FC43008F470CFDF9152
:10848000CF911F910F91FF90EF90DF90CF90BF9011
:10849000AF9008958091E2129091E3129093A70A11
:1084A0008093A60A81E090E09093190C8093180CB9
:1084B0008091E6129091E7120E9411AD86E090E063
:1084C0000E943A910C94CB69AF92BF92CF92DF9207
:1084D000EF92FF920F931F93CF93DF93109249096E
:1084E0008091400990914109A0914209B0914309BE
:1084F00081309048A105B10540F0109240091092DA
:1085000041091092420910924309809140098093D9
:10851000480990914709891710F480934709D09131
:10852000470910914B0912FB112710F9C0E083E0B5
:10853000C82ED12CE12CF12C93E0B92E22E0A22EF2
:1085400090914809D1112BC081E0911180E0809376
:10855000460990912B02992369F0E091DC0BF09190
:10856000DD0BEA5AFF4F4081518100E22EE36C2F70
:108570000E94DA69112309F44CC0809146098823CE
:1085800009F447C00E94545DDF91CF911F910F9174
:10859000FF90EF90DF90CF90BF90AF907BCFD13026
:1085A00089F481E0913009F080E080934609909150
:1085B0002B029923F9F2E091DC0BF091DD0BE85AE4
:1085C000FF4FD1CFD23089F481E0923009F080E0C2
:1085D0008093460990912B02992361F2E091DC0B84
:1085E000F091DD0BE65AFF4FBECFD33091F481E01E
:1085F000933009F080E08093460990912B029923F3
:1086000009F4B8CFE091DC0BF091DD0BE45AFF4F99
:10861000AACF80914809843050F0C0924009D0928E
:108620004109E0924209F0924309B0924809209131
:1086300048098091470990E00396422F50E0841743
:1086400095074CF48DEF820F80934709A0922B027F
:10865000DCEFD20FCFEFCF5FDF5FC43008F470CF15
:10866000DF91CF911F910F91FF90EF90DF90CF900E
:10867000BF90AF9008958091DC129091DD1290939D
:10868000A50A8093A40A81E090E09093190C80934E
:10869000180C8091E0129091E1120E9411AD83E0DC
:1086A00090E00E943A910C94CB69AF92BF92CF9226
:1086B000DF92EF92FF920F931F93CF93DF9310926D
:1086C00049098091400990914109A0914209B091D6
:1086D000430981309048A105B10540F0109240094E
:1086E0001092410910924209109243098091400969
:1086F0008093480990914709891710F4809347099E
:10870000D091470910914B0912FB112710F9C0E0D5
:1087100083E0C82ED12CE12CF12C93E0B92E22E07D
:10872000A22E90914809D1112BC081E0911180E0D7
:108730008093460990912B02992369F0E091DC0B1C
:10874000F091DD0BEA5AFF4F4081518100E22EE3A8
:108750006C2F0E94DA69112309F44CC080914609FC
:10876000882309F447C00E94545DDF91CF911F9187
:108770000F91FF90EF90DF90CF90BF90AF907BCFA5
:10878000D13089F481E0913009F080E0809346098E
:1087900090912B029923F9F2E091DC0BF091DD0B23
:1087A000E85AFF4FD1CFD23089F481E0923009F0FE
:1087B00080E08093460990912B02992361F2E09129
:1087C000DC0BF091DD0BE65AFF4FBECFD33091F4B6
:1087D00081E0933009F080E08093460990912B026C
:1087E000992309F4B8CFE091DC0BF091DD0BE45A4A
:1087F000FF4FAACF80914809843050F0C0924009C1
:10880000D0924109E0924209F0924309B09248099E
:10881000209148098091470990E00396422F50E04B
:10882000841795074CF48DEF820F80934709A0922F
:108830002B02DCEFD20FCFEFCF5FDF5FC43008F445
:1088400070CFDF91CF911F910F91FF90EF90DF904C
:10885000CF90BF90AF9008958091E2129091E31273
:108860009093A50A8093A40A81E090E09093190C5C
:108870008093180C8091E6129091E7120E9411AD3E
:1088800085E090E00E943A910C94CB69AF92BF9240
:10889000CF92DF92EF92FF920F931F93CF93DF93CC
:1088A000109249098091400990914109A091420993
:1088B000B091430981309048A105B10540F0109274
:1088C0004009109241091092420910924309809187
:1088D00040098093480990914709891710F48093C3
:1088E0004709D091470910914B0912FB112710F944
:1088F000C0E083E0C82ED12CE12CF12C93E0B92EFE
:1089000022E0A22E90914809D1112BC081E0911153
:1089100080E08093460990912B02992369F0E091C1
:10892000DC0BF091DD0BEA5AFF4F4081518100E2F0
:108930002EE36C2F0E94DA69112309F44CC0809158
:108940004609882309F447C00E94545DDF91CF9106
:108950001F910F91FF90EF90DF90CF90BF90AF905D
:108960007BCFD13089F481E0913009F080E08093B1
:10897000460990912B029923F9F2E091DC0BF091DA
:10898000DD0BE85AFF4FD1CFD23089F481E092302D
:1089900009F080E08093460990912B02992361F2BF
:1089A000E091DC0BF091DD0BE65AFF4FBECFD330E8
:1089B00091F481E0933009F080E080934609909132
:1089C0002B02992309F4B8CFE091DC0BF091DD0B79
:1089D000E45AFF4FAACF80914809843050F0C092EA
:1089E0004009D0924109E0924209F0924309B092C5
:1089F0004809209148098091470990E00396422F49
:108A000050E0841795074CF48DEF820F809347094F
:108A1000A0922B02DCEFD20FCFEFCF5FDF5FC4302D
:108A200008F470CFDF91CF911F910F91FF90EF90DD
:108A3000DF90CF90BF90AF900895CF92DF92EF92EA
:108A4000FF920F931F938091400990914109A0914B
:108A50004209B09143090097A105B10509F441C04D
:108A6000BC01990F880B990B0E9472D320911709B2
:108A7000309118094091190950911A090E9485CE28
:108A80009B01AC0160916D0A70916E0A80916F0A32
:108A90009091700A0E94E7D660936D0A70936E0AF7
:108AA00080936F0A9093700A1092400910924109C6
:108AB000109242091092430981E2C82E8AE0D82E12
:108AC000E12CF12C00E81FE32DE63AE049E65AE0FC
:108AD00065E67AE081E69AE00E94D07181E08093B9
:108AE0002B0280912B02882349F08DE69AE00E94A8
:108AF000BE5BBC0184E496E00E94C86E80914B0985
:108B000082FF10C00E94545D86EF9FE390930202A3
:108B1000809301021092400910924109109242097B
:108B2000109243091F910F91FF90EF90DF90CF902B
:108B30000895CF92DF92EF92FF920F931F9380914F
:108B4000400990914109A0914209B0914309892BB4
:108B50008A2B8B2B09F47BC00E94E1C26093DE0B51
:108B60007093DF0B8093E00B9093E10B60914009D1
:108B700070914109072E000C880B990B0E9472D34B
:108B800020911709309118094091190950911A093B
:108B90000E9485CE2091690A30916A0A40916B0A41
:108BA00050916C0A0E94E7D66B017C0120E030E016
:108BB000A9010E946CD387FD09C0C092690AD092B6
:108BC0006A0AE0926B0AF0926C0A08C01092690A75
:108BD00010926A0A10926B0A10926C0A20E030E040
:108BE0004EE353E46091690A70916A0A80916B0ABE
:108BF00090916C0A0E942DD9181664F480E090E0E0
:108C0000AEE3B3E48093690A90936A0AA0936B0A77
:108C1000B0936C0A109240091092410910924209D7
:108C20001092430981E2C82E8AE0D82EE12CF12C63
:108C300000E810E42DE63AE049E65AE065E67AE01D
:108C400081E69AE00E94D07181E080932B028091AE
:108C50002B02882349F089E69AE00E94BE5BBC01A2
:108C600082E496E00E94C86E80914B0982FF10C09A
:108C70000E94545D86EF9FE390930202809301026D
:108C80001092400910924109109242091092430932
:108C90001F910F91FF90EF90DF90CF9008959091EA
:108CA000C00095FFFCCF8093C6000895CF93DF935B
:108CB000EB018991882311F0F2DFFBCFDF91CF9197
:108CC0000895CF93DF93EB01FE018491882319F07F
:108CD000E6DF2196F9CFDF91CF9108950F931F938F
:108CE000CF93DF93EC018B01E881F9810480F5815A
:108CF000E02D6DE476E01995E881F9810480F58135
:108D0000E02DB801CE01DF91CF911F910F91199401
:108D1000CF93DF93CDB7DEB7DF91CF91089508955C
:108D20000C94CECF0C94CECF0C94CECF0C94CECF4F
:108D30000C94CECF0C94CECF0C94CECF2F923F92EA
:108D40004F925F926F927F928F929F92AF92BF925B
:108D5000CF92DF92EF92FF920F931F93CF93DF9307
:108D600000D01F921F92CDB7DEB7EB8CFC8CCD8C60
:108D7000DE8CDE015F96F60184911B8200E010E03C
:108D8000970126573F4F3A832983882309F42FC13F
:108D9000853209F01EC1E981FA81808382E0A82E24
:108DA000B12C21E030E0FFEFCF1ADF0AF601649129
:108DB000653239F4F701E00FF11FE05CFF4F60838B
:108DC0000EC1462F062E000C550B40535109C90108
:108DD0004A30510550F401962E0D3F1DF901E6571A
:108DE000FF4F6083FB81F1115A016E3259F4F70194
:108DF000E80FF91FE657FF4F6083019621E02B83B0
:108E00009C01D1CF693611F0693449F58E0D9F1D53
:108E1000FC01E657FF4F6083319610825D0132E01E
:108E2000A30EB11C11968C9111978F938C918F93F7
:108E30008A818F9399819F93C801805C9F4F8E0D8B
:108E40009F1D9F938F930E94E5DB080F191F0F90C2
:108E50000F900F900F900F900F90D501C2C06F7DB3
:108E6000663409F0A2C0FD013496FD83EC834D9079
:108E70005D906D907C9020E030E0A901C301B201CB
:108E80000E946CD387FF0DC0F701E00FF11FE05C7B
:108E9000FF4F2DE2208377FA709477F870940F5F7C
:108EA0001F4F912C60E070E080E09FE3292D30E0BF
:108EB0002A153B0544F420E030E040E251E40E94F2
:108EC000D0D79394F3CF9B01AC01C301B2010E94B0
:108ED000E7D62B013C010E9447D8262E972E882EDC
:108EE000392E0E9470D39B01AC01C301B2010E94D4
:108EF000E6D62B013C013F928F929F922F92A4E5E0
:108F0000B6E0BF93AF93C801805C9F4F8E0D9F1D4D
:108F10009F938F930E943DD3080F191F0FB6F894AB
:108F2000DEBF0FBECDBF1A141B044CF4F701E00FD7
:108F3000F11FE05CFF4F3EE230830F5F1F4F4501A2
:108F4000180180E4280E311C2E0C3F1C1814190443
:108F50001CF520E030E040E251E4C301B2010E9480
:108F600085CE2B013C010E9441D820E3260FD10180
:108F70002D931D01072E000C880B990B0E9472D3B4
:108F80009B01AC01C301B2010E94E6D62B013C015A
:108F9000B1E08B1A9108DACFB7FE02C0A12CB12C38
:108FA0000A0D1B1DAC81BD811CC0633509F028CFA3
:108FB000FD01408151811296FA018191AF01882310
:108FC00081F00F5F1F4F9701200F311FF90187AF0D
:108FD000F3CFF701E00FF11FE05CFF4F80830F5FDD
:108FE0001F4FFFEFCF1ADF0AF6018491CECE0E0D90
:108FF0001F1DF801E05CFF4F1082F0E4EF0EF11C42
:10900000D7018D917D01882311F049DEF9CF0F90B2
:109010000F900F900F900F90DF91CF911F910F91B4
:10902000FF90EF90DF90CF90BF90AF909F908F9088
:109030007F906F905F904F903F902F90089587FFA3
:1090400020C090912B09803C50F0911108C0825CA7
:1090500080932A0981E080932B0980E00895992369
:1090600071F0E0912A0990E4E99FF0011124B09792
:109070008F73E80FF11DE95AF94F649103C06FE354
:1090800001C0682F89EF96E10E943F9A10922B0948
:1090900081E0089508951F920F920FB60F92112448
:1090A0000BB60F922F933F934F935F936F937F93E2
:1090B0008F939F93AF93BF93EF93FF938091C70AD2
:1090C0009091C80A8130910599F1F4F48F3F2FEF08
:1090D000920719F1892B09F0E1C088E080937B00A9
:1090E00085E480937C00E091350BF091360B809104
:1090F000780090917900EE0FFF1FEB5EF44F9183A3
:10910000808381E090E01CC08330910509F467C042
:10911000E4F0049709F46CC0C1C088E080937B0040
:1091200086E480937C001092C80A1092C70ACFC0D0
:1091300088E080937B0085E480937C0082E090E06F
:109140009093C80A8093C70AC7C088E080937B00C9
:1091500087E480937C00E091350BF091360B809191
:10916000780090917900EE0FFF1FE656F54F94AF0F
:1091700083AF809178009091790074E0880F991FF7
:109180007A95E1F72091370B3091380B2817390782
:1091900060F460E070E080E090E00E94D5B583E08C
:1091A00090E09093440B8093430B809178009091D2
:1091B000790054E0880F991F5A95E1F720913B0BF5
:1091C00030913C0B8217930708F05EC060E070E0BE
:1091D00080E090E00E94D5B584E090E051C088E046
:1091E00080937B0087E480937C0084E090E051C012
:1091F00088E080937B0086E480937C00E091350BCF
:10920000F091360B8091780090917900EE0FFF1F5E
:10921000EB50F54F91838083809178009091790095
:1092200044E0880F991F4A95E1F72091370B309160
:10923000380B2817390760F460E070E081E090E0B7
:109240000E94D5B585E090E09093440B8093430B4A
:10925000809178009091790024E0880F991F2A95D9
:10926000E1F720913B0B30913C0B8217930760F4A0
:1092700060E070E081E090E00E94D5B586E090E08B
:109280009093440B8093430B8091C70A9091C80A36
:1092900001969093C80A8093C70A19C088E080930A
:1092A0007B0086E480937C001092C80A1092C70A63
:1092B0008091350B9091360B01969093360B8093ED
:1092C000350B8F7099279093360B8093350B8091D7
:1092D0007A00806480937A0080917A008064809321
:1092E0007A00FF91EF91BF91AF919F918F917F9104
:1092F0006F915F914F913F912F910F900BBE0F9007
:109300000FBE0F901F9018951F920F920FB60F92DD
:1093100011240BB60F922F933F934F935F936F934C
:109320007F938F939F93AF93BF93EF93FF930E948D
:109330000A5C8091470B8F5F8093470B87FF05C0C6
:1093400081E08093480B1092470B8091BF0A909167
:10935000C00A0196813D23E092072CF49093C00A45
:109360008093BF0A0AC01092C00A1092BF0A90915F
:10937000170C81E089278093170CFF91EF91BF9123
:10938000AF919F918F917F916F915F914F913F919D
:109390002F910F900BBE0F900FBE0F901F9018953E
:1093A0000F931F93CF93DF93EC01888199810197ED
:1093B00019F40E94E1C204C0688579858A859B857D
:1093C0000C811D812E813F81601B710B820B930BE1
:1093D00028EE33E040E050E00E94ABD68A819B81CA
:1093E000820F931FDF91CF911F910F910895CF931B
:1093F000DF93FC012081318121303105E1F0EC0166
:109400002230310521F4CCDF9B838A830AC0148289
:109410001582168217821086118612861386138291
:10942000128281E090E0998388830E94E1C26C837C
:109430007D838E839F83DF91CF91089508951F923E
:109440000F920FB60F9211240BB60F922F933F93EA
:109450004F935F936F937F938F939F93AF93BF933C
:10946000EF93FF93E0917C0CF0917D0C81A1813012
:1094700011F4459A01C0149A8091710C9091720C6C
:1094800001979093720C8093710C81A1813011F43B
:10949000459801C014981092250110922401FF9163
:1094A000EF91BF91AF919F918F917F916F915F915C
:1094B0004F913F912F910F900BBE0F900FBE0F90C9
:1094C0001F9018951F920F920FB60F9211240BB692
:1094D0000F920F931F932F933F934F935F936F932D
:1094E0007F938F939F93AF93BF93CF93DF93EF932C
:1094F000FF93809171008D7F809371007894E0914B
:109500007C0CF0917D0C309709F0DFC08091371210
:1095100090913612981759F097E5899FF001112420
:10952000DF01A45EB24F81E08C93EA53F34FF093D6
:109530007D0CE0937C0C309709F4C7C080A1809328
:10954000730CDF01AA5ABF4F11E01C931092780CE4
:109550001092790C10927A0C10927B0CEE5BFF4FFC
:10956000808191810E947C5490939A0C8093990CF5
:109570008091980C082E000C990B90939C0C809372
:109580009B0CE0917C0CF0917D0CEA5BFF4F80819D
:1095900091819093930C8093920C0E947C54AC0127
:1095A00060E070E04093740C5093750C6093760CFF
:1095B0007093770C9093990080939800E0917C0CC5
:1095C000F0917D0C80899189A289B389B695A79580
:1095D00097958795B095A095909581959F4FAF4FA2
:1095E000BF4F80937E0C90937F0CA093800CB09320
:1095F000810C8093820C9093830CA093840CB09385
:10960000850C8093860C9093870CA093880CB09364
:10961000890C80938A0C90938B0CA0938C0CB09344
:109620008D0C1092940C1092950C1092960C109236
:10963000970C8091730C80FF05C0899A9FEF9093DF
:109640008E0C03C0899810938E0C81FF03C08F98F5
:109650009FEF02C08F9A91E090938F0C9FB782FF8B
:109660000BC0F89480910B01826080930B019FBF27
:109670008FEF8093900C10C0F89480910B018D7F38
:1096800080930B019FBF81E08093900C80E090E479
:109690009093A9008093A8008091730CE0917C0CBA
:1096A000F0917D0C83FF08C081A1813011F4439AB1
:1096B00001C016988FEF07C081A1813011F4439843
:1096C00001C0169A81E08093910CE0917C0CF0919E
:1096D0007D0C309739F480ED97E09093990080935A
:1096E0009800CDC39091730C90FD38C08091700CA0
:1096F0008823A1F18CB121E085FB882780F982279E
:1097000059F130912909332339F140815181628126
:1097100073811416150616061706F4F44091100A04
:109720005091110A6091120A7091130A40931D0919
:1097300050931E0960931F097093200920939D0C7C
:1097400040895189628973894093940C5093950C98
:109750006093960C7093970C8093290991FD38C003
:109760008091700C8823A1F18091030121E08695FE
:109770008170822759F130911C09332339F14481DA
:109780005581668177811416150616061706F4F4BE
:109790004091140A5091150A6091160A7091170AA7
:1097A000409321095093220960932309709324095F
:1097B00020939E0C40895189628973894093940C4F
:1097C0005093950C6093960C7093970C80931C09A2
:1097D00092FF38C08091700C8823A1F189B191E08B
:1097E00083FB882780F9892759F120911B092223BF
:1097F00039F1408551856285738514161506160664
:109800001706F4F44091180A5091190A60911A0A47
:1098100070911B0A409325095093260960932709EC
:109820007093280990939F0C4089518962897389AC
:109830004093940C5093950C6093960C7093970CF6
:1098400080931B0982A193A1A4A1B5A118161906A2
:109850001A061B06ACF58091910C813009F00FC3FC
:1098600082A193A1A4A1B5A19093720C8093710CD5
:10987000A1A1B0E0AA0FBB1FA852BD4E8D919C9133
:10988000880F991F90932901809328011092250138
:109890001092240180917300826080937300809104
:1098A000710C9091720C18161906CCF3809173000C
:1098B0008D7F8093730012A213A214A215A2DFC29F
:1098C00020E08091980C28170CF07AC1E0917C0C74
:1098D000F0917D0C40917E0C50917F0C6091800C3A
:1098E0007091810C80819181A281B381840F951F39
:1098F000A61FB71F80937E0C90937F0CA093800CC3
:10990000B093810C181619061A061B066CF5889A76
:109910004089518962897389841B950BA60BB70B0B
:1099200080937E0C90937F0CA093800CB093810C5D
:109930004091100A5091110A6091120A7091130A15
:1099400080918E0C082E000C990BAA0BBB0B840F78
:10995000951FA61FB71F8093100A9093110AA0931A
:10996000120AB093130A88984091820C5091830C8C
:109970006091840C7091850C84819581A681B7815A
:10998000840F951FA61FB71F8093820C9093830CA2
:10999000A093840CB093850C181619061A061B06A2
:1099A0006CF58E9A4089518962897389841B950B65
:1099B000A60BB70B8093820C9093830CA093840C1E
:1099C000B093850C4091140A5091150A6091160AC3
:1099D0007091170A80918F0C082E000C990BAA0B1E
:1099E000BB0B840F951FA61FB71F8093140A90937B
:1099F000150AA093160AB093170A8E984091860C08
:109A00005091870C6091880C7091890C80859185AC
:109A1000A285B385840F951FA61FB71F8093860C60
:109A20009093870CA093880CB093890C1816190694
:109A30001A061B060CF047C09FB7F89480910B01E3
:109A4000886080930B019FBFE0917C0CF0917D0CAE
:109A50008091860C9091870CA091880CB091890C14
:109A60004089518962897389841B950BA60BB70BBA
:109A70008093860C9093870CA093880CB093890CEC
:109A80004091180A5091190A60911A0A70911B0AA4
:109A90008091900C082E000C990BAA0BBB0B840F25
:109AA000951FA61FB71F8093180A9093190AA093B9
:109AB0001A0AB0931B0A9FB7F89480910B01877F15
:109AC00080930B019FBFE0917C0CF0917D0C409145
:109AD0008A0C50918B0C60918C0C70918D0C84854C
:109AE0009585A685B785840F951FA61FB71F809300
:109AF0008A0C90938B0CA0938C0CB0938D0C181641
:109B000019061A061B060CF03FC081A1813011F422
:109B1000459A01C0149A80918A0C90918B0CA09167
:109B20008C0CB0918D0C4089518962897389841B9A
:109B3000950BA60BB70B80938A0C90938B0CA0937C
:109B40008C0CB0938D0C40911C0A50911D0A6091B1
:109B50001E0A70911F0A8091910C082E000C990B1F
:109B6000AA0BBB0B840F951FA61FB71F80931C0A5F
:109B700090931D0AA0931E0AB0931F0A81A1813001
:109B800011F4459801C014988091940C9091950C13
:109B9000A091960CB091970C0196A11DB11D8093D8
:109BA000940C9093950CA093960CB093970C4089CD
:109BB00051896289738984179507A607B707B0F0A2
:109BC0008091940C9091950CA091960CB091970C6B
:109BD000E0917C0CF0917D0C4489558966897789E8
:109BE000481759076A077B0718F467C02F5F69CECB
:109BF0004091740C5091750C6091760C7091770CBB
:109C0000048D158D268D378DAA27419FB12D529F2A
:109C1000C001629F900D619F800D911D429FB00D0C
:109C2000811D9A1F519FB00D811D9A1F609FB00D1D
:109C3000811D9A1F509FB10D8A1F9A1FB6958A1FCA
:109C40009A1F1124DF01AA5BBF4F2D913C91820F17
:109C5000931F9093930C8093920CEE5BFF4F408187
:109C6000518162817381A0E0B0E0481759076A070B
:109C70007B0720F45093930C4093920C8091920CAC
:109C80009091930C39D69C01909399008093980001
:109C90008091740C9091750CA091760CB091770C1A
:109CA000820F931FA11DB11D8093740C9093750CAE
:109CB000A093760CB093770C76C0408D518D628D59
:109CC000738D481759076A077B0708F060C04091F9
:109CD000780C5091790C60917A0C70917B0C048D0A
:109CE000158D268D378DAA27419FB12D529FE001FA
:109CF000629FD00D619FC00DD11D429FB00DC11D4F
:109D0000DA1F519FB00DC11DDA1F609FB00DC11D3C
:109D1000DA1F509FB10DCA1FDA1FB695CA1FDA1F8E
:109D200011248091920C9091930CE65BFF4F8C175D
:109D30009D0718F48081918102C08C1B9D0B40818E
:109D40005181628173818C0120E030E00417150796
:109D50002607370708F4CA01CFD59C0190939900D4
:109D6000809398008091780C9091790CA0917A0C56
:109D7000B0917B0C820F931FA11DB11D8093780CB5
:109D80009093790CA0937A0CB0937B0C0CC08091CB
:109D9000990C90919A0C90939900809398008091DF
:109DA0009B0C8093980CE0917C0CF0917D0C409181
:109DB000940C5091950C6091960C7091970C808941
:109DC0009189A289B389481759076A077B0708F464
:109DD00056C086A197A1A0A5B1A5B7FF42C08091AA
:109DE000910C8130F1F581A1813011F4439A01C0C9
:109DF000169886A197A1A0A5B1A5919581959109E5
:109E00009093720C8093710CA1A1B0E0AA0FBB1FBC
:109E1000A852BD4E8D919C91880F991F9093290156
:109E200080932801109225011092240180917300E3
:109E30008260809373008091710C9091720C18165F
:109E40001906CCF3809173008D7F8093730016A266
:109E500017A210A611A681A1813011F4439801C068
:109E6000169A10927D0C10927C0C80913712909172
:109E70003612981721F08F5F8F7080933712809180
:109E80007100826080937100F894FF91EF91DF91EF
:109E9000CF91BF91AF919F918F917F916F915F9182
:109EA0004F913F912F911F910F910F900BBE0F90EB
:109EB0000FBE0F901F901895089508954F925F92CE
:109EC0006F927F92AF92BF92CF92DF92EF92FF920A
:109ED0000F931F93CF93DF938C01EB01FC0140A8FC
:109EE00051A862A873A8A8A8B9A8CAA8DBA8950118
:109EF000A601C301B2010E946CD387FF41C0A30138
:109F00009201C301B2010E9485CE2B013C01F801F0
:109F100084AD95ADA6ADB7ADBC01CD0190589B0108
:109F2000AC010E94E7D6F80120AD31AD42AD53AD92
:109F30000E9485CE9B01AC01C301B2010E94E6D60E
:109F40000E9418DA7B018C019B01AC01B501C601AE
:109F50000E946CD387FF02C0750186019701A8019A
:109F6000B501C6010E946CD3882351F0A701B80146
:109F700048AB59AB6AAB7BABC05CDF4F81E08883F9
:109F8000DF91CF911F910F91FF90EF90DF90CF90D5
:109F9000BF90AF907F906F905F904F90089508951D
:109FA0009091C00095FFFCCF8093C600089508955E
:109FB0001F93CF93DF93182FEB0161E039D72097E0
:109FC00011F460E004C0CF3FD10531F461E0812F8E
:109FD000DF91CF911F91FDC6E12FF0E0EF56F84FD2
:109FE000E4914E2F50E0FA013197E231F10508F08B
:109FF000A2C08827EE58FF4F8F4F0C94B4DA84B577
:10A00000806884BDC7BD9CC084B5806284BDC8BD66
:10A0100097C080918000806880938000D0938900F1
:10A02000C09388008DC08091800080628093800002
:10A03000D0938B00C0938A0083C080918000886099
:10A0400080938000D0938D00C0938C0079C0809164
:10A05000B00080688093B000C093B30071C080915D
:10A06000B00080628093B000C093B40069C080915A
:10A070009000806880939000D0939900C0939800DE
:10A080005FC080919000806280939000D0939B008D
:10A09000C0939A0055C08091900088608093900092
:10A0A000D0939D00C0939C004BC08091A00080681D
:10A0B0008093A0008091A0008F7B8093A000D0931C
:10A0C000A900C093A8003CC08091A000806280934A
:10A0D000A000D093AB00C093AA0032C08091A00032
:10A0E00088608093A0008091A00081608093A00090
:10A0F000D093AD00C093AC0023C080912001806854
:10A1000080932001D0932901C093280119C0809128
:10A110002001806280932001D0932B01C0932A01FB
:10A120000FC080912001886080932001D0932D0181
:10A13000C0932C0105C0C038D1050CF047CF41CFEA
:10A14000DF91CF911F910895089590E0FC01319720
:10A15000E231F10508F04EC08827EC57FF4F8F4FD2
:10A160000C94B4DA809180008F7703C080918000D6
:10A170008F7D80938000089580918000877FF9CF44
:10A1800084B58F7702C084B58F7D84BD089580919A
:10A19000B0008F7703C08091B0008F7D8093B000B6
:10A1A0000895809190008F7707C0809190008F7DF7
:10A1B00003C080919000877F8093900008958091E4
:10A1C000A0008F7707C08091A0008F7D03C0809191
:10A1D000A000877F8093A0000895809120018F7751
:10A1E00007C0809120018F7D03C080912001877F6F
:10A1F000809320010895CF92DF92EF92FF920F9308
:10A200001F93CF93DF938C0110928B1610928816B8
:10A2100010928D168EE896E190938A168093891697
:10A220000E94E1C26B017C018091891690918A168F
:10A23000DC01ED91FC910280F381E02D69E119953B
:10A240008091891690918A16DC01ED91FC9100882D
:10A25000F189E02D62E570E0199588E896E10E94A9
:10A260007C9865EB70E18AED9BE00E94AE2A8091BC
:10A27000891690918A16DC01ED91FC910288F38990
:10A28000E02D1995DAE06FEF8091891690918A168A
:10A290000E944C98D150B9F7E601809189169091AF
:10A2A0008A16DC01ED91FC910684F785E02D199565
:10A2B00020E030E0A90160E088E896E10E94E098A3
:10A2C000813049F00E94E1C26C1B7D0B613D7740FB
:10A2D00078F380E27AC02AEA31E040E050E068E0BA
:10A2E00088E896E10E94E098853021F481E080932F
:10A2F0008D1628C064EA70E18AED9BE00E94AE2AC8
:10A3000094E0F92E8091891690918A160E945398B4
:10A3100080938C16FA94F110F5CF8A3A51F482E0CA
:10A3200080938D1665E970E18AED9BE00E94AE2A6C
:10A3300009C00E94E1C26C1B7D0B613D774058F261
:10A3400085E243C080918D16823021F0C12CD12C42
:10A35000760105C0C12CD12CE12C80E4F82E66E8F2
:10A3600070E18AED9BE00E94AE2A20E030E0A90176
:10A3700067E388E896E10E94E098A701960169E208
:10A3800088E896E10E94E098882349F00E94E1C2A3
:10A390006C1B7D0B613D774040F383E416C06AE798
:10A3A00070E18AED9BE00E94AE2A80918D1682308A
:10A3B00009F043C020E030E0A9016AE388E896E1B3
:10A3C0000E94E098882379F087E38093881688E8D4
:10A3D00096E10E945A9864E170E18AED9BE00E9448
:10A3E000AE2A80E047C08091891690918A160E941B
:10A3F0005398807C803C49F483E080938D166BE613
:10A4000070E18AED9BE00E94AE2A809189169091BE
:10A410008A160E9453988091891690918A160E94FC
:10A4200053988091891690918A160E9453986FE4F0
:10A4300070E18AED9BE00E94AE2A88E896E10E94D6
:10A440005A9863E470E18AED9BE00E94AE2A809105
:10A45000891690918A16DC01ED91FC910088F189B2
:10A46000E02DB801199567E270E18AED9BE00E944A
:10A47000AE2A81E0DF91CF911F910F91FF90EF9075
:10A48000DF90CF900895CF92DF92EF92FF920F93DB
:10A490001F93CF93DF93CDB7DEB760970FB6F894D5
:10A4A000DEBF0FBECDBF109296131092951380E5BC
:10A4B00091E0A1DE811106C080E590E09CDE88235A
:10A4C00051F005C00E94F193811111C0F5CF0E9497
:10A4D000F19381110CC0E091DC0BF091DD0BE85F92
:10A4E000FE4F608171818AED9BE00E94AE2A20E0E0
:10A4F00030E0A90169E088E896E10E94E0988823AD
:10A5000021F082E58093881642C040E150E0BE0110
:10A510006F5F7F4F88E896E10E949B988823B9F18E
:10A5200088E896E10E945A988981807CA9F58F81FC
:10A530008370C82ED12CDC2CCC24DD0CDD0C88855E
:10A5400024E0829FC0011124C82AD92A89858295D6
:10A55000869586958370C82A8FEFC81AD80AE12C91
:10A56000F12C2A852370220F8B8587FB882780F9A1
:10A57000282B8E818F7090E0820F911D079704C069
:10A58000CC0CDD1CEE1CFF1C8A95D2F733C088E88A
:10A5900096E10E945A982BC0803449F5CA84D12C88
:10A5A000E12CF12C2FEFC21AD20AE20AF20A8985B5
:10A5B00090E0A0E0B0E0BA2FA92F982F8827C80E0E
:10A5C000D91EEA1EFB1E88858F7390E0A0E0B0E0E4
:10A5D000DC0199278827C80ED91EEA1EFB1E4AE017
:10A5E000CC0CDD1CEE1CFF1C4A95D1F703C0C12C1E
:10A5F000D12C7601C114D104E104F10469F4E09195
:10A60000DC0BF091DD0BE85FFE4F608171818AED1C
:10A610009BE00E94AE2A88C068E070E18AED9BE072
:10A620000E94614680918D16823039F0833041F06E
:10A630008130A9F463E070E114C06EEF7FE011C0D7
:10A6400080E8C8168DE1D8068CE2E80684E0F806BA
:10A6500018F467EF7FE005C061EF7FE002C068EEAD
:10A660007FE08AED9BE00E946146C701B6010E942F
:10A6700070D32DEB37E346E05AE30E9485CE0E946B
:10A6800041D87F936F9387ED9FE09F938F930AED5F
:10A690001BE01F930F930E949E46809146140F90DB
:10A6A0000F900F900F900F900F90E091DC0BF091B6
:10A6B000DD0B811108C0E65FFE4F60817181C8012A
:10A6C0000E94614631C01F928F93E45FFE4F8181EB
:10A6D0008F9380818F931F930F930E949E46E091EA
:10A6E000DC0BF091DD0BE25FFE4F608171818AED42
:10A6F0009BE00E94D12A61E088E696E10E9499934E
:10A7000046E450E06BE973E188E696E10E948488B4
:10A7100081E090E090939613809395130F900F90A3
:10A720000F900F900F900F9060960FB6F894DEBFC9
:10A730000FBECDBFDF91CF911F910F91FF90EF9092
:10A74000DF90CF900895CF92DF92EF92FF920F9318
:10A750001F93CF93DF938C016A017B01EC01CC0F37
:10A76000DD1FCC0FDD1FFE01E15AF54F42835383FD
:10A7700064837583FE01E45CFD4E2081318142815A
:10A780005381C701B6010E9485CE0E94DAD9FE012D
:10A79000E056F34F62837383848395838FB7F89475
:10A7A0004281538164817581C05FD54F488359834D
:10A7B0006A837B838FBF0330110541F4C0920A0A7C
:10A7C000D0920B0AE0920C0AF0920D0ADF91CF9121
:10A7D0001F910F91FF90EF90DF90CF900895CF934E
:10A7E000DF93CDB7DEB7A0970FB6F894DEBF0FBEEC
:10A7F000CDBF19821A821092DE161092DD1640E04B
:10A8000050E0BA0188E696E10E947A9468E676E123
:10A81000CE0101960E942293882389F0898181FDCF
:10A8200009C08091DD169091DE1601969093DE1698
:10A830008093DD16CE0101960E949596E7CF809118
:10A84000DD169091DE16A0960FB6F894DEBF0FBE0F
:10A85000CDBFDF91CF910895CF93DF93CDB7DEB712
:10A86000A0970FB6F894DEBF0FBECDBF19821A8233
:10A87000FC0120812F32E9F4218121111AC088E6E0
:10A8800096E10E94959661E474E188E696E10E9463
:10A890008795811102C080E026C08091681680777C
:10A8A000D1F388E696E190930F0A80930E0A81E037
:10A8B0001AC021E0AC0168E676E1CE0101960E9463
:10A8C000A396882341F39981907729F390E2FE01C2
:10A8D0003196A8E6B6E101900D929A95E1F7909134
:10A8E00068169077F1F6A0960FB6F894DEBF0FBE0B
:10A8F000CDBFDF91CF91089581342CE9920728F4E0
:10A9000081322EE4920748F002C080E49CE99695DB
:10A9100087959695879524E007C0813127E29207B5
:10A9200030F09695879522E02093980C08C021E09E
:10A930002093980C8032910510F480E290E0AC01F5
:10A9400040525109411588E05807D8F0E52FFF27FC
:10A95000EE0FFF1FEE0FFF1FCF018952944FFC0136
:10A96000329665917491AA27479F9001469F210DC9
:10A970003A1F06942A1F3A1F1124FC0185919491D5
:10A980001CC09A01369527952C7F2952384FF90122
:10A9900085919491F9013296A591B491BA016770AD
:10A9A0007727A69F9001A79F300DB69F300D1124E9
:10A9B00063E0369527956A95E1F7821B930B843601
:10A9C0009105D0F45F934F938AED9BE0E091DC0B0F
:10A9D000F091DD0BE45CFE4F21812F9320812F93BA
:10A9E0009F938F930E949E460F900F900F900F9011
:10A9F0000F900F9084E690E008958F929F92AF920F
:10AA0000BF92CF92DF92EF92FF920F931F93CF935B
:10AA1000DF93EB01670178016091010270910202FE
:10AA20007093450960934409609140097091410910
:10AA300070933F0960933E09812C912C60E8A62E0B
:10AA40006FE3B62E80923A0990923B09A0923C099E
:10AA5000B0923D0962E060932B0260E770E670936C
:10AA60000202609301029093390980933809D093D0
:10AA70003709C0933609CA01B9010E9441D86093D1
:10AA80003209709333098093340990933509C701D3
:10AA9000B6010E9441D860932E0970932F098093CC
:10AAA00030099093310988819981092E000CAA0BF5
:10AAB000BB0B8093400990934109A0934209B09346
:10AAC0004309DF91CF911F910F91FF90EF90DF909D
:10AAD000CF90BF90AF909F908F9008950F931F934A
:10AAE00020910102309102023093450920934409DC
:10AAF000209140093091410930933F0920933E094C
:10AB000000E010E020E83FE300933A0910933B098E
:10AB100020933C0930933D0922E020932B0224EB43
:10AB20003FE530930202209301029093390980930C
:10AB300038097093370960933609109232091092E0
:10AB4000330910923409109235098EE091E0A0E0AB
:10AB5000B0E080932E0990932F09A0933009B09311
:10AB60003109FB0180819181092E000CAA0BBB0BDE
:10AB70008093400990934109A0934209B0934309FF
:10AB800050932D0940932C091F910F910895CF9256
:10AB9000DF92EF92FF92CF93DF93EB0169017A018D
:10ABA000209101023091020230934509209344091B
:10ABB000209140093091410930933F0920933E098B
:10ABC000C0923A09D0923B09E0923C09F0923D09CB
:10ABD00022E020932B0228E63DE5309302022093E9
:10ABE0000102909339098093380970933709609373
:10ABF000360920E030E048EC52E4C701B6010E947B
:10AC000085CE0E9441D860933209709333098093B6
:10AC100034099093350920E03CE541EC57E4C70145
:10AC2000B6010E9485CE0E9441D860932E09709390
:10AC30002F098093300990933109688179818A8145
:10AC40009B810E9470D3A70196010E9485CE0E942D
:10AC500047D86093400970934109809342099093CB
:10AC600043098BE29FE990932D0980932C09DF9192
:10AC7000CF91FF90EF90DF90CF900895E091F9167B
:10AC8000F091FA160190F081E02D682F89EF96E19E
:10AC90001994FF920F931F93CF93DF93F82E142FE5
:10ACA000052FE90180E00E94AA7FFF2011F08EE3CA
:10ACB00001C080E2E3DF89818F9388818F930F93B6
:10ACC0001F93AFD30F900F900F900F90DF91CF9104
:10ACD0001F910F91FF900C94AE6EFF920F931F93F4
:10ACE000CF93DF93F82E142F052FE90180E00E9407
:10ACF000AA7FFF2011F08EE301C080E2BFDF8B81CD
:10AD00008F938A818F9389818F9388818F930F93FB
:10AD10001F9387D30F900F900F900F900F900F906D
:10AD2000DF91CF911F910F91FF900C94AE6EFF9227
:10AD30000F931F93CF93DF93F82E142F052FE90164
:10AD400080E00E94AA7FFF2011F08EE301C080E224
:10AD500095DF8B818F938A818F9389818F938881EF
:10AD60008F930F931F935DD30F900F900F900F90C1
:10AD70000F900F90DF91CF911F910F91FF900C9446
:10AD8000AE6ECF93DF93282F30E0F901EF56F84FE6
:10AD90008491F901E55BF84FD491F901EB5FF84F2D
:10ADA000C491CC2389F08111D0D9EC2FF0E0EE0FC3
:10ADB000FF1FE551F94FA591B491EC91ED2381E08E
:10ADC00090E021F480E002C080E090E0DF91CF913C
:10ADD00008951F93CF93DF93282F30E0F901EF56AA
:10ADE000F84F8491F901E55BF84FD491F901EB5FDD
:10ADF000F84FC491CC23C1F0162F8111A6D9EC2FA6
:10AE0000F0E0EE0FFF1FEF52F94FA591B4918FB70D
:10AE1000F894111105C09C91ED2FE095E92302C033
:10AE2000EC91ED2BEC938FBFDF91CF911F910895A3
:10AE3000CF93DF9390E0FC01E55BF84F2491FC0198
:10AE4000EB5FF84F8491882361F190E0880F991FA0
:10AE5000FC01E954F94FC591D491FC01EF52F94F2F
:10AE6000A591B491611109C09FB7F894888120958C
:10AE700082238883EC912E230BC0623061F49FB74C
:10AE8000F8943881822F809583238883EC912E2B30
:10AE90002C939FBF06C08FB7F894E8812E2B288390
:10AEA0008FBFDF91CF9108958F929F92AF92BF9203
:10AEB000CF92DF92EF92FF926B017C010E94BCC2A5
:10AEC0004B015C01C114D104E104F104F1F00E94D2
:10AED000BCC2DC01CB0188199909AA09BB09883ECB
:10AEE0009340A105B10570F321E0C21AD108E10831
:10AEF000F10888EE880E83E0981EA11CB11CC114D5
:10AF0000D104E104F10419F7DDCFFF90EF90DF9059
:10AF1000CF90BF90AF909F908F90089585ED8093D4
:10AF2000BC008091BC0084FDFCCF1092D309089531
:10AF30001F920F920FB60F9211240BB60F922F9300
:10AF40003F934F935F936F937F938F939F93AF93B1
:10AF5000BF93EF93FF938091B900887F803609F407
:10AF60009CC068F5883209F45BC090F4803109F424
:10AF700054C038F4882309F4F6C0883009F44DC071
:10AF8000F5C0883109F44CC0803209F45DC0EEC0D0
:10AF9000803409F468C048F4803309F455C088331C
:10AFA00009F0E4C08093D209D8C0803509F44FC0BD
:10AFB000883509F45DC0883409F0D8C0D6C0883916
:10AFC00009F4C7C0A8F4883709F467C038F4883694
:10AFD00009F463C0803709F460C0C8C0883809F438
:10AFE000B8C0803909F45FC0803809F0BFC05BC0C9
:10AFF000803B09F486C038F4803A09F466C0883A88
:10B0000009F47FC0B3C0803C09F4A7C0883C09F4B0
:10B01000A4C0883B09F48AC0A9C08091F80910C077
:10B020009091F7098091F609981770F5E091F7096A
:10B0300081E08E0F8093F709F0E0EA52F64F8081AD
:10B040008093BB0085EC86C08093D2098EC0E091CE
:10B05000F70981E08E0F8093F7098091BB00F0E043
:10B06000EA52F64F80839091F7098091F6096EC0FD
:10B07000E091F70981E08E0F8093F7098091BB0082
:10B08000F0E0EA52F64F80838091D50981116DC0BE
:10B0900081E08093D40984EA61C083E08093D3097E
:10B0A0001092D109CFCF8091D109803208F051C0E0
:10B0B000E091D10981E08E0F8093D1098091BB008E
:10B0C000F0E0EF54F64F8083BDCF85EC8093BC0059
:10B0D0001092D3098091D109803230F4E091D109E6
:10B0E000F0E0EF54F64F10826091D10970E0E091EA
:10B0F000AF09F091B00981EB99E019951092D1094F
:10B1000035C084E08093D3091092AE091092AD0946
:10B11000E091AB09F091AC0919958091AD098111CD
:10B1200005C081E08093AD0910928B09E091AE09D2
:10B1300081E08E0F8093AE09F0E0E557F64F8081F5
:10B140008093BB009091AE098091AD09981708F4E7
:10B1500079CF85E88093BC0009C085EC8093BC0062
:10B160001092D30903C01092D209D8DEFF91EF915B
:10B17000BF91AF919F918F917F916F915F914F910F
:10B180003F912F910F900BBE0F900FBE0F901F900D
:10B1900018954091AD09262F30E0240F311D213242
:10B1A0003105DCF42091D3092430C9F4FC0180E09E
:10B1B00090E0861758F43091AD092191DC01A55734
:10B1C000B64FA30FB11D2C930196F3CF8091AD091B
:10B1D000680F6093AD0980E0089581E0089582E0F2
:10B1E00008954F925F926F927F928F929F92AF924B
:10B1F000BF92CF92DF92EF92FF920F931F93CF9364
:10B20000DF9300D01F92CDB7DEB74B0129833A837D
:10B210004B835C83209101023091020230934509F7
:10B2200020934409209140093091410930933F090E
:10B2300020933E09A0923A09B0923B09C0923C0982
:10B24000D0923D0922E020932B0223E33EE5309388
:10B250000202209301029093390980933809709378
:10B26000370960933609A601950169817A818B813E
:10B270009C810E9485CE0E9441D8609332097093D0
:10B2800033098093340990933509A6019501C801CB
:10B29000B7010E9485CE0E9441D860932E09709319
:10B2A0002F098093300990933109F4012081318175
:10B2B00042815381C601B5010E9485CE0E9447D8C4
:10B2C0006093400970934109809342099093430928
:10B2D0000F900F900F900F90DF91CF911F910F91D2
:10B2E000FF90EF90DF90CF90BF90AF909F908F90A6
:10B2F0007F906F905F904F9008952F923F924F9262
:10B300005F926F927F928F929F92AF92BF92CF92F5
:10B31000DF92EF92FF920F931F93CF93DF9300D0B2
:10B320001F92CDB7DEB73B0129833A834B835C8301
:10B330002091010230910202309345092093440983
:10B34000209140093091410930933F0920933E09F3
:10B35000A0923A09B0923B09C0923C09D0923D09B3
:10B3600022E020932B022DEE3EE530930202209343
:10B3700001029093390980933809709337096093DB
:10B380003609A601950169817A818B819C810E9491
:10B3900085CE0E9441D8609332097093330980931F
:10B3A000340990933509A6019501C801B7010E949F
:10B3B00085CE0E9441D860932E0970932F09809307
:10B3C000300990933109F301208131814281538109
:10B3D000C601B5010E9485CE0E9447D860934009FE
:10B3E00070934109809342099093430990922D09EB
:10B3F00080922C090F900F900F900F90DF91CF91BA
:10B400001F910F91FF90EF90DF90CF90BF90AF9082
:10B410009F908F907F906F905F904F903F902F9074
:10B4200008952F923F924F925F926F927F928F92E8
:10B430009F92AF92BF92CF92DF92EF92FF920F93C3
:10B440001F93CF93DF931F921F92CDB7DEB7DE011C
:10B450005896ED90FD90F701849100E010E088236C
:10B4600009F471C1853209F062C18093810982E0DB
:10B47000282E312C812C912C60E081E090E0FFEFB0
:10B48000EF1AFF0AF7017491753229F4F801E75AAF
:10B49000F64F708350C1272F072E000C330B20531B
:10B4A00031092A30310568F4AC014F5F5F4FFC0170
:10B4B000EF57F64F7083662311F0190101C049015F
:10B4C000CA017E3239F4FC01EF57F64F70830196C2
:10B4D00061E0D5CF793611F0793419F5FC01EF57D9
:10B4E000F64F708311826D01F2E0CF0ED11C1196E0
:10B4F0008C9111978F938C918F93A1E8B9E0BF93B2
:10B50000AF93C801875A964F9F938F930E94E5DBB4
:10B51000080F191F0F900F900F900F900F900F9022
:10B520002DC07C3611F07C3459F5FC01EF57F64FF5
:10B53000708311826D01F4E0CF0ED11C13968C91B3
:10B5400013978F9312968C9112978F9311968C91DB
:10B5500011978F938C918F93A1E8B9E0BF93AF932C
:10B56000C801875A964F9F938F930E94E5DB080F7F
:10B57000191F0FB6F894DEBF0FBECDBFD601DDC0D8
:10B580007F7D763409F0BAC0CD0104969A83898311
:10B590004D905D906D907C9020E030E0A901C3015A
:10B5A000B2010E946CD387FF0BC0F801E75AF64F37
:10B5B0008DE2808377FA709477F870940F5F1F4F55
:10B5C000D12C60E070E080E09FE32D2D30E022156B
:10B5D000330544F420E030E040E251E40E94D0D74B
:10B5E000D394F3CF9B01AC01C301B2010E94E7D613
:10B5F0002B013C010E9447D8D62EC72EB82EA92E6B
:10B600000E9470D39B01AC01C301B2010E94E6D637
:10B610002B013C01C801875A964FA2E08A1691047B
:10B6200071F0B3E08B16910489F08A948928A9F40B
:10B63000AF92BF92CF92DF92AFE0B1E114C0AF9270
:10B64000BF92CF92DF92ABE0B1E10DC0AF92BF925B
:10B65000CF92DF92A7E0B1E106C0AF92BF92CF9246
:10B66000DF92A4E0B1E1BF93AF939F938F930E94C9
:10B670003DD3080F191F0FB6F894DEBF0FBECDBF24
:10B68000121413043CF4F801E75AF64F3EE23083FB
:10B690000F5F1F4F6101C801875A964F5C011C1450
:10B6A0001D041CF520E030E040E251E4C301B2018A
:10B6B0000E9485CE2B013C010E9441D820E3260F39
:10B6C000D5012D935D01072E000C880B990B0E946C
:10B6D00072D39B01AC01C301B2010E94E6D62B01DB
:10B6E0003C01B1E0CB1AD108DACF37FE02C0212CE1
:10B6F000312C020D131DA981BA811FC0733509F0C9
:10B70000BECEFD01C801875A964F608171811296A5
:10B710009801261B370B8901060F171FFB0141916A
:10B72000BF01442351F0FC014193CF01F4CFF80154
:10B73000E75AF64F80830F5F1F4FFFEFEF1AFF0AA4
:10B74000F70184918CCEF801E75AF64F108289E513
:10B7500099E00F900F90DF91CF911F910F91FF9083
:10B76000EF90DF90CF90BF90AF909F908F907F90A1
:10B770006F905F904F903F902F90089520E030E0C1
:10B7800040E251E4FC0160817181828193810E94D9
:10B7900085CE0E9441D877FF02C02DE201C02BE286
:10B7A000209351099B0177FF04C022273327261BD2
:10B7B000370BC90168EE73E00E9485DACB01EAE03D
:10B7C000F0E0BF010E9485DA805D80935209C901D3
:10B7D00064E670E00E9485DACB01BF010E9485DA41
:10B7E000805D80935309C901BF010E9485DA282F2B
:10B7F000CB01BF010E9485DA805D809354098EE2FF
:10B8000080935509205D209356091092570981E5D0
:10B8100099E00895CF92DF92EF92FF92CF93C0917B
:10B820000001C095C1708091000181FFC260C0908D
:10B830004D09D0904E09E0904F09F09050090E94B8
:10B84000E1C2C616D706E806F90610F4019B39C016
:10B85000C0934B0980914B09817090914B0991FDE8
:10B86000826090914C09891721F18130F1F028F024
:10B87000823089F08330A1F01CC0913021F4909186
:10B88000F5059F5F05C09230A1F49091F5059150A8
:10B890009093F5050EC0992391F3933051F4F5CFB1
:10B8A000923069F3913029F4F0CF933041F399232A
:10B8B00061F380934C09CF91FF90EF90DF90CF9090
:10B8C0000895C46068E97AE380E090E00E9463AA8A
:10B8D000BFCF4CE350E0BC0182E29AE00E9414D357
:10B8E0000E948BB582E080932B0208950F931F93E3
:10B8F00091DF0E94E1C20091020C1091030C209193
:10B90000040C3091050C061717072807390708F0B3
:10B91000A1C08091F505282F082E000C330B37FFAE
:10B9200003C03195219531092430310544F191E06E
:10B9300090932B0287FD8D5F85958595082E000CD1
:10B94000990BAA0BBB0B40914009509141096091A2
:10B95000420970914309840F951FA61FB71F80935A
:10B96000400990934109A0934209B0934309109272
:10B97000F50568E873E180E090E00E9463AA809199
:10B980004B0982FF12C080910102909102028F58F0
:10B990009B4B29F460E67AEE80E090E004C068E911
:10B9A0007AE380E090E00E9463AAE0910102F091C6
:10B9B000020219950E94E1C20091F20B1091F30B63
:10B9C0002091F40B3091F50B06171707280739075C
:10B9D00090F480910102909102028E599F4659F095
:10B9E00068E97AE380E090E00E9463AA0E94CB6954
:10B9F00082E080932B0280912B02823021F489EF28
:10BA000096E10E944D9A80912B02882319F0815073
:10BA100080932B028091710A882349F09091720AD9
:10BA2000992331F09091730A81E0892701C081E068
:10BA300080934A090E94E1C2DC01CB018C599F4FDF
:10BA4000AF4FBF4F8093020C9093030CA093040C54
:10BA5000B093050C1F910F9108959093020280936B
:10BA6000010210924009109241091092420910926D
:10BA7000430968E97AE380E090E00C9463AA90932C
:10BA80000202809301021092400910924109109223
:10BA900042091092430982E080932B0268E97AE31D
:10BAA00080E090E00C9463AA82E080932B020E94D5
:10BAB000E1C2DC01CB018C509E4FAF4FBF4F809352
:10BAC0004D0990934E09A0934F09B09350090895E2
:10BAD000EF92FF920F931F93CF93DF931F921F92CA
:10BAE000CDB7DEB78091320990913309A091340926
:10BAF000B091350940914009509141096091420946
:10BB000070914309481759076A077B0744F48093EB
:10BB1000400990934109A0934209B0934309809151
:10BB20002E0990912F09A0913009B09131094091CF
:10BB3000400950914109609142097091430984176D
:10BB40009507A607B70744F48093400990934109ED
:10BB5000A0934209B093430980912B02882399F165
:10BB60006091400970914109809142099091430987
:10BB70000E9470D320913A0930913B0940913C09D1
:10BB800050913D090E94D0D70E9447D8162F082F08
:10BB9000F0903809E090390961E081E079839A8377
:10BBA0000E94AA7F9A819F930F9379817F931F931D
:10BBB000EF92FF9236DC0E94AE6E0F900F900F90C6
:10BBC0000F900F900F9080914B0982FF43C000911E
:10BBD00036091091370960914009709141098091AF
:10BBE0004209909143090E9470D320913A09309103
:10BBF0003B0940913C0950913D090E94D0D70E94D9
:10BC000047D8F80160837183828393834DDF8091ED
:10BC1000440990914509909302028093010280911A
:10BC20003E0990913F09A0E0B0E0809340099093D5
:10BC30004109A0934209B0934309E0912C09F09186
:10BC40002D090F900F90DF91CF911F910F91FF90D1
:10BC5000EF9019940F900F90DF91CF911F910F915A
:10BC6000FF90EF900895EF92FF920F931F93CF9361
:10BC7000DF931F921F92CDB7DEB78091320990916A
:10BC80003309A0913409B091350940914009509190
:10BC900041096091420970914309481759076A07A1
:10BCA0007B0744F48093400990934109A093420993
:10BCB000B093430980912E0990912F09A0913009EA
:10BCC000B091310940914009509141096091420978
:10BCD0007091430984179507A607B70744F480932A
:10BCE000400990934109A0934209B0934309809180
:10BCF0002B02882389F1609140097091410980915C
:10BD00004209909143090E9470D320913A093091E1
:10BD10003B0940913C0950913D090E94D0D7162F14
:10BD2000082FF0903809E090390961E081E07983CB
:10BD30009A830E94AA7F9A819F930F9379817F9320
:10BD40001F93EF92FF926DDB0E94AE6E0F900F90EB
:10BD50000F900F900F900F9080914B0982FF34C08D
:10BD6000009136091091370960914009709141099D
:10BD700080914209909143090E9470D320913A0921
:10BD800030913B0940913C0950913D090E94D0D728
:10BD9000F801608371838283938386DE80914409F6
:10BDA00090914509909302028093010280913E098F
:10BDB00090913F09A0E0B0E0809340099093410941
:10BDC000A0934209B09343090F900F90DF91CF9158
:10BDD0001F910F91FF90EF900895EF92FF920F93B4
:10BDE0001F93CF93DF931F921F92CDB7DEB7809141
:10BDF000320990913309A0913409B09135094091ED
:10BE000040095091410960914209709143094817D6
:10BE100059076A077B0744F48093400990934109CE
:10BE2000A0934209B093430980912E0990912F0964
:10BE3000A0913009B09131094091400950914109D8
:10BE4000609142097091430984179507A607B707C7
:10BE500044F48093400990934109A0934209B09320
:10BE6000430980912B02882389F1609140097091E8
:10BE7000410980914209909143090E9470D3209119
:10BE80003A0930913B0940913C0950913D090E948B
:10BE9000D0D7162F082FF0903809E090390961E0CB
:10BEA00081E079839A830E94AA7F9A819F930F935E
:10BEB00079817F931F93EF92FF92B3DA0E94AE6E67
:10BEC0000F900F900F900F900F900F9080914B0953
:10BED00082FF41C0009136091091370960914009F5
:10BEE0007091410980914209909143090E9470D359
:10BEF00020913A0930913B0940913C0950913D090C
:10BF00000E94D0D7F8016083718382839383CCDD54
:10BF10008091440990914509909302028093010217
:10BF200080913E0990913F09A0E0B0E080934009E4
:10BF300090934109A0934209B0934309E0912C09E1
:10BF4000F0912D090F900F90DF91CF911F910F91DC
:10BF5000FF90EF9019940F900F90DF91CF911F9168
:10BF60000F91FF90EF900895FF920F931F93CF933F
:10BF7000DF931F92CDB7DEB78091320990913309DC
:10BF8000A0913409B091350940914009509141097F
:10BF90006091420970914309481759076A077B0766
:10BFA00044F48093400990934109A0934209B093CF
:10BFB000430980912E0990912F09A0913009B091E9
:10BFC00031094091400950914109609142097091B5
:10BFD000430984179507A607B70744F480934009DF
:10BFE00090934109A0934209B093430980912B0299
:10BFF000882361F160914009709141098091420963
:10C00000909143090E9470D320913A0930913B09E5
:10C0100040913C0950913D090E94D0D70E9441D8DF
:10C02000162F00913809F090390961E081E0798399
:10C030000E94AA7F79817F931F93FF920F93F1D97A
:10C040000E94AE6E0F900F900F900F9080914B0951
:10C0500082FF3FC000913609109137096091400975
:10C0600070914109072E000C880B990B0E9472D326
:10C0700020913A0930913B0940913C0950913D098A
:10C080000E94D0D70E9441D8F801718360830CDDF3
:10C090008091440990914509909302028093010296
:10C0A00080913E0990913F09A0E0B0E08093400963
:10C0B00090934109A0934209B0934309E0912C0960
:10C0C000F0912D090F90DF91CF911F910F91FF906B
:10C0D00019940F90DF91CF911F910F91FF900895C8
:10C0E000FF920F931F93CF93DF931F92CDB7DEB7CD
:10C0F0008091320990913309A0913409B0913509AA
:10C100004091400950914109609142097091430961
:10C11000481759076A077B0744F4809340099093B6
:10C120004109A0934209B093430980912E0990914F
:10C130002F09A0913009B0913109409140095091E7
:10C140004109609142097091430984179507A60738
:10C15000B70744F48093400990934109A0934209A2
:10C16000B093430980912B02882361F160914009CB
:10C170007091410980914209909143090E9470D3C6
:10C1800020913A0930913B0940913C0950913D0979
:10C190000E94D0D70E9441D8162F00913809F09004
:10C1A000390961E081E079830E94AA7F79817F93D8
:10C1B0001F93FF920F9335D90E94AE6E0F900F9090
:10C1C0000F900F9080914B0982FF34C00091360987
:10C1D000109137096091400970914109809142099D
:10C1E000909143090E9470D320913A0930913B0904
:10C1F00040913C0950913D090E94D0D70E9441D8FE
:10C20000F8017183608350DC809144099091450965
:10C21000909302028093010280913E0990913F0920
:10C22000A0E0B0E08093400990934109A0934209B7
:10C23000B09343090F90DF91CF911F910F91FF9021
:10C240000895AF92BF92CF92DF92EF92FF920F9339
:10C250001F93CF93DF9310924909809140099091E9
:10C260004109A0914209B091430981309048A1054C
:10C27000B10540F010924009109241091092420914
:10C280001092430980914009809348099091470991
:10C29000891710F480934709D091470910914B09F1
:10C2A00012FB112710F9C0E083E0C82ED12CE12C3D
:10C2B000F12C93E0B92E22E0A22E90914809D111E1
:10C2C00025C081E0911180E08093460990912B0276
:10C2D000992339F000E22EE342EF50E16C2F0E94E7
:10C2E000DA69112309F446C080914609882309F4CC
:10C2F00041C0DADBDF91CF911F910F91FF90EF905A
:10C30000DF90CF90BF90AF900C94CB69D13079F48F
:10C3100081E0913009F080E08093460990912B02F2
:10C320009923F9F200E22EE34FED50E1D7CFD2305E
:10C3300079F481E0923009F080E080934609909191
:10C340002B02992371F200E22EE341ED50E1C6CFBA
:10C35000D33081F481E0933009F080E08093460986
:10C3600090912B02992309F4BCCF00E22EE341EC1B
:10C3700050E1B4CF80914809843050F0C092400918
:10C38000D0924109E0924209F0924309B0924809E3
:10C39000209148098091470990E00396422F50E090
:10C3A000841795074CF48DEF820F80934709A09274
:10C3B0002B02DCEFD20FCFEFCF5FDF5FC43008F48A
:10C3C0007CCFDF91CF911F910F91FF90EF90DF9085
:10C3D000CF90BF90AF9008958091010A9091020A8A
:10C3E000A091030AB091040A809390129093911245
:10C3F000A0939212B093931208958091010A9091A4
:10C40000020AA091030AB091040A80938C129093BF
:10C410008D12A0938E12B0938F1208958F929F92D7
:10C42000AF92BF92CF92DF92EF92FF920F931F9342
:10C43000CF93DF931092490980914009909141096F
:10C44000A0914209B091430981309048A105B105FE
:10C4500040F0109240091092410910924209109246
:10C4600043098091400980934809909147098917B1
:10C4700010F480934709D091470910914B0912FBA2
:10C48000112710F9C0E0EE24E394F12C0FE0802E88
:10C49000912CA12CB12C8FE0D82E92E0C92E909136
:10C4A0004809D1112BC081E0911180E080934609A9
:10C4B00090912B02992351F0E091DC0BF091DD0B70
:10C4C0004689578903E023E06C2F74D7112309F4C0
:10C4D000B2C080914609882309F4ADC0E5DA8EEA3E
:10C4E00096E6DF91CF911F910F91FF90EF90DF9033
:10C4F000CF90BF90AF909F908F90C1CAD13059F527
:10C5000081E0913009F080E08093460990912B0200
:10C51000992369F0E091DC0BF091DD0BE257FF4FBE
:10C520004081518124EA3AE06C2F0E944956112340
:10C5300009F481C080914609882309F47CC0B4DAEB
:10C54000E091DC0BF091DD0BE257FF4F49EC59E62F
:10C5500064EA7AE02CC0D230D1F581E0923009F063
:10C5600080E08093460990912B02992369F0E09135
:10C57000DC0BF091DD0BE057FF4F4081518126EA43
:10C580003AE06C2F0E944956112309F454C080915F
:10C590004609882309F44FC087DAE091DC0BF0915B
:10C5A000DD0BE057FF4F4AEC59E666EA7AE08081FE
:10C5B0009181DF91CF911F910F91FF90EF90DF90CC
:10C5C000CF90BF90AF909F908F900C946E55D330CA
:10C5D00091F581E0933009F080E0809346099091D5
:10C5E0002B02992369F0E091DC0BF091DD0BEC5606
:10C5F000FF4F408151812EEA3AE06C2F0E9449564C
:10C600001123C9F0809146098823A9F04DDAE09101
:10C61000DC0BF091DD0BEC56FF4FE12CF12C0FE71A
:10C6200013E420E030E0A9016EEA7AE08081918194
:10C630000E94FD5426C31092060A1092050A2DEBA3
:10C6400037E346E05EE36091941270919512809119
:10C650009612909197120E94D0D76093FD09709323
:10C66000FE098093FF099093000A2DEB37E346E023
:10C670005EE360919C1270919D1280919E12909148
:10C680009F120E9485CE6093F9097093FA098093F6
:10C69000FB099093FC0980918C1290918D12A091CE
:10C6A0008E12B0918F128093010A9093020AA09388
:10C6B000030AB093040A90914809D43059F581E0F7
:10C6C000943009F080E08093460990912B029923E1
:10C6D00069F0E091DC0BF091DD0BEC55FF4F4081F0
:10C6E000518121E03AE06C2F0E946D56112309F42C
:10C6F000F0C080914609882309F4EBC0D5D9E091B8
:10C70000DC0BF091DD0BEC55FF4F7DEF872E71E6D2
:10C71000972E4DC1D53009F040C081E0953009F029
:10C7200080E08093460990912B02992369F0E09173
:10C73000DC0BF091DD0BEA55FF4F408151812DEF6D
:10C7400039E06C2F0E946D56112309F4C2C080910C
:10C750004609882309F4BDC0A7D9E091DC0BF0910C
:10C76000DD0BEA55FF4F66E9862E66E6962EA12C74
:10C77000B12C48ECC42E42E4D42EE12C18E1F12E69
:10C780000CE116E42AE037ED43E25CE36DEF79E07B
:10C79000808191810E947D5974C2D63059F581E023
:10C7A000963009F080E08093460990912B029923FE
:10C7B00069F0E091DC0BF091DD0BE855FF4F408113
:10C7C000518129EF39E06C2F0E946D56112309F435
:10C7D00080C080914609882309F47BC065D9E09127
:10C7E000DC0BF091DD0BE855FF4F3EE7832E36E67C
:10C7F000932E48C1D730B9F581E0973009F080E039
:10C800008093460990912B02992369F0E091DC0B0B
:10C81000F091DD0BE655FF4F4081518124EA32E172
:10C820006C2F0E946D56112309F453C08091460964
:10C83000882309F44EC038D9E091DC0BF091DD0B70
:10C84000E655FF4FA12CB12C90E8C92E9FE3D92EBD
:10C85000E12C18E1F12E0CE116E420E030E0A90112
:10C8600064EA72E193C1D830A1F581E0983009F013
:10C8700080E08093460990912B02992369F0E09122
:10C88000DC0BF091DD0BE455FF4F408151812CEA28
:10C8900032E16C2F0E946D561123D9F08091460928
:10C8A0008823B9F001D9E091DC0BF091DD0BE45560
:10C8B000FF4FA12CB12CD8E4CD2ED2E4DD2EE12CFB
:10C8C000F12C00E81FE320E030E0A9016CEA72E1FE
:10C8D0005DC1F092060AE092050A2DEB37E346E0CF
:10C8E0005EE3609198127091991280919A129091E2
:10C8F0009B120E94D0D76093FD097093FE0980932C
:10C90000FF099093000A2DEB37E346E05EE3609168
:10C91000A0127091A1128091A2129091A3120E9474
:10C9200085CE6093F9097093FA098093FB0990937F
:10C93000FC098091901290919112A0919212B09165
:10C9400093128093010A9093020AA093030AB09372
:10C95000040A90914809D930E1F581E0993009F055
:10C9600080E08093460990912B02992369F0E09131
:10C97000DC0BF091DD0BE255FF4F4081518121E04E
:10C980003AE06C2F0E946D56112309F453C1809137
:10C990004609882309F44EC187D8E091DC0BF09159
:10C9A000DD0BE255FF4FCCEE8C2EC1E69C2EA12C68
:10C9B000B12CA8ECCA2EA2E4DA2EE12C18E1F12E5B
:10C9C0000CE116E420E030E040E85FE361E07AE06B
:10C9D000DFCEDA3059F581E09A3009F080E08093BB
:10C9E000460990912B02992369F0E091DC0BF091BC
:10C9F000DD0BE055FF4F408151812DEF39E06C2F69
:10CA00000E946D56112309F415C1809146098823AF
:10CA100009F410C149D8E091DC0BF091DD0BE05531
:10CA2000FF4F76E6872E76E6972EA1CEDB30E1F536
:10CA300081E09B3009F080E08093460990912B02C1
:10CA4000992369F0E091DC0BF091DD0BEE54FF4F80
:10CA50004081518129EF39E06C2F0E946D561123DE
:10CA600009F4E8C080914609882309F4E3C01CD882
:10CA7000E091DC0BF091DD0BEE54FF4F6EE4862E5F
:10CA800066E6962EA12CB12C48ECC42E42E4D42E9E
:10CA9000E12C18E1F12E0CE116E420E030E040E852
:10CAA0005FE369EF79E074CEDC30C1F581E09C3062
:10CAB00009F080E08093460990912B02992369F058
:10CAC000E091DC0BF091DD0BEC54FF4F4081518184
:10CAD00028EA32E16C2F0E946D56112309F4AAC096
:10CAE00080914609882309F4A5C00E94545DE09115
:10CAF000DC0BF091DD0BEC54FF4FA12CB12C20E8A6
:10CB0000C22E2FE3D22EE12C18E1F12E0CE116E417
:10CB100020E030E0A90168EA72E138C0DD30D9F5E3
:10CB200081E09D3009F080E08093460990912B02CE
:10CB3000992369F0E091DC0BF091DD0BEA54FF4F93
:10CB40004081518120EB32E16C2F0E946D56112300
:10CB500009F470C080914609882309F46BC00E94D3
:10CB6000545DE091DC0BF091DD0BEA54FF4FA12CFA
:10CB7000B12C88E4C82E82E4D82EE12CF12C00E8F8
:10CB80001FE320E030E0A90160EB72E18081918138
:10CB90000E94F15876C0DE30F9F481E09E3009F051
:10CBA00080E08093460990912B02992351F0E09107
:10CBB000DC0BF091DD0B40A151A10EE72EE36C2FB1
:10CBC000F9D31123B9F180914609882399F10E9484
:10CBD000545D8DE29FE920C0DF3061F581E09F3038
:10CBE00009F080E08093460990912B02992351F03F
:10CBF000E091DC0BF091DD0B42A153A10EE72EE397
:10CC00006C2FD8D31123B1F080914609882391F07D
:10CC10000E94545D8BE590EADF91CF911F910F91B7
:10CC2000FF90EF90DF90CF90BF90AF909F908F904C
:10CC30000C942D5D80914809803150F0809240091C
:10CC400090924109A0924209B0924309D0924809BA
:10CC5000209148098091470990E00396422F50E0C7
:10CC6000841795074CF48DEF820F80934709C0928B
:10CC70002B02DCEFD20FCFEFCF5FDF5FC43008F4C1
:10CC80000ECCDF91CF911F910F91FF90EF90DF902D
:10CC9000CF90BF90AF909F908F9008952DEB37E38A
:10CCA00046E05EE36091F9097091FA098091FB0911
:10CCB0009091FC090E94D0D76093A0127093A112AA
:10CCC0008093A2129093A3120C94F6B42DEB37E349
:10CCD00046E05EE36091FD097091FE098091FF09D5
:10CCE0009091000A0E9485CE6093981270939912D9
:10CCF00080939A1290939B120C94F6B42DEB37E329
:10CD000046E05EE36091F9097091FA098091FB09B0
:10CD10009091FC090E94D0D760939C1270939D1251
:10CD200080939E1290939F120C94F6B42DEB37E3F0
:10CD300046E05EE36091FD097091FE098091FF0974
:10CD40009091000A0E9485CE609394127093951280
:10CD500080939612909397120C94F6B4AF92BF9270
:10CD6000CF92DF92EF92FF920F931F93CF93DF93B7
:10CD7000109249098091400990914109A09142097E
:10CD8000B091430981309048A105B10540F010925F
:10CD90004009109241091092420910924309809172
:10CDA00040098093480990914709891710F48093AE
:10CDB0004709D091470910914B0912FB112710F92F
:10CDC000C0E086E0C82ED12CE12CF12C96E0B92EE3
:10CDD00022E0A22E90914809D1112BC081E091113F
:10CDE00080E08093460990912B02992351F0E091C5
:10CDF000DC0BF091DD0B4685578503E023E06C2FBB
:10CE0000D9D2112309F409C180914609882309F474
:10CE100004C10E94545D8FE49CE6DF91CF911F9185
:10CE20000F91FF90EF90DF90CF90BF90AF900C9458
:10CE30003F5DD13009F581E0913009F080E08093C9
:10CE4000460990912B02992351F0E091DC0BF0916F
:10CE5000DD0B44A555A50EE72EE36C2FABD21123B5
:10CE600009F4DBC080914609882309F4D6C00E94EA
:10CE7000545D8EE092E622C0D23061F581E09230BE
:10CE800009F080E08093460990912B02992351F09C
:10CE9000E091DC0BF091DD0B46A557A50EE72EE3E4
:10CEA0006C2F88D2112309F4B8C0809146098823D9
:10CEB00009F4B3C00E94545D84E59AE9DF91CF91F3
:10CEC0001F910F91FF90EF90DF90CF90BF90AF90A8
:10CED0000C942D5DD33009F581E0933009F080E0AA
:10CEE0008093460990912B02992351F0E091DC0B3D
:10CEF000F091DD0B40A951A90EE72EE36C2F5AD219
:10CF0000112309F48AC080914609882309F485C059
:10CF10000E94545D8BE799EBD1CFD43051F581E07D
:10CF2000943009F080E08093460990912B02992378
:10CF300051F0E091DC0BF091DD0B44A955A900E222
:10CF40002EE36C2F37D2112309F467C08091460974
:10CF5000882309F462C00E94545DDF91CF911F9134
:10CF60000F91FF90EF90DF90CF90BF90AF900C9417
:10CF70004780D53041F581E0953009F080E080931D
:10CF8000460990912B02992351F0E091DC0BF0912E
:10CF9000DD0B46A957A900E22EE36C2F0BD211231B
:10CFA000E1F1809146098823C1F10E94545DDF912F
:10CFB000CF911F910F91FF90EF90DF90CF90BF9096
:10CFC000AF900C94618BD63041F581E0963009F03A
:10CFD00080E08093460990912B02992351F0E091D3
:10CFE000DC0BF091DD0B40AD51AD00E22EE36C2F78
:10CFF000E1D1112391F080914609882371F00E94BC
:10D00000545DDF91CF911F910F91FF90EF90DF90D2
:10D01000CF90BF90AF900C94758080914809873075
:10D0200050F0C0924009D0924109E0924209F0923A
:10D030004309B0924809209148098091470990E03E
:10D040000396422F50E0841795074CF48DEF820F22
:10D0500080934709A0922B02DCEFD20FCFEFCF5F76
:10D06000DF5FC43008F4B6CEDF91CF911F910F91EE
:10D07000FF90EF90DF90CF90BF90AF900895AF9268
:10D08000BF92CF92DF92EF92FF920F931F93CF93B5
:10D09000DF93109249098091400990914109A09134
:10D0A0004209B091430981309048A105B10540F093
:10D0B00010924009109241091092420910924309BE
:10D0C000809140098093480990914709891710F48D
:10D0D00080934709D091470910914B0912FB112702
:10D0E00010F9C0E084E0C82ED12CE12CF12C94E0A2
:10D0F000B92E22E0A22E90914809D1112BC081E0D7
:10D10000911180E08093460990912B02992351F070
:10D11000E091DC0BF091DD0B4489558903E023E0BD
:10D120006C2F48D1112309F402C18091460988234C
:10D1300009F4FDC00E94545D8CE497EADF91CF9121
:10D140001F910F91FF90EF90DF90CF90BF90AF9025
:10D150000C943F5DD130A9F581E0913009F080E079
:10D160008093460990912B02992351F0E091DC0BBA
:10D17000F091DD0B44AD55AD00E22EE36C2F1AD1DA
:10D18000112309F4D4C080914609882309F4CFC043
:10D190000E94545D8091E2129091E3129093A50A4F
:10D1A0008093A40A81E090E09093190C8093180C6E
:10D1B0008091E6129091E7120E9411AD89E090E013
:10D1C000A9C0D230B9F581E0923009F080E08093B7
:10D1D000460990912B02992361F0E091DC0BF091CC
:10D1E000DD0BEC5BFF4F4081518100E22EE36C2FA1
:10D1F000E1D0112309F49BC080914609882309F4EA
:10D2000096C00E94545D8091DC129091DD12909343
:10D21000A50A8093A40A81E090E09093190C809372
:10D22000180C8091E0129091E1120E9411AD87E0FC
:10D2300090E070C0D330B9F581E0933009F080E020
:10D240008093460990912B02992361F0E091DC0BC9
:10D25000F091DD0BE05CFF4F4081518100E22EE355
:10D260006C2FA8D0112309F462C08091460988234D
:10D2700009F45DC00E94545D8091E2129091E31226
:10D280009093A70A8093A60A81E090E09093190CEE
:10D290008093180C8091E6129091E7120E9411ADD4
:10D2A0008AE090E037C0D43009F041C081E094308A
:10D2B00009F080E08093460990912B02992361F058
:10D2C000E091DC0BF091DD0BE85BFF4F4081518179
:10D2D00000E22EE36C2F6ED0112349F180914609B4
:10D2E000882329F10E94545D8091DC129091DD1217
:10D2F0009093A70A8093A60A81E090E09093190C7E
:10D300008093180C8091E0129091E1120E9411AD6F
:10D3100088E090E00E943A91DF91CF911F910F91A8
:10D32000FF90EF90DF90CF90BF90AF9034C080918E
:10D330004809853050F0C0924009D0924109E092EE
:10D340004209F0924309B09248092091480980911E
:10D35000470990E00396422F50E0841795074CF45C
:10D360008DEF820F80934709A0922B02DCEFD20F42
:10D37000CFEFCF5FDF5FC43008F4BDCEDF91CF9138
:10D380001F910F91FF90EF90DF90CF90BF90AF90E3
:10D39000089508950895109240091092410910923D
:10D3A0004209109243098EE99FE69093020280930E
:10D3B00001020895EF92FF920F931F93CF93DF9393
:10D3C0001F92CDB7DEB7182F7A0180E029830E9423
:10D3D000AA7F2981112311F0822F01C080E20E94CF
:10D3E0003E5612E1F7018491882311F0111111C00A
:10D3F000112329F080E20E943E561150F9CF802F70
:10D400000F90DF91CF911F910F91FF90EF900C94AF
:10D410003E560E941F48181BFFEFEF1AFF0AE2CF8B
:10D42000AF92BF92CF92DF92EF92FF920F931F9332
:10D43000CF93DF931092490980914009909141095F
:10D44000A0914209B091430981309048A105B105EE
:10D4500040F0109240091092410910924209109236
:10D4600043098091400980934809909147098917A1
:10D4700010F480934709D091470910914B0912FB92
:10D48000112710F9C0E058E0C52ED12CE12CF12C69
:10D4900068E0B62E72E0A72E90914809D1112BC0FA
:10D4A00081E0911180E08093460990912B029923AD
:10D4B00051F0E091DC0BF091DD0B4685578503E0E0
:10D4C00023E06C2F77DF112309F4B7C1809146095F
:10D4D000882309F4B2C10E94545D8FE49CE6DF9179
:10D4E000CF911F910F91FF90EF90DF90CF90BF9061
:10D4F000AF900C943F5DD13099F581E0913009F007
:10D5000080E08093460990912B02992369F0E09185
:10D51000DC0BF091DD0BE059FF4F4081518129E296
:10D5200032E06C2F0E944956112309F486C1809184
:10D530004609882309F481C10E94545DE091DC0B07
:10D54000F091DD0BE059FF4FE12C10ECF12E09E7D3
:10D5500014E420E030E040E251E469E272E03AC1D4
:10D56000D23061F581E0923009F080E08093460985
:10D5700090912B02992369F0E091DC0BF091DD0B87
:10D58000E257FF4F4081518124EA3AE06C2F0E941C
:10D590004956112309F451C180914609882309F4A1
:10D5A0004CC10E94545DE091DC0BF091DD0BE25721
:10D5B000FF4F49EC59E664EA7AE02DC0D330C9F553
:10D5C00081E0933009F080E08093460990912B022E
:10D5D000992369F0E091DC0BF091DD0BE057FF4FF0
:10D5E0004081518126EA3AE06C2F0E94495611236E
:10D5F00009F423C180914609882309F41EC10E94C1
:10D60000545DE091DC0BF091DD0BE057FF4F4AECED
:10D6100059E666EA7AE080819181DF91CF911F918E
:10D620000F91FF90EF90DF90CF90BF90AF900C9450
:10D630006E55D43089F581E0943009F080E0809314
:10D64000460990912B02992369F0E091DC0BF0914F
:10D65000DD0BEC56FF4F408151812EEA3AE06C2FF2
:10D660000E944956112309F4E8C080914609882395
:10D6700009F4E3C00E94545DE091DC0BF091DD0BF6
:10D68000EC56FF4FE12CF12C0FE713E420E030E0E3
:10D69000A9016EEA7AE09EC0D53099F581E0953017
:10D6A00009F080E08093460990912B02992369F05C
:10D6B000E091DC0BF091DD0BE256FF4F4081518190
:10D6C00027E032E06C2F0E944956112309F4B5C0BF
:10D6D00080914609882309F4B0C00E94545DE0910E
:10D6E000DC0BF091DD0BE256FF4FE12C10ECF12E3C
:10D6F00009E714E420E030E040E251E467E072E042
:10D7000069C0D63099F581E0963009F080E08093C9
:10D71000460990912B02992369F0E091DC0BF0917E
:10D72000DD0BE056FF4F4081518123E032E06C2F4A
:10D730000E944956112309F480C08091460988232C
:10D7400009F47BC00E94545DE091DC0BF091DD0B8D
:10D75000E056FF4FE12C10ECF12E09E714E420E035
:10D7600030E040E251E463E072E034C0D730B9F514
:10D7700081E0973009F080E08093460990912B0278
:10D78000992369F0E091DC0BF091DD0BEE55FF4F32
:10D790004081518125E032E06C2F0E9449561123CF
:10D7A00009F44BC080914609882309F446C00E94C1
:10D7B000545DE091DC0BF091DD0BEE55FF4FE12C59
:10D7C00010ECF12E09E714E420E030E040E251E4EF
:10D7D00065E072E0808191810E94FD5455C0D8308F
:10D7E00061F581E0983009F080E0809346099091DE
:10D7F0002B02992361F0E091DC0BF091DD0BE257F5
:10D80000FE4F4081518100E22EE36C2FD3DD1123C6
:10D81000A1F080914609882381F00E94545D81E146
:10D8200090E0DF91CF911F910F91FF90EF90DF90EB
:10D83000CF90BF90AF900C943A9180914809893075
:10D8400050F0C0924009D0924109E0924209F09212
:10D850004309B0924809209148098091470990E016
:10D860000396422F50E0841795074CF48DEF820FFA
:10D8700080934709A0922B02DCEFD20FCFEFCF5F4E
:10D88000DF5FC43008F408CEDF91CF911F910F9174
:10D89000FF90EF90DF90CF90BF90AF900895FF92F0
:10D8A0000F931F93CF93DF93109249098091400902
:10D8B00090914109A0914209B0914309813090486B
:10D8C000A105B10540F01092400910924109109253
:10D8D0004209109243098091400980934809909130
:10D8E0004709891710F480934709D091470910918F
:10D8F0004B0912FB112710F9C0E082E0F82ED1117C
:10D9000026C081E090914809911180E080934609FA
:10D9100090912B02992351F0E091DC0BF091DD0BFB
:10D920004089518903E023E06C2F44DD112379F015
:10D9300080914609882359F00E94545D8EE99FE644
:10D94000DF91CF911F910F91FF900C943F5D8091DB
:10D95000361290913712891B8F709091480981116E
:10D960002AC020919513309196132230310519F178
:10D97000D13019F581E0913009F080E080934609BB
:10D9800090912B02992351F0E091DC0BF091DD0B8B
:10D99000448955890EE72EE36C2F0CDD112309F421
:10D9A00043C080914609882309F43EC00E94545D1B
:10D9B0008CE497EA6FC1D13009F1D230A9F581E04A
:10D9C000923009F080E08093460990912B029923D0
:10D9D00051F0E091DC0BF091DD0B468957890EE7A1
:10D9E0002EE36C2FE7DC1123F9F0809146098823A0
:10D9F000D9F00E94545D8EEA96E64CC181E09130E8
:10DA000009F080E08093460990912B02992351F010
:10DA1000E091DC0BF091DD0B428953890EE72EE398
:10DA20006C2FC8DC11112DC12091951330919613E4
:10DA3000909148092115310509F4EDC0E091931644
:10DA4000F0919416309709F497C08081882309F4E7
:10DA500093C022303105B9F5D33009F05DC081E0C3
:10DA6000933009F080E08093460990912B0299232E
:10DA700061F0E091DC0BF091DD0BE05AFF4F40814B
:10DA8000518100E22EE36C2F95DC112309F4EAC0EA
:10DA900080914609882309F4E5C00E94545D809175
:10DAA000951390919613029709F052C183E090E08C
:10DAB0009093961380939513DF91CF911F910F91BF
:10DAC000FF900C94E3B1D33039F581E0933009F045
:10DAD00080E08093460990912B02992361F0E091B8
:10DAE000DC0BF091DD0BEE59FF4F4081518100E2DC
:10DAF0002EE36C2F5FDC112309F4B4C0809146093A
:10DB0000882309F4AFC00E94545DDF91CF911F912B
:10DB10000F91FF900C94A191D43009F0A3C081E043
:10DB2000943009F080E08093460990912B0299236C
:10DB300061F0E091DC0BF091DD0BEC59FF4F40817F
:10DB4000518100E22EE36C2F35DC112309F48AC0E9
:10DB500080914609882309F485C00E94545D81E0C4
:10DB600090E090939613809395130E940A930E94DD
:10DB700087918DE090E048C0D33019F581E0933073
:10DB800009F080E08093460990912B02992361F07F
:10DB9000E091DC0BF091DD0BEA59FF4F40815181A0
:10DBA0000EE72EE36C2F06DC112309F45BC0809195
:10DBB0004609882309F456C00E94545D83E597EB1B
:10DBC00069C0D43009F04EC081E0943009F080E0A3
:10DBD0008093460990912B02992361F0E091DC0B30
:10DBE000F091DD0BE659FF4F4081518100E22EE3B9
:10DBF0006C2FE0DB1123B1F180914609882391F16C
:10DC00000E94545D8BE090E0DF91CF911F910F91C6
:10DC1000FF900C943A91D33091F481E0933009F065
:10DC200080E08093460990912B02992309F4BCCFA0
:10DC3000E091DC0BF091DD0BE25AFF4FAFCFD43017
:10DC400089F481E0943009F080E080934609909156
:10DC50002B02992379F2E091DC0BF091DD0BE8596E
:10DC6000FF4FC2CF8091361290913712891B8F706F
:10DC7000C1F48091951390919613029709F043C0D7
:10DC800010C080914609882309F4CECE0E94545DCD
:10DC900080E19AE6DF91CF911F910F91FF900C9454
:10DCA0002D5D85E090914809981798F0482F50E035
:10DCB00041505109052E000C660B770B409340092B
:10DCC00050934109609342097093430981508093B6
:10DCD0004809209148098091470990E00396422F16
:10DCE00050E0841795074CF48DEF820F809347091D
:10DCF000F0922B02DCEFD20FCFEFCF5FDF5FC430AB
:10DD000008F4FDCD25C0D530C1F481E090914809DB
:10DD1000953009F080E08093460990912B02992379
:10DD200051F0E091DC0BF091DD0B408D518D0EE751
:10DD30002EE36C2F3FDB111102C086E0B3CF809140
:10DD400046098823D1F30E94545D81E291E6A2CF77
:10DD5000DF91CF911F910F91FF9008950F931F9323
:10DD6000CF93DF938C0190E0C0E0D1E0D90FF801B0
:10DD7000E90FF11D8081882329F00E941F48C80FF8
:10DD80009D2FF3CF8C2FDF91CF911F910F9108958D
:10DD9000EF92FF920F931F93CF93DF931F92CDB714
:10DDA000DEB7F82E8B0161E081E099830E94AA7FA3
:10DDB000EF2D9981F92F84917F019FEFE91AF90ADC
:10DDC000882321F00E941F48F701F5CF01151105A6
:10DDD000B1F08AE30E943E56F80101900020E9F775
:10DDE000802F8E1B61E08C5E0E94AA7FC8010F907D
:10DDF000DF91CF911F910F91FF90EF90AFCF0F90D8
:10DE0000DF91CF911F910F91FF90EF900895CF93E5
:10DE1000DF93CDB7DEB7C054D1090FB6F894DEBF9B
:10DE20000FBECDBF44E064E189EF96E10E94FB7E26
:10DE300088E0E8ECF3E0DE01D99601900D928A9536
:10DE4000E1F788E0E0EDF3E0DE01D19601900D927C
:10DE50008A95E1F788E0E8EDF3E0DE01999601901C
:10DE60000D928A95E1F788E0E0EEF3E0DE0191960D
:10DE700001900D928A95E1F788E0E8EEF3E0DE018B
:10DE8000599601900D928A95E1F788E0E0EFF3E072
:10DE9000DE01519601900D928A95E1F788E0E8EF56
:10DEA000F3E0DE01199601900D928A95E1F788E082
:10DEB000E0E0F4E0DE01119601900D928A95E1F721
:10DEC000BE01675E7F4F80E00E94CD7EBE016F5C29
:10DED0007F4F81E00E94CD7EBE01675D7F4F82E073
:10DEE0000E94CD7EBE016F5D7F4F83E00E94CD7E9C
:10DEF000BE01675C7F4F84E00E94CD7EBE016F5EF5
:10DF00007F4F85E00E94CD7EBE01675F7F4F86E038
:10DF10000E94CD7EBE016F5F7F4F87E00E94CD7E65
:10DF200089EF96E10E944D9AC05CDF4F0FB6F894DE
:10DF3000DEBF0FBECDBFDF91CF910895CF92DF92AC
:10DF4000EF92FF920F931F93CF93DF938091090A73
:10DF5000882321F081508093090A03C081E08093D7
:10DF60002B0280912B02882309F496C160E080E0A7
:10DF70000E94AA7F6091A40A7091A50A072E000C46
:10DF8000880B990B0E9472D39F938F937F936F930B
:10DF900080919F0A8F9380919E0A8F9380919D0A12
:10DFA0008F9380919C0A8F936091A60A7091A70A23
:10DFB000072E000C880B990B0E9472D39F938F93AE
:10DFC0007F936F938091A30A8F938091A20A8F937E
:10DFD0008091A10A8F938091A00A8F938EE691E1A0
:10DFE0009F938F930E94115AB9DE61E080E00E94F6
:10DFF000AA7F8DB79EB742960FB6F8949EBF0FBE0C
:10E000008DBF8091710A882349F08091720A88231C
:10E0100029F08091730A811110924A0940914A09AE
:10E0200030916C0A20916B0A90916A0A8091690A7A
:10E03000442381F14091170C442361F13F932F93C6
:10E040009F938F936091650A7091660A8091670A29
:10E050009091680A0E9441D87F936F936091610A02
:10E060007091620A8091630A9091640A0E9441D87B
:10E070007F936F9387E591E19F938F930E94115A4D
:10E080006DDE8DB79EB70A960FB6F8949EBF0FBE91
:10E090008DBF2BC03F932F939F938F936091650A01
:10E0A0007091660A8091670A9091680A0E9441D82F
:10E0B0007F936F936091610A7091620A8091630A05
:10E0C0009091640A0E9441D87F936F9383E491E119
:10E0D0009F938F930E94115A41DE8DB79EB70A9687
:10E0E0000FB6F8949EBF0FBE8DBF62E080E00E9425
:10E0F000AA7F8091951390919613029709F059C0C9
:10E100008AE09CE00E94D0492CE330E0B9010E94F3
:10E1100071DACB01B9010E9471DAEB01182F092FD6
:10E12000E0919316F0919416309731F120812223DB
:10E1300021F18091D0169091D116A091D216B09174
:10E14000D3160097A105B105B9F0BC01CD016D59F9
:10E150007F4F8F4F9F4F24E630E040E050E00E9419
:10E16000ABD66091D8167091D9168091DA1690913D
:10E17000DB160E94ABD601C020E00F931F93DF9304
:10E18000CF931F922F9380912A028F93809129021F
:10E190008F938AE291E19F938F930E94115ADEDD63
:10E1A0008DB79EB70A960FB6F8949EBF0FBE8DBF6F
:10E1B00011C080912A028F93809129028F9383E16D
:10E1C00091E19F938F930E94115AC8DD0F900F9099
:10E1D0000F900F9063E080E00E94AA7F0091070AF1
:10E1E0001091080AC091180CD091190C0C171D073A
:10E1F00009F44CC00E94E1C2C090060CD090070CFC
:10E20000E090080CF090090CC616D706E806F9064F
:10E21000E8F5C330D10501F16CF4E091DC0BF0912D
:10E22000DD0BC130D105A9F0C230D10519F58085CB
:10E23000918526C0C430D105B1F0CE010697029772
:10E24000C8F486E090E09093190C8093180CE801D4
:10E2500019C08681978114C0E091DC0BF091DD0B31
:10E26000828593850DC0E091DC0BF091DD0B8281FE
:10E27000938106C0E091DC0BF091DD0B84819581E8
:10E280000E94695CD093080AC093070A82E29AE070
:10E2900065DD8AE08093090A80914B0982FF11C0F5
:10E2A0008FE49CE690930202809301021092400951
:10E2B0001092410910924209109243090E94545D44
:10E2C000A6DD2091290230912A0280914009909187
:10E2D00041092436310534F4820F931F85369105A8
:10E2E0004CF416C02436310599F0820F931F843602
:10E2F000910574F41092400910924109109242095C
:10E300001092430984E690E090932A0280932902B8
:10E310002091290230912A0280914009909141096F
:10E320002436310569F4833091051CF08E599F4FD6
:10E3300009C08E3F2FEF92078CF48A599F4F02C07D
:10E34000820F931F90932A02809329021092400912
:10E3500010924109109242091092430980912902BA
:10E3600090912A020A9734F48AE090E090932A026E
:10E37000809329028091290290912A02883E93403D
:10E3800034F087EE93E090932A0280932902DF9184
:10E39000CF911F910F91FF90EF90DF90CF90089554
:10E3A0002F923F924F925F926F927F928F929F92A5
:10E3B000AF92BF92CF92DF92EF92FF920F931F9393
:10E3C000CF93DF93CDB7DEB7C557D1090FB6F89419
:10E3D000DEBF0FBECDBF3C014B015A01E4963FAFFB
:10E3E0002EAFE4972C96EFAE2C972D96FFAE2D977F
:10E3F0002E960FAF2E972F961FAF2F97A696DFAEB4
:10E40000CEAEA697809136128F5F68968FAF6897D1
:10E41000803119F468961FAE689768962FAD68979B
:10E42000022F220F110B8091371290E08017910775
:10E4300019F40E94B3B3F7CF20913C1230913D12F2
:10E4400040913E1250913F12D3016D917D918D917B
:10E450009C910E9485CE0E94DAD96C966CAF7DAFFC
:10E460008EAF9FAF6C972091401230914112409136
:10E47000421250914312F401608171818281938133
:10E480000E9485CE0E94DAD9A0966CAF7DAF8EAF88
:10E490009FAFA097209144123091451240914612AF
:10E4A00050914712D5016D917D918D919C910E9463
:10E4B00085CE0E94DAD9A4966CAF7DAF8EAF9FAFA8
:10E4C000A497209148123091491240914A125091DC
:10E4D0004B12E496EEADFFADE497608171818281CD
:10E4E00093810E9485CE0E94DAD92B966CAF7DAFC6
:10E4F0008EAF9FAF2B978091AE0C9091AF0CA091F7
:10E50000B00CB091B10C2B962CAD3DAD4EAD5FADC6
:10E510002B97281739074A075B0709F485C083E062
:10E5200090E09093190C8093180CE091210A34E04C
:10E53000E39FF0011124E656F54F20E030E040E281
:10E5400053E462817381848195810E946CD387FF3B
:10E550001AC02B964CAD5DAD6EAD7FAD2B97409341
:10E56000AE0C5093AF0C6093B00C7093B10CE09173
:10E57000DC0BF091DD0BE858FE4F608171818AED74
:10E580009BE00E94AE2A8091AE0C9091AF0CA091BE
:10E59000B00CB091B10C2B962CAD3DAD4EAD5FAD36
:10E5A0002B97281B390B4A0B5B0BCA01B90157FF8C
:10E5B00007C090958095709561957F4F8F4F9F4FC5
:10E5C0000E9472D36B017C0120E030E049EB53E400
:10E5D000609148127091491280914A1290914B12A9
:10E5E0000E9485CE9B01AC01C701B6010E942DD9C6
:10E5F0001816D4F42B964CAD5DAD6EAD7FAD2B9758
:10E600004093AE0C5093AF0C6093B00C7093B10C70
:10E61000E091DC0BF091DD0BE658FE4F60817181DB
:10E620008AED9BE00E94AE2AE09136122E2E312C0C
:10E6300057E5E59FF0011124E056F34FDF01A458A0
:10E64000BF4F1C926091A20C7091A30C8091A40CFE
:10E650009091A50C6BA37CA38DA39EA36C968CAD0F
:10E660009DADAEADBFAD6C972BA13CA14DA15EA100
:10E67000821B930BA40BB50BB7FF07C0B095A095F9
:10E68000909581959F4FAF4FBF4F86A397A3A0A7AB
:10E69000B1A74091A60C5091A70C6091A80C709165
:10E6A000A90C4FA358A769A77AA787E5829DF00117
:10E6B000839DF00D1124E056F34FA0968CAD9DADD7
:10E6C000AEADBFADA097841B950BA60BB70BB7FFE4
:10E6D00007C0B095A095909581959F4FAF4FBF4FC4
:10E6E00082A793A7A4A7B5A76091AA0C7091AB0CC1
:10E6F0008091AC0C9091AD0C6BA77CA78DA79EA7C9
:10E7000087E5829DF001839DF00D1124E056F34FC3
:10E71000A4968CAD9DADAEADBFADA4972BA53CA589
:10E720004DA55EA5821B930BA40BB50BB7FF07C0CD
:10E73000B095A095909581959F4FAF4FBF4F86A7FD
:10E7400097A7A0ABB1ABC090AE0CD090AF0CE0904F
:10E75000B00CF090B10C2B966CAD7DAD8EAD9FAD35
:10E760002B976C197D098E099F0997FF07C090951B
:10E770008095709561957F4F8F4F9F4F0E9472D308
:10E78000E091210A34E0E39FF0011124E75FFD4F9F
:10E7900020813181428153810E9485CE0E9441D8DF
:10E7A0009B01AC01A0910702B09108020E94BCDA63
:10E7B00024E630E040E050E00E9498DAB90187E5B5
:10E7C000829DF001839DF00D1124E056F34F22ABA2
:10E7D00073AB44AB55AB06A117A120A531A582A40C
:10E7E00093A4A4A4B5A446A457A460A871A8CB017F
:10E7F000DA0184159505A605B70514F4D301C20105
:10E80000B901A80188159905AA05BB0544F00817A8
:10E8100019072A073B0754F4AC01BD0107C00815CE
:10E8200019052A053B0514F4B501A40187E5829D6D
:10E83000F001839DF00D1124E056F34F46AB57AB2A
:10E8400060AF71AF463051056105710510F40C944D
:10E85000B37EDF01A858BF4F8091AE0A9091AF0AF6
:10E86000AC01990F660B770B4D935D936D937C9381
:10E870001397EA5BFF4F6C964CAD5DAD6EAD7FAD0F
:10E880006C978BA19CA1ADA1BEA1481759076A073F
:10E890007B0714F0108202C081E08083A0964CAD0B
:10E8A0005DAD6EAD7FADA0978FA198A5A9A5BAA5C6
:10E8B000481759076A077B075CF487E5829DF001DA
:10E8C000839DF00D1124EA51F34F80818260808393
:10E8D000A4964CAD5DAD6EAD7FADA4978BA59CA508
:10E8E000ADA5BEA5481759076A077B075CF487E505
:10E8F000829DF001839DF00D1124EA51F34F808138
:10E90000846080832B964CAD5DAD6EAD7FAD2B9753
:10E910004C155D056E057F055CF487E5829DF00171
:10E92000839DF00D1124EA51F34F8081886080832C
:10E93000A696AEADBFADA6974C9157E5529DC001CE
:10E94000539D900D11248056934FFC01E95BFF4FBE
:10E950004083319610821182128213823496108283
:10E96000118212821382EC91F0E0EE0FFF1FE85249
:10E97000FD4E40815181FC01E05BFF4F518340839C
:10E98000012B022B032B09F05F9887E5829DF00194
:10E99000839DF00D1124E056F34F82A593A5A4A505
:10E9A000B5A5892B8A2B8B2B09F08A9887E5829D48
:10E9B000F001839DF00D1124E056F34F86A597A535
:10E9C000A0A9B1A9892B8A2B8B2B41F09FB7F89472
:10E9D000809108018D7F809308019FBF87E5829D0C
:10E9E000F001839DF00D1124E056F34F82A993A905
:10E9F000A4A9B5A9892B8A2B8B2B11F012984798C3
:10EA000087E5829DF001839DF00D1124E056F34FC0
:10EA100022A933A944A955A92BAF3CAF4DAF5EAF96
:10EA2000232B242B252B49F4E0907C12F0907D12AF
:10EA300000917E1210917F1208C0E0905C12F0905D
:10EA40005D1200915E1210915F129701A8012C9641
:10EA50006FAD2C972D967FAD2D972E968FAD2E975F
:10EA60002F969FAD2F970E946CD387FF0CC02C96DA
:10EA7000EFAE2C972D96FFAE2D972E960FAF2E97BB
:10EA80002F961FAF2F978091A20C9091A30CA0916D
:10EA9000A40CB091A50C6C962CAD3DAD4EAD5FAD08
:10EAA0006C97281B390B4A0B5B0BCA01B9010E94FA
:10EAB00072D320913C1230913D1240913E12509100
:10EAC0003F120E94D0D72B013C01698B7A8B8B8B34
:10EAD0009C8B8091A60C9091A70CA091A80CB09152
:10EAE000A90CA0962CAD3DAD4EAD5FADA097281BF7
:10EAF000390B4A0B5B0BCA01B9010E9472D32091FA
:10EB000040123091411240914212509143120E94A2
:10EB1000D0D74B015C016D8B7E8B8F8B988F809152
:10EB2000AA0C9091AB0CA091AC0CB091AD0CA4963A
:10EB30002CAD3DAD4EAD5FADA497281B390B4A0BF4
:10EB40005B0BCA01B9010E9472D32091441230912B
:10EB5000451240914612509147120E94D0D76B0146
:10EB60007C01698F7A8F8B8F9C8F8091AE0C9091F6
:10EB7000AF0CA091B00CB091B10C2B962CAD3DAD6B
:10EB80004EAD5FAD2B97281B390B4A0B5B0BCA01AF
:10EB9000B9010E9472D320914812309149124091DC
:10EBA0004A1250914B120E94D0D7E091210A34E0D2
:10EBB000E39FF0011124E75FFD4F20813181428105
:10EBC00053810E9485CE6BA37CA38DA39EA36091ED
:10EBD000070270910802072E000C880B990B0E9407
:10EBE00072D39B01AC016BA17CA18DA19EA10E945F
:10EBF00085CE20E030E048EC52E40E94D0D76D8F03
:10EC00007E8F8F8F98A327E5229DF001239DF00D25
:10EC10001124E056F34F26A137A140A551A52BABF7
:10EC20003CAB4DAB5EAB2630310541055105E4F4FC
:10EC300002A513A524A535A506301105210531052A
:10EC40009CF406A517A520A931A9063011052105B8
:10EC5000310554F4E25AFF4FDC01CB01BF778083CA
:10EC60009183A283B3832AC0C301B2010E9482CEE2
:10EC70002B013C01C501B4010E9482CE9B01AC0175
:10EC8000C301B2010E94E7D64B015C01C701B60186
:10EC90000E9482CE9B01AC01C501B4010E94E7D65F
:10ECA0000E9418DA27E5229DF001239DF00D112422
:10ECB000E250F34F608371838283938387E5829D63
:10ECC000F001839DF00D1124E250F34F40815181FA
:10ECD0006281738123964CAF5DAF6EAF7FAF239798
:10ECE0009A01AB0160E070E080E89FE30E94D0D71A
:10ECF0009B01AC012C966FAD2C972D967FAD2D9777
:10ED00002E968FAD2E972F969FAD2F970E9485CE72
:10ED10004B015C018091361290E020913712821BEA
:10ED20009109BC016F70772778AF6FABA501940193
:10ED300060E074E284E799E40E94D0D70E94DAD9B7
:10ED40006B017C018FA998AD823091050CF441C014
:10ED50002C01990F66087708C301B2010E9472D393
:10ED600020E030E040E051E40E946CD387FF31C0E6
:10ED70008091F8129091F912A091FA12B091FB12C1
:10ED8000C816D906EA06FB0620F58C199D09AE09BE
:10ED9000BF09BC01CD01660F771F881F991FA30112
:10EDA00092010E94ABD6CA01B9010E9470D30E94A1
:10EDB000DAD96C0D7D1D8E1D9F1D0E9470D39B01A5
:10EDC000AC0160E074E284E799E40E94D0D74B0183
:10EDD0005C0187E5829D8001839D100D1124005602
:10EDE000134FF801EE5AFF4F2C968FAD2C972D96AE
:10EDF0009FAD2D972E96AFAD2E972F96BFAD2F9727
:10EE000080839183A283B383D801D6966D917D913F
:10EE10008D919C91D9970E9470D36BA37CA38DA3F5
:10EE20009EA3A50194010E9485CE0E94B9D70E949D
:10EE300047D827966CAF7DAF8EAF9FAF2797F8016D
:10EE4000E859FF4F6083718382839383FE0171963B
:10EE5000FAAFE9AF9E012F5F3F4F3AAB29AB4CE4CD
:10EE600052E165965FAF4EAF6597BE016F5D7F4F14
:10EE70007AA369A361963FAF2EAF61971FA21BA62D
:10EE800070E87FA78FE388ABA9ADBAAD6D917D9196
:10EE90008D919D91BAAFA9AFA50194010E9485CE35
:10EEA0006196EEADFFAD61976193719381939193FC
:10EEB0006196FFAFEEAF61976B017C01E894F7F8C4
:10EEC0006596AEADBFAD65974D905D906D907D90B0
:10EED0006596BFAFAEAF6597A3019201C701B601BA
:10EEE0000E942DD91816B4F4A7019601C301B201EE
:10EEF0000E94D0D77B018C019B01AC016FA17BA547
:10EF00008FA598A90E946CD387FD04C0EFA2FBA631
:10EF10000FA718ABE9ADFAAD29A13AA1E217F307A3
:10EF200009F0B2CF20E030E040E85FE36FA17BA5BD
:10EF30008FA598A90E946CD387FF55C08E010F5EE4
:10EF40001F4F2FA13BA54FA558A9A9A9BAA96D91FB
:10EF50007D918D919C910E9485CEE9A9FAA961933A
:10EF6000719381939193FAABE9ABE017F10749F7FD
:10EF700087E5829D8001839D100D11240056134F5B
:10EF80007801F2E5EF0EF11C2FA13BA54FA558A982
:10EF90002C966FAD2C972D967FAD2D972E968FAD1D
:10EFA0002E972F969FAD2F970E9485CED7016D93F8
:10EFB0007D938D939C93139708591F4F27966CADA3
:10EFC0007DAD8EAD9FAD27970E9470D32FA13BA53D
:10EFD0004FA558A90E9485CE0E9447D8F8016083AA
:10EFE00071838283938323962CAD3DAD4EAD5FAD8F
:10EFF00023976BA17CA18DA19EA10E94D0D76B010C
:10F000007C012BA93CA94DA95EA9232B242B252BE0
:10F0100091F587E5829D8001839D100D1124005696
:10F02000134FF80182A593A5A4A5B5A5892B8A2B1A
:10F030008B2B09F586A597A5A0A9B1A9892B8A2BA9
:10F040008B2BC9F4209164123091651240916612A5
:10F0500050916712C701B6010E9485CE0E94B9D7B0
:10F060000C581F4F0E9447D8D8016D937D938D9304
:10F070009C9313972EC120916012309161124091A0
:10F08000621250916312C701B6010E9485CE0E94A0
:10F09000B9D70E9447D827E5229D8001239D100DF6
:10F0A00011240C5E124FF801608371838283938375
:10F0B0008090FC129090FD12A090FE12B090FF1272
:10F0C0000E9470D32B013C016BA97CA98DA99EA93C
:10F0D0000E9472D39B01AC01C301B2010E9485CE94
:10F0E0002BA13CA14DA15EA10E94D0D72B013C01D8
:10F0F000C501B4010E9470D39B01AC01C301B201F0
:10F100000E942DD9181634F4D8018D929D92AD929B
:10F11000BC9213978090001390900113A09002135B
:10F12000B090031327E5229DC001239D900D11246B
:10F130009C012056334F89010C581F4FF801608104
:10F14000718182819381E5962FAFE597E6963FAF77
:10F15000E6970E9470D32B013C01E5962FADE59711
:10F16000E6963FADE697D9019A966D917D918D9186
:10F170009C919D970E9472D39B01AC01C301B20187
:10F180000E9485CE2BA13CA14DA15EA10E94D0D7AB
:10F190002B013C01C501B4010E9470D39B01AC015D
:10F1A000C301B2010E942DD918162CF4F8018082F7
:10F1B0009182A282B3828090081390900913A0904C
:10F1C0000A13B0900B1387E5829D8001839D100D7B
:10F1D00011240C5E124FD8016D917D918D919C91FF
:10F1E0000E9470D32B013C016BAD7CAD8DAD9EAD0B
:10F1F0000E9472D39B01AC01C301B2010E9485CE73
:10F200002BA13CA14DA15EA10E94D0D72B013C01B6
:10F21000C501B4010E9470D39B01AC01C301B201CE
:10F220000E942DD918162CF4F80180829182A282B6
:10F23000B3828090041390900513A0900613B090B1
:10F24000071327E5229DC001239D900D11249C01E9
:10F250002056334F89010C581F4FD8016D917D9175
:10F260008D919C91E5962FAFE597E6963FAFE69797
:10F270000E9470D32B013C01E5962FADE597E696F1
:10F280003FADE697F90166A577A580A991A90E94EF
:10F2900072D39B01AC01C301B2010E9485CE2BA1A8
:10F2A0003CA14DA15EA10E94D0D72B013C01C5011C
:10F2B000B4010E9470D39B01AC01C301B2010E9452
:10F2C0002DD9181634F4D8018D929D92AD92BC922E
:10F2D000139787E5829D8001839D100D11240056B0
:10F2E000134FF801EC58FF4F608171818281938147
:10F2F0000E9470D34B015C01A70196010E94D0D7F8
:10F30000AA966CAF7DAF8EAF9FAFAA97F801EE596A
:10F31000FF4F60837183828393830E5B1F4F2DEBBE
:10F3200037E346E051E4C501B4010E9485CE0E9456
:10F3300041D8F8016083718382839383C0906C12FB
:10F34000D0906D12E0906E12F0906F1220E030E0DD
:10F3500040E05FE3C701B6010E9485CE6BA37FA3A7
:10F360008BA79FA729853A854B855C85AE962CAFE8
:10F370003DAF4EAF5FAFAE97409174125091751292
:10F38000609176127091771263964CAF5DAF6EAF5D
:10F390007FAF639720E030E040E05FE363966CADC1
:10F3A0007DAD8EAD9FAD63970E9485CE5B018C01D4
:10F3B000AE966CAD7DAD8EAD9FADAE979F7795014E
:10F3C000A8010E942DD9181674F49501A8016BA10B
:10F3D0007FA18BA59FA50E946CD387FD04C0ABA223
:10F3E000BFA20BA71FA76D857E858F859889E296A2
:10F3F0006CAF7DAF8EAF9FAFE29780917812909106
:10F400007912A0917A12B0917B1267968CAF9DAF62
:10F41000AEAFBFAF679720E030E040E05FE3BC01F4
:10F42000CD010E9485CE5B018C01E2966CAD7DAD75
:10F430008EAD9FADE2979F779501A8010E942DD9CF
:10F44000181674F49501A8016BA17FA18BA59FA547
:10F450000E946CD387FD04C0ABA2BFA20BA71FA75D
:10F4600087E5829DF001839DF00D1124EE50F34F4E
:10F47000908199AFA181ABAFB281BFAF23812496B8
:10F480002FAF2497292F3A2F4B2F24965FAD249727
:10F490006BA17FA18BA59FA50E946CD387FD0AC09D
:10F4A00039AD3BA34BAD4FA35FAD5BA724966FADCA
:10F4B00024976FA78FA998AD02970CF4EBC0909199
:10F4C000C20C98ABA091C30CA9ABB091C40CBBAB60
:10F4D000E091C50CEFAB27E137EB41ED58E3692F25
:10F4E0007A2F8B2F9E2F0E942DD918160CF0DBC07F
:10F4F0002091B20C3091B30C4091B40C5091B50CEA
:10F5000069817A818B819C810E94E6D62B013C0126
:10F510002091B60C3091B70C4091B80C5091B90CB9
:10F520006D817E818F8198850E94E6D64B015C01BA
:10F53000A3019201C301B2010E9485CE2B013C01BF
:10F54000A5019401C501B4010E9485CE9B01AC01C7
:10F55000C301B2010E94E7D60E9418DA4B015C0198
:10F56000A70196010E942DD918164CF4A50194010B
:10F57000C701B6010E94D0D77B018C0104C0E12CE9
:10F58000F12C00E81FE32091BA0C3091BB0C4091A4
:10F59000BC0C5091BD0CAE966CAD7DAD8EAD9FADEB
:10F5A000AE970E94E6D64B015C01E894B7F86396EB
:10F5B0002CAD3DAD4EAD5FAD6397C501B4010E946A
:10F5C0002DD91816B4F4A501940163966CAD7DADE8
:10F5D0008EAD9FAD63970E94D0D75B016C019B01FC
:10F5E000AC01B701C8010E946CD387FD02C0750150
:10F5F00086012091BE0C3091BF0C4091C00C5091FF
:10F60000C10CE2966CAD7DAD8EAD9FADE2970E94D0
:10F61000E6D64B015C01E894B7F867962CAD3DAD9A
:10F620004EAD5FAD6797C501B4010E942DD9181684
:10F63000B4F4A501940167966CAD7DAD8EAD9FAD20
:10F6400067970E94D0D75B016C019B01AC01B701A9
:10F65000C8010E946CD387FD02C075018601970125
:10F66000A80169AD7BAD8FAD24969FAD24970E9414
:10F6700085CE7B018C019B01AC0168A979A98BA97E
:10F680009FA90E946CD387FD16C0E8AAF9AA0BAB0C
:10F690001FAB11C0FBA1F8AB2FA129AB3BA53BAB26
:10F6A0004FA54FAB08C05BA158AB6FA169AB7BA561
:10F6B0007BAB8FA58FAB87E5829DF001839DF00D1D
:10F6C0001124E056F34FDF01A65ABF4F48A959A9AC
:10F6D0006BA97FA94D935D936D937C93139786A13E
:10F6E00097A1A0A5B1A5181619061A061B0654F075
:10F6F00082A593A5A4A5B5A5181619061A061B067A
:10F700000CF058C0A696AEADBFADA697EC91B4E094
:10F71000EB9FF0011124E053FD4EC080D180E280C8
:10F72000F38020E030E0A9016D8D7E8D8F8D98A152
:10F730000E942DD91816F4F5A70196012C966FADED
:10F740002C972D967FAD2D972E968FAD2E972F96B9
:10F750009FAD2F970E9485CE9F770E9441D833E0BE
:10F76000759567953A95E1F743E0660F771F4A95DF
:10F77000E1F78B01072E000C220B330B47E5429D6E
:10F78000C001439D900D11248056934FFC01E85B0E
:10F79000FF4F008311832283338344275527461B61
:10F7A000570B052E000C660B770B34964083518364
:10F7B00062837383E496EEADFFADE497808191811F
:10F7C000A281B38180930A0A90930B0AA0930C0A3A
:10F7D000B0930D0AAA966CAD7DAD8EAD9FADAA9784
:10F7E00090589B01AC010E94E7D627E5229DF001CD
:10F7F000239DF00D1124E250F34F2081318142818D
:10F8000053810E9485CE9B01AC016BE077ED83E2D2
:10F810009BE30E94E6D60E9418DA5B016C019B0113
:10F82000AC0168A979A98BA99FA90E946CD387FD17
:10F8300003C07501360104C0E8A8F9A86BA87FA829
:10F8400087E5829D8001839D100D11240056134F82
:10F85000F801EA5AFF4FC701D30180839183A28345
:10F86000B3839501A60169AD7BAD8FAD24969FADA5
:10F8700024970E946CD3F801E959FF4F18161CF029
:10F8800081E0808301C0108287E5829D6001839DB5
:10F89000D00C1124F601EA5FF24F81E0808380E111
:10F8A000FE013196A2EBBCE001900D928A95E1F742
:10F8B00089AD9BADAFAD2496BFAD24978093C20CAC
:10F8C0009093C30CA093C40CB093C50C9C01AD01E4
:10F8D0006BA17FA18BA59FA50E94D0D74B015C0196
:10F8E00029AD3BAD4FAD24965FAD2497B701C30161
:10F8F0000E94D0D7AB01BC0195018401C6018A5397
:10F90000934F0E94FAB16896FFAD6897F093361254
:10F910006C962CAD3DAD4EAD5FAD6C972093A20CB7
:10F920003093A30C4093A40C5093A50CA0964CAD1F
:10F930005DAD6EAD7FADA0974093A60C5093A70C24
:10F940006093A80C7093A90CA4966CAD7DAD8EADA0
:10F950009FADA4976093AA0C7093AB0C8093AC0CF2
:10F960009093AD0C2B968CAD9DADAEADBFAD2B97EE
:10F970008093AE0C9093AF0CA093B00CB093B10CED
:10F980008FB7F894609037128FBF20913612822F74
:10F9900090E0861991098F70992704974CF4109183
:10F9A0003712F12C00E080E090E027E5E22E11C153
:10F9B00023502F70F22EA12CB12C00E010E097E51F
:10F9C000492E55245394F61451F38F2DF11001C094
:10F9D00080E1FF24FA94F80E4F9C90011124D90184
:10F9E000AA53B34FBCA3ABA30115110509F4DCC0A6
:10F9F000F80182A193A1A4A1B5A1181619061A06AF
:10FA00001B060CF05AC042A153A164A175A1F901D3
:10FA1000E451F34F80819181A281B381B095A0958B
:10FA2000909581959F4FAF4FBF4F84179507A607BD
:10FA3000B7071CF520813181428153812FA338A75C
:10FA400049A75AA7D80192964D915D916D917C91ED
:10FA500095978FA198A5A9A5BAA5480F591F6A1F08
:10FA60007B1FD80192964D935D936D937C939597F0
:10FA7000108211821282138220C0D80192962D9199
:10FA80003D914D915C9195972FA338A749A75AA70F
:10FA900040815181628173818FA198A5A9A5BAA5E2
:10FAA000840F951FA61FB71F80839183A283B38302
:10FAB000F80112A213A214A215A2A114B10409F410
:10FAC00073C0D801D4967C90D497D596CC90D59716
:10FAD000D696DC90D697D796EC90D797272D3C2DCD
:10FAE0004D2D5E2DD0966D917D918D919C91D397EA
:10FAF0000E946CD3882309F457C0F801EF5BFF4FD5
:10FB00008081811144C0F50180A891A8A2A8B3A862
:10FB1000A5019401672D7C2D8D2D9E2D0E942DD940
:10FB20001816ACF5A5019401C501B4010E9485CE5B
:10FB30004B015C01F80184AD95ADA6ADB7ADBC013C
:10FB4000CD0190589B01AC010E94E7D6D801D89610
:10FB50002D913D914D915C91DB970E9485CE9B014B
:10FB6000AC01C501B4010E94E6D60E9418DA1B015F
:10FB70005C019B01AC01672D7C2D8D2D9E2D0E947B
:10FB80006CD387FD04C0722CC32CDA2CEB2C872D90
:10FB90009C2DAD2DBE2DF80180AB91ABA2ABB3ABCC
:10FBA000F801E05CFF4F508258010BA11CA10BCF64
:10FBB000E19E90011124A9014A53534F6A01009715
:10FBC00069F41F5F103109F410E08F2D902FFC2C89
:10FBD0000D2D209136121213EBCF0BC0FC01EF5B01
:10FBE000FF4F20812111EDCF6F2D702F0E945E4FAE
:10FBF000E8CF009751F0FC01EF5BFF4F208121110E
:10FC000004C06F2D702F0E945E4FD0903712E12CF0
:10FC1000F12C87E5C82E2D2D0D2C000C330B809177
:10FC2000361290E02817390709F44CC0C29EC00173
:10FC3000C39E900D1124BC016A53734F1B01E11444
:10FC4000F104C9F1D701A05CBF4FBCA3ABA34C9199
:10FC5000411106C0FC01EA5FF24F8081882359F10F
:10FC6000F70144A455A466A477A4C29EF001C39EE4
:10FC7000F00D1124EA50F34FA301920160817181CC
:10FC8000828193810E94D0D74B015C01A301920134
:10FC9000D701D0966D917D918D919C91D3970E94C3
:10FCA000D0D7AB01BC0195018401C7010E94FAB114
:10FCB000EBA1FCA11082D394F0E1DF1201C0D12CA2
:10FCC0007101A9CFE114F10429F1D7019C968D901F
:10FCD0009D90AD90BC909F97A50194016DEC7CEC3C
:10FCE0008CE49DE30E94D0D72B013C01A501940137
:10FCF000F70160A971A982A993A90E94D0D7AB018D
:10FD0000BC0193018201C7010E94FAB1F701E05CD6
:10FD1000FF4F10828091710082608093710080E6B5
:10FD20009AEEA0E0B0E08093E60B9093E70BA093EF
:10FD3000E80BB093E90B0E94E1C20091E60B109131
:10FD4000E70B2091E80B3091E90BDC01CB01800F30
:10FD5000911FA21FB31F8093FA0B9093FB0BA093EC
:10FD6000FC0BB093FD0BCB58DF4F0FB6F894DEBF02
:10FD70000FBECDBFDF91CF911F910F91FF90EF90FC
:10FD8000DF90CF90BF90AF909F908F907F906F90BB
:10FD90005F904F903F902F900895EF92FF920F93B6
:10FDA0001F93CF93DF931F92CDB7DEB7162F8770C7
:10FDB00028E0829FC0011124682F606489EF96E1DA
:10FDC00079830E94449AE12E7981F72E8701085F9A
:10FDD0001F4FF70161917F0189EF96E10E943F9AE1
:10FDE000E016F106B1F70F90DF91CF911F910F91BF
:10FDF000FF90EF900895EF92FF920F931F93CF9390
:10FE0000DF93EC01423018F08F8588608F874B8B31
:10FE10001C8A80E48D8B6E8B70E0605C7F4F6F8BF3
:10FE200061E08C810E9418578D818F3F19F061E04D
:10FE30000E94185761E08E810E9418577E0187E06A
:10FE4000E80EF11C00E010E08F8584FD03C084E023
:10FE500090E002C088E090E0081719074CF461E0D8
:10FE6000F70181917F010E9418570F5F1F4FECCF60
:10FE70008BE39DE00197F1F760E08C810E94E956E9
:10FE800060E08E810E94E9568D818F3F19F060E01D
:10FE90000E94E9566F8564FD1DC063E0CE010E949B
:10FEA000C3990BE416E4C8010197F1F763E0CE01B2
:10FEB0000E94C399C8010197F1F763E0CE010E9447
:10FEC000C39983E592E00197F1F762E0CE010E94C9
:10FED000C39916C06062CE010E94449A8BE496E4F6
:10FEE0000197F1F76F856062CE010E94449A83E525
:10FEF00092E00197F1F76F856062CE010E94449A0B
:10FF00006F856062CE010E94449A84E0888BCE01A6
:10FF10000E94469ACE010E944D9A82E0898B66E04B
:10FF2000CE01DF91CF911F910F91FF90EF900C9434
:10FF3000449A009761F0FC0101900020E9F73197A5
:10FF4000AF01481B590BBC0189EF96E1B6C280E0B6
:10FF500090E00895643008F063E090910C17691701
:10FF600010F06FEF690FE62FF0E0E750F94E94893B
:10FF7000682F690F606889EF96E10C94449ACF93DB
:10FF8000DF93C8EED2E169917991899199910E94AC
:10FF900070D3FE01E05BF109208131814281538100
:10FFA0000E9485CE0E9447D8688B798B8A8B9B8B69
:10FFB00082E1C83FD80739F7DF91CF910895CF93F9
:10FFC000DF9348E352E1052E000C660B770B8AE3C2
:10FFD00092E1092E000CAA0BBB0B841B950BA60B00
:10FFE000B70B64ED70E0681B790B0296885C9D4E40
:10FFF0004FEF50E02FEF30E06115710501F1DB01AB
:020000021000EC
:100000006531710510F0A4E1B0E06A1B7B0BFC01C7
:100010008A0F9B1FA1912A0F311D420F531FE81712
:10002000F907C1F7E32FFF27DF01A20FB11D9D01E3
:10003000E52FFF27DF01A40FB11DAD01DDCF832F19
:100040009927C52FDD27C40FD11DDC2FCC27820FA8
:10005000911DC82BD92BDF93CF938AED9BE0E091C4
:10006000DC0BF091DD0BEA5BFE4F21812F932081A9
:100070002F939F938F930E949E460F900F900F9007
:100080000F900F900F90CE01DF91CF9108950F93B5
:100090001F93CF93DF9308E312E1C4E6D0E0F801A9
:1000A00061918F01CE010E947BD62196CA33F1E087
:1000B000DF07A9F784DF08E312E1012E000C220B11
:1000C000330B4AE352E1052E000C660B770B401B05
:1000D000510B620B730B4C595F4FBC01CA01DF918E
:1000E000CF911F910F910C9489D64F925F926F928E
:1000F0007F928F929F92AF92BF92CF92DF92EF92B8
:10010000FF92CF93DF93CDB7DEB7E4970FB6F894A5
:10011000DEBF0FBECDBF80E1E8E0F4E0DE019196E6
:1001200001900D928A95E1F780E1E8E1F4E0DE01CB
:10013000519601900D928A95E1F780E1E8E2F4E0B2
:10014000DE01119601900D928A95E1F7CE0181961C
:10015000ACE3B2E19E012F5E3F4FAE014F5F5F4FB8
:100160005A01405D5F4FFC01C190D190E190F19048
:10017000CF01CD92DD92ED92FD92F901C190D19027
:10018000E190F1909F011C96CD92DD92ED92FC9250
:100190001F97F501C190D190E190F1905F01BD01F1
:1001A00068557F4FFB01C082D182E282F3828417BF
:1001B0009507C9F680E090E8ABEBB5E48093601258
:1001C00090936112A0936212B093631280936412B1
:1001D00090936512A0936612B093671280E090E846
:1001E000ABE3B5E48093681290936912A0936A120E
:1001F000B0936B1210925C1210925D1210925E120C
:1002000010925F1280E29EE4A0E0B0E08093F812CA
:100210009093F912A093FA12B093FB1210927C12F1
:1002200010927D1210927E1210927F1280E090E068
:10023000A0E2B1E48093701290937112A0937212B5
:10024000B093731280936C1290936D12A0936E1200
:10025000B0936F1280E090E0A0E0BFE3809374124F
:1002600090937512A0937612B093771280E090E08D
:10027000A0EAB1E48093781290937912A0937A1255
:10028000B0937B12109288121092891210928A12E7
:1002900010928B1210928412109285121092861274
:1002A0001092871210928012109281121092821274
:1002B0001092831282ED90E09093DD128093DC1215
:1002C0001092DF121092DE128CE390E09093E11214
:1002D0008093E01225EF30E03093E3122093E21296
:1002E0001092E5121092E4129093E7128093E612B6
:1002F00080E090E0A0E6B1E480938C1290938D12A0
:10030000A0938E12B0938F124DEB57E366E07EE31D
:100310004093941250939512609396127093971293
:1003200049AB5AAB6BAB7CAB0E94F6B480EB482E6A
:1003300083E8582E85E0682E84E4782E40929C1243
:1003400050929D1260929E1270929F120E94F6B47B
:10035000812C912C90E8A92E9FE3B92E8092A412B3
:100360009092A512A092A612B092A7122DECC22EC6
:100370002CECD22E2CE4E22E2EE3F22EC092AC1204
:10038000D092AD12E092AE12F092AF1280E090E007
:10039000A0E6B1E48093901290939112A0939212F0
:1003A000B093931249A95AA96BA97CA940939812BA
:1003B0005093991260939A1270939B120E94F6B414
:1003C0004092A0125092A1126092A2127092A312B7
:1003D0000E94F6B48092A8129092A912A092AA123A
:1003E000B092AB12C092B012D092B112E092B2129F
:1003F000F092B3128AE999E9ADEBB1E48093B412BB
:100400009093B512A093B612B093B7121092BC128B
:100410001092BD121092BE121092BF121092D01202
:100420001092D1121092D2121092D3121092D912AD
:100430001092D8121092B8121092B9121092BA12E9
:100440001092BB121092C0121092C1121092C212DE
:100450001092C3121092D4121092D5121092D6128A
:100460001092D7121092DB121092DA1210920D1322
:1004700010920C130E94F6B482DDE091DC0BF09137
:10048000DD0BE458FE4F608171818AED9BE0E496BC
:100490000FB6F894DEBF0FBECDBFDF91CF91FF90B6
:1004A000EF90DF90CF90BF90AF909F908F907F9014
:1004B0006F905F904F900C94D12ACF92DF92EF9281
:1004C000FF920F931F93CF93DF936C017A018B01FF
:1004D000C0E0D0E0CE15DF0589F0D8016D918D0127
:1004E000D601ED91FC910190F081E02DC6011995A6
:1004F000892B11F47E0102C02196ECCFC701DF9158
:10050000CF911F910F91FF90EF90DF90CF900895C2
:100510000E94AADBEF92FF920F931F93CF93DF937A
:10052000EC017B018A0188819981009729F02A8159
:100530003B8124173507F8F4B8016F5F7F4F0E94A5
:10054000C2DA009759F0998388831B830A832C8130
:100550003D81232B81F4FC0110820DC0888199819B
:10056000009711F00E94CECF198218821D821C8242
:100570001B821A8207C01D830C83B7018881998171
:100580000E94CFDBCE01DF91CF911F910F91FF90A1
:10059000EF900895FB01DC0111961C921E921396B8
:1005A0001C921E92129715961C921E9214978617F3
:1005B000970741F0608171816115710519F04481DF
:1005C0005581A8CF0895FC011182108213821282F6
:1005D000158214826115710549F0FB01019000201C
:1005E000E9F73197AF01461B570B94CF0895BF929F
:1005F000CF92DF92EF92FF920F931F93CF93DF93EF
:100600007C016B01EA0189012417350720F48D2F45
:10061000E901042F182F6FEB75E0C701D4DFD60175
:1006200014968D919C911597C817D907C0F580171E
:10063000910708F48C01D601ED91FC911197E00F20
:10064000F11FB08010824D915C91BA016C0F7D1F3B
:100650006115710559F0FB0101900020E9F7319710
:10066000AF01461B570BC70155DF13C0F70180814F
:100670009181009711F00E94CECFD70111961C9264
:100680001E9215961C921E92149713961C921E92FF
:100690001297D601ED91FC91E00FF11FB082C701D6
:1006A000DF91CF911F910F91FF90EF90DF90CF904E
:1006B000BF900895EF92FF921F93CF93DF93FC01B9
:1006C000208120FF32C0EC017C01F7E0EF0EF11C2D
:1006D0004B815C816D817E81E981FA819701808106
:1006E00091810E944C99182F811102C010E01EC008
:1006F000888181FD04C088818E7F888317C0E9814D
:10070000FA8144855585668577858B819C81AD818D
:10071000BE81480F591F6A1F7B1F970180819181FD
:100720000E944C998111E7CFE1CF11E0812FDF9139
:10073000CF911F91FF90EF900895CF92DF92EF92AB
:10074000FF921F93CF93DF93EC016A017B01122F7D
:100750008B819C81AD81BE8184179507A607B70761
:10076000E9F0CE01A7DF811103C080E090E01CC05A
:1007700012FF06C01882CB82DC82ED82FE820EC0A0
:10078000E981FA819E01295F3F4FB701A60180816F
:1007900091810E9495998111EDCFE7CF13708881E7
:1007A000182B1883CE010796DF91CF911F91FF90F0
:1007B000EF90DF90CF9008958F929F92AF92BF926B
:1007C000CF92DF92EF92FF920F931F936A017B010A
:1007D00048015901FC012581203249F54489558998
:1007E0006689778997018601E7E036952795179501
:1007F0000795EA95D1F7400F511F621F731F23E041
:1008000080969BDF009711F480E02CC0E894C7F835
:10081000DD24EE24FF24CC0CDD1CCC0CDD1CFC0103
:10082000EC0DFD1D80829182A282B3821AC020311C
:1008300059F7FC0144895589668977894D0D511D09
:10084000611D711D23E0809678DF0097E9F2DD24B9
:10085000EE24FF24CC0CDD1CFC01EC0DFD1D91826F
:10086000808281E01F910F91FF90EF90DF90CF90F9
:10087000BF90AF909F908F900895CF92DF92EF92AC
:10088000FF920F931F93CF93DF93EC016A017B01DB
:1008900089018D81803249F58C899D89AE89BF8916
:1008A000E7E07695679557954795EA95D1F7480F14
:1008B000591F6A1F7B1F22E0CE0180963EDF009702
:1008C00011F48FEF3FC0E894C7F8DD24EE24FF2435
:1008D000CC0CDD1CCC0CDD1CFC01EC0DFD1D808165
:1008E0009181A281B381BF701CC0803151F74C89C6
:1008F0005D896E897F894D0D511D611D711D22E03D
:10090000CE0180961ADF0097E1F2DD24EE24FF2469
:10091000CC0CDD1CFC01EC0DFD1D80819181A0E063
:10092000B0E0488D598D6A8D7B8D481759076A074D
:100930007B0738F0F80180839183A283B38381E041
:1009400001C080E0DF91CF911F910F91FF90EF9058
:10095000DF90CF9008959F92AF92BF92CF92DF9297
:10096000EF92FF920F931F93CF93DF9300D01F92CC
:10097000CDB7DEB75C016A017B019E012F5F3F4F5F
:10098000B701A601C50179DF982E87FF02C080E07C
:100990001DC000E010E09801B701A601C5010CDF01
:1009A0008823A9F3F5014085518562857385C416B6
:1009B000D506E606F70620F4C086D186E286F386E1
:1009C000C980DA80EB80FC809110D7CF0F900F9018
:1009D0000F900F90DF91CF911F910F91FF90EF90AB
:1009E000DF90CF90BF90AF909F9008952F923F924D
:1009F0004F925F926F927F928F929F92AF92BF922F
:100A0000CF92DF92EF92FF920F931F93CF93DF93DA
:100A1000CDB7DEB764970FB6F894DEBF0FBECDBF7B
:100A20008C013B01FA01418152815B874A87DB01DE
:100A30008C91807709F44EC3D8018C9181114AC3FF
:100A40008081837009F43AC38A859B850C966DE09A
:100A500070E00E9471DA6F5F6F83288BFE83ED83F5
:100A60001B8B0A8B40E050E0BA01C3010E947A94CC
:100A7000B12CA12CE12C10E0F12C00E0198ACD80E2
:100A8000DE80B6E0CB0ED11C5DE0952EF3018089AF
:100A90009189A289B3891C012D0145E056944794A0
:100AA000379427944A95D1F73986288661E0C301A7
:100AB0000E943E95009739F4D30111968C918823BA
:100AC00009F499C007C3FC012081253E11F02111D2
:100AD0000BC0F11002C0B22CA32CFF81FF1608F44A
:100AE000F394211106C087C03F81F31608F4E9C2D0
:100AF00002C0253EF1F12E32E1F1DC011B963C9162
:100B00001B973F3009F057C0011108C026FFBECF28
:100B1000022F0F711D96EC90102F07C0115021135A
:100B200028C0FC012585E21224C0412F50E041502D
:100B30005109949E9001959E300D11244A855B8544
:100B400024173507B0F4FC0160E0653018F48181AA
:100B5000928107C06B3018F48481958102C0868130
:100B60009781AA85BB852A173B0729F4892B09F4AD
:100B70008DCF00E08BCF8F3F910509F0D0F74FEB81
:100B8000480F4A3110F0782F02C070E2780FC90187
:100B90000196AD81BE8113964D915C911497DA0157
:100BA000A20FB31F2C913FEB320F3A3108F4205EB5
:100BB0007213DFCF88C233FDDCCF002341F0113048
:100BC00009F088C20E9467948E1184C210C04BE065
:100BD00050E0B6010E94AEDB892B09F057CFED81C2
:100BE000FE81808180FF03C0E1E0E98B4FCFF8896F
:100BF000F7FF5BC26FC288898274823409F06AC2CF
:100C0000FF2051F0B886A98607C060E0C3010E94AA
:100C10003E95892B29F0F394BF81FB16B0F3D3C026
:100C2000D30111968C91882309F4CDC053C2F301EE
:100C3000808185FD4FC280899189A289B389811500
:100C40009E4FAF41B10508F045C2D30112968C9179
:100C50001297806812968C9312971C962D903D9057
:100C60004D905C901F971696CD90DC9017972114AD
:100C700031044104510409F0ABC0D60118962D91FE
:100C80003D914D915C911B972C873D874E875F87E7
:100C90008C849D84AE84BF84BFEF8B1A9B0AAB0A01
:100CA000BB0AF601808D918DA28DB38D88159905B3
:100CB000AA05BB0528F432E0832E912CA12CB12C7F
:100CC0009E012F5F3F4FB501A401C601D6DD87FD10
:100CD00001C2882309F481C089819A81AB81BC81DA
:100CE000892B8A2B8B2B09F078C00FEF1FEF2FEF8A
:100CF0003FE0B501A401C6015FDD882309F4EAC124
:100D0000211431044104510409F472C09501840195
:100D1000B201A101C60150DD882309F4DBC1F30152
:100D200084869586A686B7860680F781E02D22E028
:100D3000821A9108A108B108048004C0880C991C8B
:100D4000AA1CBB1C0A94D2F780899189A289B38915
:100D5000880E991EAA1EBB1E25E0B501A401CF0175
:100D60008096EBDC8C01009709F4B4C1DC01E0E073
:100D7000F2E01D923197E9F7EE24E394F301C68087
:100D8000D780D60112968C91E816D0F190E0A0E0C1
:100D9000B0E029E0880F991FAA1FBB1F2A95D1F741
:100DA0004089518962897389840F951FA61FB71FD7
:100DB000808B918BA28BB38BD60112968C91823053
:100DC00080F5E0E1FE0EFF81FF1608F430CF29C068
:100DD0002C863D864E865F865BCF2C853D854E8575
:100DE0005F8582169306A406B50609F055CF72C139
:100DF000D60118968D929D92AD92BC921B978FCF83
:100E00009801B501A4014E0D511D611D711DD60142
:100E10008D919C910E944C99882309F45BC1E394C5
:100E2000ADCFB989BB2309F475C0AD81BE811596DC
:100E3000DC90159702E010E08EE7C82E7D01B6E049
:100E4000EB0EF11C41C0F3E0FD1510F473E0D72E5A
:100E500094E09D0D822F8F70E92FF0E08A3008F02A
:100E600052C0805D4D815E81E40FF51F868364E092
:100E7000369527956A95E1F79150D91658F3FA01FE
:100E8000ED0DF11DC68240E050E0BA01C3010E94A1
:100E90007A9461E0C3010E943E950097B1F1FC0194
:100EA00020812223B9F1238523FDF3CF4BE050E0CD
:100EB000BC01C7010E94AEDB892B59F70F5F1F4FA2
:100EC0000436110509F406C1ED81FE81418152818C
:100ED0009801240F351F0380F481E02D4E0F5F1F12
:100EE000E417F50709F4AFCFC901A5E0880F991FF2
:100EF000AA95E1F7280F391F8191082E000C990B54
:100F000028273927EDCF895CADCFD30111968C917D
:100F10008111E0C028853985A90160E070E025E0F5
:100F2000440F551F661F771F2A95D1F7C3010E94F2
:100F30007A94882309F4CEC00F810150A02E1FE0BF
:100F4000ED80FE8036E0E30EF11C9DE0B92EAA2074
:100F500009F460C060E0C3010E943E956C01892BDA
:100F600009F4B8C0D3011696ED91FC91179780A1B2
:100F7000816080A32A2DA01201C02064F601208385
:100F800013871486C7012C8B0E946794D6011D9687
:100F90008C931D975B961C921E925A97ED81FE8151
:100FA000438154812C892F7130E021503109B29E48
:100FB000C001B39E900D1124F60160E02A853B85A7
:100FC0008217930740F4DA01A80FB91F2C91022E63
:100FD000000C330B0CC021E030E0AA85BB858A17DA
:100FE0009B0711F420E030E03195219531096530FF
:100FF00018F43283218307C06B3018F435832483BF
:1010000002C0378326836F5F019632966D30B1F64A
:10101000AA949DCFF301408951896289738985E043
:1010200076956795579547958A95D1F7598748875B
:1010300060E0C3010E943E95009709F44BC020E296
:10104000DC011D922A95E9F7ED81FE8136962BE0B1
:10105000DC0101900D922A95E1F7ED81FE8120815E
:101060002871DC011C962C931C9721E238E25196E2
:101070003C932E93509740E058E01F965C934E931C
:101080001E9753963C932E93529759963C932E93CA
:10109000589757965C934E935697D3011696ED91B9
:1010A000FC91179780A1816080A328894885598584
:1010B000B3018A899B890E94A1950DC0B1E0BF83CD
:1010C000CCCCF12C18CD6F5F32966D3009F4DECCAC
:1010D0009C013BCD80E064960FB6F894DEBF0FBE56
:1010E000CDBFDF91CF911F910F91FF90EF90DF90D7
:1010F000CF90BF90AF909F908F907F906F905F90B8
:101100004F903F902F9008954F925F926F927F92F1
:101110008F929F92AF92BF92CF92DF92EF92FF9207
:101120000F931F93CF93DF93CDB7DEB7A1970FB681
:10113000F894DEBF0FBECDBF7C018B016A0119821E
:101140001A82DC018C91811103C0F801108204C065
:101150004D305105D0F302C070E0E8C0D7011396BE
:101160009C9191113BC0807631F08FE2D8018C9335
:1011700011961C9231C060E0C7010E9441967C012B
:10118000009751F3FC0148E090E020E05EE28081AE
:101190008032D1F0283039F4B801690F711DDB01BC
:1011A0005C939F5F40E130818FEB830F8A3130F495
:1011B000D7011C968C91842309F0305EB801690F29
:1011C000711DDB013C939F5F2F5F31962B30F9F649
:1011D000F801E90FF11D108271E0A8C0F7018085C8
:1011E0009185A285B385668177819E012F5F3F4FF0
:1011F00059010097A105B10539F4C9010E948795ED
:10120000882309F4A2CF0FC020E2F50111922A959C
:10121000E9F720E1298321E02B8378876F838D8F85
:101220009E8FAF8FB8A3772473949DE0692E280119
:101230004C0C5D1CF1E04F1A5108F70183818715B2
:1012400008F483CF872C912CD70114964D915C9193
:1012500015974819590960E070E085E0440F551F63
:10126000661F771F8A95D1F7C5010E947A94782F5F
:10127000882309F46ACF60E0C50179A30E943E95F6
:10128000FC0179A1892B09F460CF83858F3009F0A7
:101290005CCF80818F7190E08816990609F055CF58
:1012A000B1E08B1A9108689C9001699C300D112463
:1012B000C801820F931F4F0160E0D401653028F40C
:1012C00011964D915C9112970BC06B3028F41496D7
:1012D0004D915C91159704C016964D915C911797AE
:1012E0004115510591F02C153D05C8F42F5F3F4F76
:1012F0004F37510508F04FE3DC014D93CD016F5F8F
:10130000B2E08B0E911C6D30C1F62C153D0538F402
:10131000808186FF04C0D801A20FB31F1C92D201A6
:101320001C92808186FD02C0739487CF872FA1967F
:101330000FB6F894DEBF0FBECDBFDF91CF911F91E6
:101340000F91FF90EF90DF90CF90BF90AF909F9064
:101350008F907F906F905F904F9008958F929F92A3
:10136000AF92BF92CF92DF92EF92FF920F931F93B3
:10137000CF93DF93EC018C01000F111F000F111FA1
:10138000C8018953974E0E9420BD9801215A354FBC
:101390004901A80140585D4E6A01FA01208131815E
:1013A000428153810E94E7D6F40162837383848370
:1013B0009583C8018554974E0E9420BD9801235EF5
:1013C0003D4F5901F60120813181428153810E94B4
:1013D000E7D6F5016083718382839383C8018155C9
:1013E000974E0E9420BD98012F5E3D4F7901F60176
:1013F00020813181428153810E94E7D6F7016083C9
:10140000718382839383C230D105E0F48091210AF5
:10141000CC0FDD1FC80FD11DCC0FDD1FCC0FDD1F82
:10142000CC54DD4E288139814A815B81F40162818F
:101430007381848195810E94E7D6F401628373836E
:1014400084839583DF91CF911F910F91FF90EF904F
:10145000DF90CF90BF90AF909F908F9008958F9224
:101460009F92AF92BF92CF92DF92EF92FF92CF9373
:10147000C82F1092461481E090E0A0E0B0E0809385
:10148000491490934A14A0934B14B0934C1481E4E4
:1014900094E19093631480936214109261148FEF1F
:1014A0009FEFDC018093641490936514A0936614FD
:1014B000B0936714CC2329F1C53008F0DFC020E0D9
:1014C00040E050E0BA0181E694E137D9009709F491
:1014D000D5C020E1C29F800D911D11244097FC01D1
:1014E000E254FE4F20812F7709F0C8C038968080E3
:1014F0009180A280B38081149104A104B10421F4ED
:10150000BDC0812C912C540120E0B501A40181E6DD
:1015100094E113D9FC01892B09F4B0C0838594852B
:101520008115924009F0AAC08089823009F0A6C0D6
:1015300086859785892B09F4A1C0258520934314BE
:101540008FEF820F8093441480E091E0291751F0CF
:1015500031E0380F393019F4809345148FC0990F5A
:10156000832FF4CF80934514C688D788C114D10443
:1015700019F0E12CF12C04C0C4A0D5A0E6A0F7A07E
:10158000C0924D14D0924E14E0924F14F092501429
:1015900086859785A5019401280F391F411D511D8E
:1015A000DA01C9012093551430935614409357140F
:1015B000509358142189328930934814209347144A
:1015C000CC0CDD1CEE1CFF1CC80ED91EEA1EFB1E37
:1015D000C0925D14D0925E14E0925F14F092601499
:1015E0008189928935E0880F991F3A95E1F78150FA
:1015F0009E4F892F99278695C80ED91EE11CF11C94
:10160000C0925114D0925214E0925314F092541498
:10161000238934892115310521F0C901A0E0B0E00A
:1016200004C080A191A1A2A1B3A1B501A4014C194C
:101630005D096E097F09480F591F6A1F7B1F0090C3
:10164000451404C076956795579547950A94D2F747
:10165000DB01CA010196A11DB11D8093591490931D
:101660005A14A0935B14B0935C14453F3FE05307BA
:101670006105710528F48CE08093461480E017C062
:10168000453F5F4F6105710510F480E10DC084A5F1
:1016900095A5A6A5B7A580935D1490935E14A0931D
:1016A0005F14B093601480E28093461481E0CF9180
:1016B000FF90EF90DF90CF90BF90AF909F908F9072
:1016C00008950F931F93CF93DF93C4E6D0E008E310
:1016D00012E1CE010E946ED6F80181938F0121960E
:1016E000CA33F1E0DF07A9F71F9286ED8F93CAEDA9
:1016F000DBE0E091DC0BF091DD0BE258FE4F8181E5
:101700008F9380818F93DF93CF930E949E460E9498
:10171000DF7F8C0148E352E1052E000C660B770B4E
:101720008AE392E1092E000CAA0BBB0B841B950BDC
:10173000A60BB70B8C599F4F0E9476D60F900F9037
:101740000F900F900F900F9008171907B1F0E091CC
:10175000DC0BF091DD0BEC5BFE4F81818F93808180
:101760008F93DF93CF930E949E460E9475800E94C4
:1017700047800F900F900F900F900E94BF7FDF91D6
:10178000CF911F910F910C94F6B48F929F92AF92CC
:10179000BF92CF92DF92EF92FF92CF93DF93EC0153
:1017A0004A015B010E94E1C26B017C0183EB9AE07C
:1017B0000E94F749209761F0C130D10591F4109251
:1017C000500B1092510B1092520B1092530B11C0F0
:1017D00010924C0B10924D0B10924E0B10924F0B1F
:1017E00008C01092540B1092550B1092560B109289
:1017F000570BC501B40128EE33E040E050E00E94F1
:10180000ABD649015A0183EB9AE00E94D049A0E08F
:10181000B0E088159905AA05BB05E0F48091480B56
:101820008823A9F00E9428AD0E94E1C2DC01CB010F
:101830008C199D09AE09BF09813D9740A105B105ED
:1018400030F00E947CAA0E94E1C26B017C010E94E0
:10185000765CD9CF1092B40A1092B30A1092B70AEC
:101860001092B80A1092B90A1092BA0A1092BB0AE2
:101870001092BC0A1092BD0A1092BE0A1092B60ACB
:101880001092B50A209759F0219791F46091500B6E
:101890007091510B8091520B9091530B11C060913C
:1018A0004C0B70914D0B80914E0B90914F0B08C0DB
:1018B0006091540B7091550B8091560B9091570B82
:1018C000DF91CF91FF90EF90DF90CF90BF90AF90DE
:1018D0009F908F900895CF92DF92EF92FF920F9397
:1018E0001F9384E79AE00E9408BE0E94E1C26093C1
:1018F000DE0B7093DF0B8093E00B9093E10B209154
:10190000740A3091750A4091760A5091770A609175
:10191000610A7091620A8091630A9091640A0E9440
:101920006CD3811179C02091780A3091790A409165
:101930007A0A50917B0A6091650A7091660A8091DB
:10194000670A9091680A0E946CD3811165C020E0FB
:1019500030E040E752E46091840A7091850A8091FA
:10196000860A9091870A0E94D0D721E2C22E2AE0EF
:10197000D22E7B018C0120E83AE04CE75AE068E780
:101980007AE084E79AE00E94D0718091740A909185
:10199000750AA091760AB091770A8093610A9093B4
:1019A000620AA093630AB093640A8091780A9091C6
:1019B000790AA0917A0AB0917B0A8093650A909384
:1019C000660AA093670AB093680A80917C0A909196
:1019D0007D0AA0917E0AB0917F0A8093690A909354
:1019E0006A0AA0936B0AB0936C0A8091800A909166
:1019F000810AA091820AB091830A80936D0A909324
:101A00006E0AA0936F0AB093700A1F910F91FF9016
:101A1000EF90DF90CF9008956091290270912A0293
:101A2000072E000C880B990B0E9472D32091840A18
:101A30003091850A4091860A5091870A0E9485CE8E
:101A400020E030E040E752E40E94D0D720E030E0D0
:101A500048EC52E488CFAF92BF92CF92DF92EF92E0
:101A6000FF920F931F93CF93DF935B016A0179017C
:101A700008E312E1F8012481358146815781FC0198
:101A800060817181828193810E9485CE0E94DAD922
:101A9000C0EADCE06A837B838C839D83F801208528
:101AA000318542855385F501608171818281938101
:101AB0000E9485CE0E94DAD96E837F8388879987BA
:101AC000F8012485358546855785F6016081718149
:101AD000828193810E9485CE0E94DAD96A877B87B2
:101AE0008C879D87F8012089318942895389F701C4
:101AF00060817181828193810E9485CE0E94DAD9B2
:101B00006E877F87888B998B8FB7F8944A815B812A
:101B10006C817D81E0E1FAE04083518362837383CD
:101B20004E815F8168857985448355836683778399
:101B30004A855B856C857D85408751876287738781
:101B40004E855F8568897989448755876687778759
:101B50008FBF1AA21BA21CA21DA21A8A1B8A1C8A52
:101B60001D8A1E8A1F8A188E198E1A8E1B8E1C8E35
:101B70001D8E1E8E1F8E18A219A2F70180819181E1
:101B8000A281B38180930A0A90930B0AA0930C0A56
:101B9000B0930D0ADF91CF911F910F91FF90EF90BD
:101BA000DF90CF90BF90AF900895909136128091C2
:101BB0003712981719F00E94B3B3F7CF08952F92F8
:101BC0003F924F925F926F927F928F929F92AF92CD
:101BD000BF92CF92DF92EF92FF920F931F93CF931A
:101BE000DF9300D01F92CDB7DEB75C018FE5282EC2
:101BF0008AE0382E4501880C991C880C991C9401A8
:101C0000215A354F3C832B83F901128213821482AF
